S02B00002F686F6D652F62616D626F6F2F62616D626F6F2D6167656E742D686F6D652F786D6C2D646174612F36
S31508004000C00200200DC30108130902080B090208A3
S31508004010A70A090100410008040E03AC5010180253
S315080040200000000000000000000000000000000082
S315080040300000000000000000000000000000000072
S315080040400000000000000000FFFFFFFFFFFFFFFF6A
S31508004050FFFFFFFF00E00708000000000000080857
S31508004060FFFFFFFFFFFFFFFFFFFFFFFFFFFFFFFF52
S31508004070FFFFFFFFFFFFFFFFFFFFFFFFFFFFFFFF42
S31508004080B2F90020C0020020B2F90020B2F90020DF
S31508004090C0020020125F030802EA0208C0000020DE
S311080040A09800002000000808B2F9002073
S31508004100C00200200DC30108130902080B090208A2
S315080041100B0902080B0902080B0902080B09020819
S315080041200B0902080B0902080B090208B19C0108D1
S3150800413027C301080B090208A59C010845BE01080A
S315080041400B0902080B090208498901080B0902082C
S315080041509DA70108850A02088B0A02080B090208AE
S31508004160619B0108219201085D8E0108B5F40108DA
S315080041703D0A0208430A0208490A02084F0A0208C9
S315080041800B090208910A0208930A02080B09020899
S31508004190074B19680868B0E8F00F80F30988BFF381
S315080041A06F8F4FF0000080F311884EF00D0E7047A8
S315080041B0C8F10020AFF30080AFF30080AFF30080B2
S315080041C038B50D4D0020296801F024FA0B4B032160
S315080041D018681CF0EBFA04462968012001F01AFA5F
S315080041E044B1636833B100212046BDE838400A4629
S315080041F01CF028BB38BD00BFF8ED002074EE002087
S3150800420008B50948782100F0C7F8084A106048B18F
S3150800421001F014FC30B101F0C5F9054B1860FFF741
S31508004220CFFFFCE708BD00BFFCED002074EE0020C0
S31508004230F8ED00201FB500F035F80020014600F023
S3150800424079F901F073FB032200238DE80C00084B73
S3150800425008490293084A4FF48053084800F050F87A
S315080042601CF099FA05B05DF804EB1CF093BA00BF90
S31508004270E0ED0020601E0308C0020020014200088D
S3150800428070B51E46064C049D20681CF0C2FA3046DE
S31508004290294618F011FF2068BDE870401CF0C6BA20
S315080042A078EE002008B52AF09DF91CF0AFFA054B08
S315080042B000211860044800F03DF9BDE808402AF0DE
S315080042C0F2B900BF78EE00208142000837B50446EF
S315080042D045691AF02BF923680246606100940120AB
S315080042E0064900F015F96069214619F0C7FF2B4603
S315080042F0206903B0BDE83040184700BF6B1E0308AD
S315080043002DE9F043984687B0530781460C46154673
S315080043100E9F109E03D01B4825211CF0D9FAE6B142
S3150800432004B3052F21DC0F9B86E830013361F76063
S31508004330C6F8149005AB02950025019300970395DE
S3150800434011482146C8F38F02334619F0FBFC0128B1
S3150800435013D06FF47A75224609E00C4A002C18BF70
S31508004360224603E00A4D094A01E02246084D009517
S31508004370012008493B4600F0CBF8284607B0BDE8BF
S31508004380F08300BFB11E0308CD4200089D1E030836
S3150800439018FCFFFFC31E030870B50D4606468908BC
S315080043A088B181B10422002319F058FA0446042082
S315080043B01CB9094932462B4602E0224633460749CC
S315080043C000F0A6F806E00420054932462B4600F020
S315080043D09FF80024204670BDF61E0308261F030812
S315080043E03E1F030870B588B008AB43F80C1D0022C1
S315080043F019461346054619F065FA01283AD0059C70
S3150800440026881CF0CAF918B11CF0C7F9036800E041
S315080044101A4B32460193042023461949009500F0A9
S3150800442077F80420174900F073F81AF04BF90024BE
S31508004430002208A941F8042D2846134619F06AFBFC
S3150800444001280ED1079B04201A880F4900925A6842
S3150800445001929A6802922246013400F059F8402CDB
S31508004460E6D11AF03DF9094892211CF031FA6FF4A9
S315080044707A7000E0002008B070BD00BF6E1F030808
S31508004480731F0308B01F0308DC1F03081620030860
S315080044901FB504AB43F80C1D194603AA002319F0EF
S315080044A0EDFA012806D00848B4211CF011FA6FF479
S315080044B07A7000E00020039B1BB1044B4FF080523A
S315080044C01A6005B05DF804FB1620030804ED00E049
S315080044D037B5044610460A4A0B46156875B1072CC7
S315080044E08BBF0849084A0919125D88BF11F8082CBC
S315080044F022B10649009008682146A84703B030BD96
S3150800450080EE0020482600204E2600207CEE002063
S315080045100EB4074B03B51B6823B104AA039901928D
S31508004520FFF7D6FF02B05DF804EB03B0704700BF93
S3150800453080EE0020024B1860024B1960704700BFDE
S3150800454080EE00207CEE00200346890541EA93218F
S315080045508005024A4FF07A431CF08BB92FDD2406FA
S3150800456038B504460025012020806160A260E3601A
S3150800457025746574A574E57404F1140002492A4685
S315080045801CF0CBF9656238BD9508020838B5456A4E
S31508004590044645B11CF001F9854204D00B4840F2A7
S315080045A01A211CF095F90123637404F1140000F034
S315080045B0F9FB50B1E0682146FFF714FF28B904F16A
S315080045C01200BDE838402AF058B838BD2E20030836
S315080045D0F8B5466A04460D4617461EB91CF0DDF8BE
S315080045E0606208E01CF0D9F8864204D00C4840F214
S315080045F0EF111CF06DF92046FFF7C8FFA37C27745E
S31508004600E374002363741434204606492A461CF0D2
S3150800461084F920462946BDE8F84000F0A9BB00BF4A
S315080046202E2003089508020838B5456A04461CF08A
S31508004630B4F8854204D00D484FF411711CF048F9BE
S31508004640A37C23B9094840F24B211CF041F904F137
S3150800465012002AF01DF8E37C1BB1013BE37400202D
S3150800466038BD607C80F0010038BD00BF2E200308ED
S3150800467070B58CB005460E4629F0DBFD01A9044647
S315080046800A22304618F064FD01A829F0D2FDC0F1CF
S315080046901E00844282BF241A2D1904462946224642
S315080046A004A829F0E1FD0CAB2344202203F8202CB2
S315080046B0601C04AB1844C4F11F0201A929F0D4FDFB
S315080046C004A9062000F026F829463246024829F0B1
S315080046D087FD0CB070BD00BF4020030810B50A4B1B
S315080046E00A4C58601C60441F032C0BD89C68012C8C
S315080046F000D03AB1986029B1BDE81040044820229C
S3150800470029F0B2BD10BD00BFC0120020CDAB3412D7
S3150800471014130020044B1A68044B9A4202D0002254
S31508004720FFF7DCBF704700BFC0120020CDAB3412C4
S3150800473010B5054C002104F108004FF4057229F064
S31508004740E9FD0123A36010BDC01200200B4910B576
S315080047508B680446053B032B0AD808314FF40572CB
S3150800476018F084FC2368053B032B04D9FFF7E0FF08
S315080047704FF0FF3010BD002010BD00BFC012002052
S31508004780054B064A1968914204D15868082801D889
S31508004790C0B2704701207047C0120020CDAB34125A
S315080047A01E2809D8054B11F8012B0130034483F85C
S315080047B053200B78002BF3D1704700BFC01200209E
S315080047C010B50A4904460020FFF7EAFF034634B14C
S315080047D00749FFF7E5FF2146FFF7E2FF0346054ACB
S315080047E01344002283F8542010BD00BFEC200308B0
S315080047F0FB200308C0120020F0B5054687B00F4617
S315080048001C460AB9284806E0012A01D1274802E0D1
S31508004810022A02D1264829F0E3FC2648C16A826AA0
S31508004820436B866B006B00960190234829F0D8FCF1
S315080048300026314655F826202048013629F0D0FCB6
S31508004840042EF6D10026311D57F826201C480136BD
S3150800485029F0C6FC082EF6D11A4B02AE0FCB86E815
S315080048600F000C35002756F82710174855F8042F5F
S31508004870013729F0B5FC042FF5D12146134829F054
S31508004880AFFC00F07DFBAFF30080114829F0A8FCCF
S31508004890251F3C3455F8041F0E4829F0A1FCA542F3
S315080048A0F8D107B0F0BD00BFAA210308BC21030850
S315080048B0C621030800ED00E08C200308DE2103086A
S315080048C08B21030838EA0208722103087E210308AF
S315080048D098210308A32103082DE9F3410D4606464E
S315080048E01F46904600F030FE0A2301930095B069F2
S315080048F071693A46089B29F0D3F9044628B19DF810
S315080049002430082B13D1022811DCB3692B60736994
S315080049106B6000F019FE032210238DE80C00384660
S31508004920089905F10802082329F0FCF9841CC8F83F
S31508004930004000F009FE0026A64206D055F82610CB
S31508004940034829F04DFC0136F6E702B0BDE8F081D0
S31508004950B12103082DE9F0410E461746804619F0A5
S31508004960E5FD044619F022FB05460B48294629F0C1
S3150800497037FCC8F800501CB120461BF0AEFF386063
S31508004980064B9B6ADB0604D5054829F029FC082353
S315080049903370BDE8F08100BF6120030800ED00E038
S315080049A0FE20030808B50448202100F065FEBDE88E
S315080049B0084000F04FBE00BF141300202DE9F8434D
S315080049C0234C9846A3680546012B8946174601D00D
S315080049D0062B19D19DF8243033B11E480021302208
S315080049E029F098FC1C4E00E01C4E002128221B488A
S315080049F029F090FCFFF7C4FE012807D100212022E8
S31508004A00174829F087FC01E0164E1DE029461022BA
S31508004A10154818F02BFB15484946202218F026FBA6
S31508004A202B69072FE3636B69C4F840806364AB693D
S31508004A30A364EB69E36402D1FFF7B4FF04E0082F2F
S31508004A4002D10898FFF7BCFE3046BDE8F88300BFE0
S31508004A50C01200205C1300206013002034130020CD
S31508004A601413002084EE0020CC120020DC12002053
S31508004A702DE9F041904604460F4686B0002301F121
S31508004A802406039304930593C369861B18BF01265E
S31508004A909A0500F1200548BF00F12405B8F1020F78
S31508004AA096BF224B052313F808308DF80B3000F01B
S31508004AB04BFD1BF06CFF2046394642462B46FFF756
S31508004AC09BFE36B104A80DF10B0105AAFFF742FFBC
S31508004AD004E0174829F084FB164B0593049B9DF8C0
S31508004AE00B208DE8480039462B462046FFF766FF1F
S31508004AF0059B014600939DF80B302046019303AAB7
S31508004B002B46FFF7E9FE0C4B1B68DB0704D50B4861
S31508004B1029F066FB00BE06E0094829F061FB9DF80E
S31508004B200B0000F0B1F906B0BDE8F0816F2103086B
S31508004B30C0200308C0020020F0ED00E0B6200308FC
S31508004B40E12003082DE9F341884604461BF0C5FE1B
S31508004B50074629F02EFD00F0F7FC1BF018FF334836
S31508004B6029F03EFB4146324829F03AFB2468314D8C
S31508004B70E36B04F140069905AB6848BF04F14406A7
S31508004B80012B01D0062B2DD1002130222A4829F0ED
S31508004B90C1FB236A2948EB60636A20212B61A36A5B
S31508004BA0274A6B61E36AAB612368EB6163682B6232
S31508004BB0A3686B62E368AB622369EB6263692B6384
S31508004BC0A3696B63E369AB63236B2E64EB63636B67
S31508004BD06B64A36BAB64E36BEB64434629F01CFB85
S31508004BE0184D00E0184D0A2301930095A06B616BE0
S31508004BF032463B4629F054F802280ED803221023E1
S31508004C008DE80C0030460823394605F1080229F0DC
S31508004C1089F8A36B2B60636B6B600C4829F0E0FA8C
S31508004C20082002B0BDE8F04100F02EB96C20030858
S31508004C30B2200308C01200205C13002014130020C1
S31508004C40522103086013002084EE00206421030823
S31508004C50094B1B682BB1834201D0DB68FAE70123B5
S31508004C6006E0064B1B681BB18342F8D0DB68FAE7FF
S31508004C7003F00100704700BFACEE0020B4EE002040
S31508004C80104B70B505460C461E68FFF7E1FF18B1D4
S31508004C900D48D52129F078FA002C08BF01243444A0
S31508004CA0B4428CBF094B0A4BAC601A6832B19168A2
S31508004CB08C4203D302F10C03D268F7E71D60EA6061
S31508004CC070BD00BFB0EE0020EB210308ACEE00205B
S31508004CD0B4EE002070B506460C4600F0B9F8144B41
S31508004CE0144D1B685BB19B682A68934205D99B1AC9
S31508004CF02268934203D2236001E0002400E00124E5
S31508004D0019F048F92B683060834203D20A48A72174
S31508004D1029F03AFA2B6832689B1A032B03D90648FE
S31508004D20AB2129F031FA00F09BF8204670BD00BF90
S31508004D30ACEE0020B0EE0020EB21030838B505469E
S31508004D4000F086F819F026F9A842044603D2064868
S31508004D50BF2129F019FA054B1868401B04441C604A
S31508004D60BDE8384000F07CB8EB210308B0EE00201F
S31508004D7038B5044608461BF02EFD2368054623B9B8
S31508004D80074840F2211129F0FFF900F061F82046A2
S31508004D902946FFF775FFBDE8384000F061B800BF47
S31508004DA0EB21030810B5044600F052F80D4A1368C3
S31508004DB03BB1A34201D1DB680CE003F10C02DB68CE
S31508004DC0F6E7094A01E003F10C0213682BB1A34286
S31508004DD0F9D1E3681360012400E01C4600F040F8AE
S31508004DE0204610BDACEE0020B4EE0020154A70B582
S31508004DF01368154D5E1C9E4216601ED229462B6806
S31508004E002BB100229A6003F10C01DB68F8E70F4A20
S31508004E1010680860136010E0A3689E4210D30A4B1E
S31508004E20E26820461A6061682368984728B11BF033
S31508004E30D2FC411E2046FFF723FF2C68002CEBD13D
S31508004E4070BD00BFB0EE0020ACEE0020B4EE00202E
S31508004E5072B6024A1378013313707047FFF50020C3
S31508004E6010B5074C23781BB90648512129F08CF94F
S31508004E702378013BDBB2237003B962B610BD00BFCD
S31508004E80FFF50020F721030810B504460021FFF7B7
S31508004E9041FC20461BF017FE023CE4B2052C96BFE7
S31508004EA0034B002033F81400BDE8104013F01CBD76
S31508004EB0F01B030838B50F4C2378CBB90E4D0123E8
S31508004EC023702B68590713D1FFF75AFC012801D024
S31508004ED020700DE0094B9B685A1F032A07D92B68D7
S31508004EE01A0701D5072302E0DB0601D50223237042
S31508004EF0207838BDFEF500204CEF0020C0120020B7
S31508004F0008B51B4B1A681B4B1A60FFF7D3FF13F043
S31508004F1091FA0820002100F0F1FC0220002100F09F
S31508004F20EDFC0320002100F0E9FC0120002100F03F
S31508004F30E5FC0020014600F0E1FC0720002100F016
S31508004F40DDFC0620002100F0D9FC0021042000F039
S31508004F50D5FC1BF0E9FC18F0E7F800F025FA28F074
S31508004F60CFFFBDE808400448044900221BF0D5BC21
S31508004F702C0000404CEF00203CEF002025090208D9
S31508004F8008B51E4829F02CF91D4B1E48196829F04A
S31508004F9027F91D4B1D48196829F022F91C4B1D4895
S31508004FA0196829F01DF91C4B1C48196829F018F9CD
S31508004FB01B4B1C48196829F013F91B4B1B48196829
S31508004FC029F00EF91A4B1B48196829F009F91A4BEA
S31508004FD01A48196829F004F9194B1A48196829F06A
S31508004FE0FFF8194B1948196829F0FAF8184B1948A7
S31508004FF0D968BDE8084029F0F3B800BF04220308C1
S3150800500048A80040162203084CA800402A22030894
S3150800501008A800403E2203080CA8004053220308B3
S315080050204CC800406822030850C800407E22030886
S3150800503044C80040942203084CC00040A922030833
S3150800504050C00040BF22030844C00040D5220308D0
S31508005050F0ED00E0EA2203081FB5019001A902A8B5
S31508005060FFF738FED0B1184B1B68BBB900F092FAAF
S3150800507088B903A800F076FA68B1039B002B04DC14
S31508005080124840F2452129F07FF80399104801F5A6
S315080050907A71FFF76DFE019814F088FF0298FFF702
S315080050A04DFE03A800F05EFA50B1039B002B04DA0C
S315080050B0064840F2562129F067F80548FFF772FEC0
S315080050C005B05DF804FB00BFB8EE0020F721030821
S315080050D03CEF002018232DE9F04F434315465D4A5F
S315080050E085B002EB03090446D9F80860904612F821
S315080050F003A0002900F0828099F80400012100F03D
S31508005100FDFB54236343544F5046F95A07EB030BF0
S3150800511064235943514B4A00B3FBF2F2B3FBF1F354
S3150800512092B2A3EB4203B266F3660223F365122139
S3150800513000F0E4FA99F80100112100F0DFFA9BF873
S315080051400230BA4613F0020F0DD0F36D122143F068
S315080051506003F36599F8030000F0D0FA99F80200A5
S31508005160082100F0CBFA4DB9542303FB04A383F8B6
S315080051704450DD6483F8455083F84350384B012783
S3150800518077651F60182303FB0488D8F80C2013687A
S315080051903B431360D8F81030324A1F6098F905303F
S315080051A0A2F5C07207FA03F3C2F880311360002D26
S315080051B04DD0542303FB04A39B6C002B47D06846B1
S315080051C014F060FF9DF80330009A1B063FD50023B4
S315080051D0029380238DF80B3098F8013007FA03F311
S315080051E0134202D1029B9A4231D12046542707FB2B
S315080051F004A7BB6C05B0BDE8F04F1847504600F051
S31508005200C5FA45B9144A542303FB042399F8010047
S315080052109D6400F0BBFA182303FB0484E07800F0D1
S31508005220B5FAA07800F0B2FA94F905200123934064
S315080052300D4A20791360E2680021136823F0010300
S315080052401360716505B0BDE8F04F00F057BB05B0B7
S31508005250BDE8F08F6CEA020850EF002000366E01B8
S3150800526008A8004080E200E080E100E010B5542381
S315080052704343064AD418D35A3BB101210A46FFF7DD
S3150800528029FFA3786FF30413A37010BD50EF002015
S315080052902DE9F7433F4F182303FB00730546002407
S315080052A03D48019403F10802D3F808C0036813F0D7
S315080052B0010351D0D2F804E0DEF8003013F0010300
S315080052C04AD0364E542202FB056292F8443092F8D0
S315080052D04510DBB2C9B28B4202F1400219D192F8ED
S315080052E0038008F0FF09B8F1000F03D0D4704FF01F
S315080052F0FF340EE04C460CE002F03F0888450FD01C
S31508005300542202FB0533DCF83C90334483F80390BF
S315080053104346DCF8482012F0020F03F10102EBD1F4
S3150800532002F03F024FF0010C8A42C0F800C005D1D6
S31508005330DEF8002022F00102CEF80020542202FBFB
S315080053400566DBB286F84430F36C48362BB1E8B212
S3150800535098470023736000E01C46182303FB057773
S3150800536097F90520012393400D4A13604CB10B4B66
S31508005370542202FB05350021286D01AA0B4618F0B8
S315080053807DFB019B1BB1074B4FF080521A6003B09F
S31508005390BDE8F0836CEA020808A8004050EF002038
S315080053A080E200E004ED00E0002008B501210323B7
S315080053B0024618F053FA014B186508BD50EF002055
S315080053C0164A182303FB002330B59C68636D13B394
S315080053D00A29134D09D1542303FB00539B7813F074
S315080053E0010F0CBF0A220D2200E00A46542303FBD4
S315080053F00050837803F00803DBB2A06C4507FCD5A0
S31508005400E26313B1A06C4006FCD58A4201D00A4675
S31508005410F3E7012030BD4FF0FF3030BD6CEA0208DB
S3150800542050EF00200D4B182202FB003291681A46F5
S315080054308B6C5B06FCD50A49542303FB001393F8CF
S315080054404510C9B283F84410182303FB0020C2682C
S315080054500120136843F00103136070476CEA0208E1
S3150800546050EF0020F8B5542343431A4D0646EB5A2D
S315080054700F464BB14FF47A71FFF7D4FF014618B9BE
S3150800548030460A46FFF726FE3C686423B4FBF3F26F
S3150800549003FB1244D4B9B2F5803F17D254237343A1
S315080054A0E918EA523A798B78C2F3400062F30003AE
S315080054B060F34103C2F3800262F382038B703046C5
S315080054C001212246FFF706FE2046F8BD6FF01500BB
S315080054D0F8BD00BF50EF002070B5542242430D4B73
S315080054E0044699189A5A1D469AB10B4A182303FB83
S315080054F000239E688B78DA0601D5FFF7B7FEB36CF2
S315080055005B06FCD5542303FB0454A37843F0080335
S31508005510A37070BD50EF00206CEA020810B5084C65
S31508005520238863B1074B9B6C5B06FBD500200146BD
S315080055300122FFF7CFFDA37843F01003A37010BD37
S3150800554050EF002000C8004008B5044B01221A603D
S3150800555018F020FD024B186008BD00BF0860004027
S31508005560ACEF0020094B10B50446186810F001008E
S315080055700BD018F00FFD064B1B68C01A28F0A0FCCC
S31508005580C0F5ED6004302060012010BD00600040C9
S31508005590ACEF0020024B1868B0FA80F0400970475B
S315080055A0A4EF002010B5FFF753FC064B18781F2808
S315080055B09BBF0446421C4FF0FF341A70FFF750FC9D
S315080055C0204610BD00F6002038B50E4B05461B7860
S315080055D00D4C984211D2FFF73BFC01232268AB40E1
S315080055E00A4D22EA03032A682360134203D1FFF710
S315080055F0ABFF2B682360FFF733FC2268044B1A6065
S3150800560038BD00BF00F60020A8EF0020A4EF002058
S31508005610DC14002038B50D4B05461B780C4699421C
S3150800562012D2FFF715FC0A4A0123A34011680DB1EF
S315080056300B4301E021EA03031360FFF711FC204640
S31508005640BDE83840FFF7C0BF38BD00BF00F60020F0
S31508005650A4EF0020044B05481978054B1A68054B3A
S315080056601B6828F0BDBD00BF00F60020F82203081D
S31508005670A4EF0020A8EF002007B5074A074B1268D9
S315080056801B780092064A12680192064A28F0C4FD61
S3150800569003B05DF804FB00BFA4EF002000F600206D
S315080056A0A8EF0020502303080048704784EA020840
S315080056B0F8B506460C4B012413F930300B4904FAA9
S315080056C003F50B4BB4401D600C234343CA185768B7
S315080056D0C8589168C0B2B847064B1C60064B1D6097
S315080056E0A3F5C0731D60F8BD9CEA0208B0EF002060
S315080056F080E100E014A8004080E200E02DE9F84FC0
S31508005700C5086D0200F0030700F0070B05F1804697
S31508005710BF004FF00F0823280C4606F530464FEA1F
S315080057209B0ADFF8649008FA07F803D91548782128
S3150800573028F02AFDFFF78CFB56F82A20012155F898
S315080057400900C4F3430301FA0BF104F0010420EA4B
S31508005750010122EA0808BB40FA4004FA0BF4D20712
S3150800576048EA030344EA01044BBF46F82A3045F8E1
S31508005770094045F8094046F82A30FFF771FB002032
S31508005780BDE8F88F742303080CB00040014B195C80
S31508005790FFF7B4BF7D230308064B82B01B88ADF81C
S315080057A0043002AB002918BF013313F8041C02B0F9
S315080057B0FFF7A4BF72230308232838B5044600F070
S315080057C0070503D90548B62128F0DEFC044BE40892
S315080057D06402E058284100F0010038BD742303082C
S315080057E008B00040F8B5C5086D0200F0070605F1D7
S315080057F0804303F53043B20853F8224000F0030310
S315080058009B001C4123280F46E4B203D90A48CC2141
S3150800581028F0BAFC04F00B04012C09D10FB1074B90
S3150800582000E0074B01222B44B2401A600020F8BD65
S315080058304FF0FF30F8BD00BF7423030810B00040D6
S3150800584014B000402DE9F04104460D4690461F4627
S31508005850FFF7FEFA082C05D00E2C07D1224B0121A2
S315080058605D6625E0204B00211D6621E01F2C05D929
S31508005870FFF7F6FA4FF0FF30BDE8F0811B49CB6918
S3150800588033B9194B02219D6603F5A1531C600FE03D
S315080058908B6A3BB9144B0321DD6603F5A153043328
S315080058A01C6005E0FFF7DCFA6FF00100BDE8F08147
S315080058B00C2048430E4B0D4E03EBC10234503518ED
S315080058C050680C4AC5F80480AF60106013F931209F
S315080058D001239340084A1360A2F5C0721360FFF7CC
S315080058E0BFFA0020BDE8F08100A80040B0EF002014
S315080058F09CEA020814A8004080E200E0B1FA81F1AF
S3150800590038B50546490901FA00F4FFF7A1FA064A2F
S3150800591001211368A94023EA010121431160BDE86A
S315080059203840FFF79DBA00BF3840004010B5FFF772
S31508005930E7FA16490020FFF795FD4FF4806014F04A
S31508005940FBF919F0A3FD19F08DFF19F09FFC04204F
S3150800595018F04AF8044618B90D48AB211AF0B8FFF2
S31508005960234600200B490C4A19F06CFC012018F05C
S315080059703BF8044618B90648B0211AF0A9FF224692
S31508005980BDE810400548064919F04EBC95230308A2
S315080059909A2303086F0A02085D0A0208590A0208D0
S315080059A0550A020810B502460B460B48962117F011
S315080059B08BFB9528044602DC00280ADD00E09524C6
S315080059C022460020044910F0FDFC002818BF4FF0BD
S315080059D0FF34204610BD00BF01F600200FB407B5FE
S315080059E0044805A90191FFF7DDFF03B05DF804EB54
S315080059F004B07047C223030800B50D4BADF5077D0B
S31508005A001A788AB9012201A81A70FEF79FFE30B9E2
S31508005A10019B062B03D1074814A9FFF7DFFFFEF702
S31508005A2087FE054B00221A600DF5077D5DF804FB1D
S31508005A3098F60020C2230308C012002030B5224D74
S31508005A4085B0286000F0B8FE204C206010B90A2006
S31508005A501F4905E028681AF0D3F820B11D490A2025
S31508005A60FEF756FD2DE0206828F09FF86B461A4A87
S31508005A701068516803C32068194600F06FFD684630
S31508005A8002A9082228F004FC18B1206802A91BF014
S31508005A90CCF9206810F0F8FF10480021FEF74AFDFF
S31508005AA020680F4900221BF0C1F810B10A200D49E1
S31508005AB0D6E700F06BFB10B10A200B49D0E7FFF7D9
S31508005AC09BFF206805B030BDE0EF0020E4EF002022
S31508005AD0D0230308F1230308BA230308C90A0208D6
S31508005AE0356200080D24030839240308014B186899
S31508005AF0704700BFE0EF002010B5BFF35F8F0E4B75
S31508005B00D3E84F2F511CC3E8401F0028F8D112F0E4
S31508005B10FF0FBFF35F8F0DD1084B09491868FEF7D1
S31508005B2061FC034630B1BDE810400A200549064A23
S31508005B30FEF7EEBC10BD00BF97F60020E0EF002090
S31508005B40BCEA020862240308AF240308054B10B513
S31508005B501A681C461AB90A200349FEF7D9FC2068B8
S31508005B6010BD00BFE4EF00208724030838B50546BA
S31508005B70FFF7ECFF044640B3154B9D4211D14FF099
S31508005B800002BFF35F8F134BD3E84F1FC3E8402FC4
S31508005B900028F9D1BFF35F8F642520461BF050FA21
S31508005BA038B920461BF04CFA78B12046FFF7A4FF17
S31508005BB00BE020461BF03FFAFFF7C8FF044620B16A
S31508005BC0013D15F0FF05ECD0E7E7002038BD00BF22
S31508005BD0BCEA020897F6002001460822014817F099
S31508005BE045BA00BFA3F6002038B50546FFF7AEFF55
S31508005BF0044698B10A4B1A784AB901221A70FFF777
S31508005C0075FF0849034622460748FEF7A9FC2946B8
S31508005C10BDE8384004480022FEF7DABC38BD00BFAC
S31508005C20ABF600204561000824F0002008B50748B7
S31508005C30FEF7ACFC08220648002128F06BFB054A53
S31508005C4000231360044A137008BD00BF24F0002027
S31508005C50A3F6002020F0002099F600202DE9F04751
S31508005C60B4B0054688461446FFF770FF0646002876
S31508005C7000F0008100212C220DA828F04BFB3046AD
S31508005C801BF0CFF88146002110220DA828F042FB10
S31508005C90FE2349468DF83430082280230FA88DF854
S31508005CA0353017F0E3F99DF83C30214683F00203BE
S31508005CB0102211A88DF83C3017F0D8F944F64C5349
S31508005CC06E4C4FF0010A27684946ADF85630ADF8D4
S31508005CD054300822FF2309A88DF859308DF858A0AA
S31508005CE017F0C4F93B0E8DF82C303B0C8DF82D308F
S31508005CF08DF82F703B0A18AF8DF82E300DA90523A5
S31508005D00102238468DF8303017F0B0F910221CA84A
S31508005D1011A917F0ABF90D238DF880302368042DEF
S31508005D204FEA13228DF882204FEA13428DF881300C
S31508005D308DF883204FEA136253448DF8842023603C
S31508005D408DF885A08DF88650A1460ED80AFA05F377
S31508005D5013F0170F09D000238DF887A08DF888A0B7
S31508005D608DF889300DF18A0401E00DF1870405F1FB
S31508005D70FF3ABAF1010F0BD8B8F1000F46D0042349
S31508005D80082223706270A01C414617F06FF90A3486
S31508005D90022D08D80323082223706270A01C3849F4
S31508005DA017F064F90A34BAF1010F11D805232370E4
S31508005DB004236370D9F8003006341A0E04F8042C4C
S31508005DC01A0C04F8032C1A0A04F8022C04F8013CED
S31508005DD000232C495A5C1AB90133082BF9D10AE079
S31508005DE0BAF1010F07D88323082223706270A01C1A
S31508005DF017F03CF90A344DB9022323700423637063
S31508005E00F023A570E57025716371063400F006FA73
S31508005E100D23E51B8DE888002623EDB202930DF1CC
S31508005E20860303930493A5F12603DBB201270593A2
S31508005E3007941021042209AB069700F05FFC304650
S31508005E4000211BF0D9FA223DEDB2044690B134A9DF
S31508005E50002301F8AD3D3A461BF07AF850B92046C2
S31508005E6020A9AA1D1BF074F820B9074821460DAAD7
S31508005E701BF0E2FA34B0BDE8F08700BF20F000203E
S31508005E809BF60020A3F60020E8EF00202DE9F04F4E
S31508005E900846B1B00C4691461BF046F80546204622
S31508005EA01BF044F8281A80B24F2800F226812046B3
S31508005EB01BF03CF80DF12B020146012320461BF08E
S31508005EC049F89DF82BA0BAF1000F40F0168120463C
S31508005ED01BF02CF8411C89B220461CAA50231BF043
S31508005EE039F8A0F10B05ADB2442D0DF150088346E3
S31508005EF000F203819DF870C0BCF10D0FCDF824C0E7
S31508005F0040F0FB809DF871309DF8724003EB042445
S31508005F109DF8733004EB03439DF8744003EB046467
S31508005F209DF87530012B40F0E88009F118073946CD
S31508005F3008220CA817F09AF89DF830300CA983F0BF
S31508005F400203082210A88DF8303017F08FF8230EB8
S31508005F508DF84830230C8DF8493009F11006230ACC
S31508005F608DF84A3031460523102240468DF84C30CC
S31508005F708DF84B4017F07AF84946102218A817F002
S31508005F8075F800F04BF926231FFA8BFBDDF824C0C1
S31508005F9002930DF17603039304930BACABF10A035A
S31508005FA0059310210422CDF800C0CDF80480CDF861
S31508005FB018A0079410AB00F0A1FB0BF11C012046BA
S31508005FC04144042228F064F9002840F096809DF8A0
S31508005FD076405CB1022C00F290800DF177031D44E7
S31508005FE00346814698460DF177022CE021460DF1CD
S31508005FF077031D44AB4212D2981C5A781B78022BA1
S3150800600009D0032B03D0012B07D1012A04E0082A63
S3150800601073D1014601E0042A6FD18318EAE7002903
S315080060206BD002203246FFF719FE66E002F1020E37
S3150800603051781278042A15D008D8012A0BD0032AD9
S315080060400CD00EEB0102AA42F0D317E0052A0DD0B8
S31508006050832A0FD0F5E70129F3D04EE008294CD161
S31508006060F046EEE7082948D17046EAE7042944D104
S315080060700123E6E7082940D1F146E2E7002B3CD0A8
S3150800608000283AD01E49082228F002F9A8BBB9F11F
S31508006090000F17D009F1FF3309F1070213F8011FA2
S315080060A011B99342FAD10DE016484946082228F05C
S315080060B0EFF838B113484946082216F0D7FF1148B9
S315080060C010F09CF9022C07D1B8F1000F15D0012069
S315080060D041463246FFF7C2FD082239460EA816F099
S315080060E0C5FF9DF838300EA883F002038DF83830C6
S315080060F010F08EF9044B02221A7031B0BDE8F08F09
S315080061009BF60020A3F6002099F6002008B51AF0A1
S31508006110DFFC00201AF0F3FC074B01221A70074B2C
S31508006120002207481A70FEF731FABDE808404FF416
S315080061301670FFF759BD00BF99F600209AF60020A1
S3150800614024F0002008B50F4A1378012B02D0022B41
S315080061500FD014E00C490B780133DBB2052B0B701A
S3150800616005D800201AF0CBFC4FF4167005E0022380
S3150800617013701AF0ADFC49F64040FFF735FD0020D4
S3150800618008BD00BF99F600209AF6002010B51B4BF3
S3150800619000241C701A4B86B01C70FFF7D7FCB0B1F0
S315080061A023461849184A1BF036F9044610BB2146FF
S315080061B0142201A828F0AEF844F64C53114801A958
S315080061C0ADF814301BF036F9044610B112E00E246F
S315080061D010E00E4808211AF0B8FB50B90C4B2146BE
S315080061E008220C481C6028F095F80B4810F0FCF8BB
S315080061F000E00124204606B010BD00BF99F6002035
S315080062009AF60020E8EF00208D5E00089BF6002035
S3150800621020F00020A3F60020C8EA0208034B044831
S315080062201B78002B08BF0020704700BFACF6002083
S31508006230ADF600207FB5830616D50D4A04AB106867
S31508006240516803C3FFF782FC70B10DF10F011AF014
S3150800625089FF084B04AA00939DF80F10082300F045
S3150800626025FA054B01221A7007B05DF804FB00BF3A
S31508006270C7240308ADF60020ACF6002070B5FFF77A
S3150800628065FC054650B3164B93F900300433042BCE
S315080062900CD8DFE803F0070B030D0500112408E00E
S315080062A0002406E00A200F49FEF732F90C2400E024
S315080062B010240D4B00221E681A6000F0F1F90B4BF2
S315080062C030B11A7828463146234627F0B5FC05E052
S315080062D01A782846314623461BF0B2FF002070BDC7
S315080062E0CDF60020CF24030868F00020CEF6002063
S315080062F008B5FFF72BFC20B1034B93F900101BF0F0
S3150800630004FF002008BD00BFCDF7002070B5064683
S315080063100D461446FFF7EAFB68B1074B07491E709E
S31508006320074B1D701CB1BDE87040FEF7B1B8BDE85B
S315080063307040FEF757B870BDCDF60020D8EA0208BF
S31508006340CEF6002030B5164B87B0834225D1FFF72D
S31508006350FDFB044608B30DF11303009303A802A935
S315080063600DF111020DF1120319F01CFE0546A0B934
S31508006370029B8DF8103000F093F9024603A92046D7
S315080063801AB12A4627F05CFC01E01BF052FF03987D
S3150800639019F04AFE00230393DDE7002007B030BD5D
S315080063A0F0EA020810B50C4660B9FFF79FFB48B142
S315080063B005491CB1BDE81040FEF76AB8BDE81040B3
S315080063C0FEF710B810BD00BFF0EA020808B5084B82
S315080063D0187031B1FFF78AFBBDE808400549FEF79A
S315080063E057B8FFF783FBBDE808400249FDF7FABF37
S315080063F0CDF70020E4EA020808B5084619F09EFC25
S3150800640028B1BDE808400A200149FEF781B808BD51
S31508006410E924030808B5084619F0A0FC28B1BDE828
S3150800642008400A200149FEF773B808BDFB24030893
S3150800643008B5084619F072FC28B1BDE808400A20DC
S315080064400149FEF765B808BD1725030808B519F010
S315080064509DFC38B119F05CFC034902460A20FEF798
S3150800646057F8052008BD00BF6E25030808B508467D
S31508006470064919F02FFD38B119F04AFC04490246BD
S315080064800A20FEF745F8052008BD00BFA5630008E9
S31508006490AA250308114AF8B51368022B1BD813F06E
S315080064A0010404D0990706D40221012400E0012141
S315080064B00B43136000E002240C2202FB04F6084F8B
S315080064C00021BD19284627F025FF064BC4EBC41446
S315080064D01C44BC5100E000252846F8BD64F00020A5
S315080064E04CF00020CFF600200E4B37B51A680C4644
S315080064F01D4692B90C4809796279009094F90630DC
S31508006500206819F081FC40B119F002FC07490246DF
S315080065100A20FDF7FDFF052001E02C60002003B0EE
S3150800652030BD00BF68F000200D630008E8250308A9
S3150800653010B528F02AF900231946074A9C5C204220
S315080065401CBFD218527803F1020318BF1143082B57
S31508006550F3D1084610BD00BF7727030808B50846DB
S3150800656019F0A4FD28B1BDE808400A200149FDF745
S31508006570CFBF08BD2726030810B581F001000C46D9
S3150800658019F072FA40B10A200CB1044900E0044936
S31508006590BDE81040FDF7BCBF10BD00BF3D2603088F
S315080065A06426030808B50846012119F0BFFA20B188
S315080065B00A200249FDF7ACFF0A2008BD8C2603080D
S315080065C008B50846012119F055FA20B10A200249F2
S315080065D0FDF79EFF0A2008BDAD26030808B5084644
S315080065E0002119F0A3FA20B10A200249FDF790FF0D
S315080065F00A2008BDD126030808B50846002119F067
S3150800660039FA20B10A200249FDF782FF0A2008BD9F
S31508006610F526030808B519F079FA28B1BDE8084047
S315080066200A200249FDF774BF08BD00BF1C270308EE
S3150800663008B528F089F828B1BDE808400A200249BB
S31508006640FDF766BF08BD00BF4827030808B508461A
S315080066501146034A28F07FF8003018BF012008BD0C
S31508006660CD63000810B5094C0846247811461A4629
S31508006670029B1CB1BDE8104019F09AB81046BDE857
S3150800668010401946024A27F0C7BD00BFCEF70020C2
S315080066907F270308014B1870704700BFCEF700200C
S315080066A0014B1878704700BFCEF700202DE9FF414F
S315080066B0064601A8884615461F460A9C1BF0B0FAEE
S315080066C00EB105B124B90C48362128F07CF8FEE74E
S315080066D001A8314642461BF0B7FA3A4601A82946B0
S315080066E01BF0B4FA01A821461BF0B2FA01A81BF068
S315080066F0A5FA04B0BDE8F081A62703082DE9F04FF6
S315080067008346DDB003A8884615469A46DDF89C916F
S31508006710689C6A9F6D9E1BF06CFABBF1000F06D051
S31508006720BAF1000F03D0699B0BB107B126B921480E
S31508006730482128F048F8FEE703A8594642461BF0C8
S31508006740A0F980BB9DF89831CDF800A0019303A865
S3150800675021466B9A2B461BF09BF964B1B9F1000FE1
S3150800676004D114484F2128F02EF8FEE703A849461D
S31508006770224600F0DFFA9DF8B03103A80093699924
S315080067806B9B3A4600F01CFB03A831460DF10B0241
S3150800679000F0A4FB9DF80B30AB4204D00548562107
S315080067A028F011F8FEE703A81BF034FA5DB0BDE83F
S315080067B0F08F00BFA627030837B5114C2368DBB94D
S315080067C0104D28461AF0F0F9284625601AF00FFAF7
S315080067D04BF280232268D35C022B0DD9032000F0EC
S315080067E03FF80546012000F047F801210090064AC7
S315080067F003202B4627F0E9FF206803B030BD00BF11
S315080068006CF0002078260020172803080362009BF6
S315080068104362009000F50D405C30014B1BF0B6BC9E
S315080068203F0D02088362009BC362009000F50D408D
S315080068305C30014B1BF0BBBC350D020849F2FB135B
S31508006840C35C013BDBB2032B9ABF024AD05C012032
S31508006850704700BF752803080048704737280308A3
S3150800686004289ABF024B53F820000248704700BF1D
S31508006870FCEA02089E2803080138C0B20B289ABF12
S31508006880024B53F820000248704700BF10EB02087D
S3150800689099280308014B53F82000704740EB02087B
S315080068A048F2042337B5C4583CB12268C2500023C5
S315080068B023600388013B038014E048F20823C0588C
S315080068C01AF0DCF902280DD90320FFF7C9FF05469F
S315080068D00820FFF7D1FF08210090044A03202B4621
S315080068E027F073FF204603B030BD00BFCF2A030848
S315080068F04A6808B50B464AB9CA683AB98A6852B9A5
S315080069001B6943B9BDE808401AF098BD04485F21E1
S3150800691027F059FFFEE70248622127F054FFFEE7F9
S31508006920F42A030808B5038CC28B1944914205DD85
S3150800693008484FF4A77127F046FFFEE789B291424F
S31508006940018405D903484FF4A97127F03CFFFEE7F7
S31508006950002008BDF42A030808B5C38B8B4205D26C
S3150800696004484FF4AE7127F02EFFFEE7018400209D
S3150800697008BD00BFF42A030808B5C38B994205D998
S315080069800A484FF4E67127F01EFFFEE75B1AC38339
S31508006990038C828B8B420A4494BF0023591A828344
S315080069A08CBF01840384002008BD00BFF42A0308B5
S315080069B02DE9F0411F46C38B80469942164651D2AF
S315080069C08A189A42828BA8BF5E1A11448CB2A8BF55
S315080069D0B6B24B2C11D8C4F14C05ADB2B54228BF9E
S315080069E0354600F13401214438462A46761B16F00E
S315080069F03DFBB6B22F44002103E0A4F14C0189B255
S31508006A000025D8F800807B2922D9B8F1000F05D1D6
S31508006A10164840F20B2127F0D6FEFEE77C39D8F857
S31508006A20008089B2EFE7C1F17C04A4B2B44228BF62
S31508006A30344608F1040338461944224616F016FB74
S31508006A40361B2544D8F80080B6B2ADB227440021DB
S31508006A504EB1B8F1000FE6D104484FF4057127F09E
S31508006A60B2FEFEE700252846BDE8F081F42A0308B1
S31508006A702DE9F0411F46C38B15468A189A420646E9
S31508006A8005DD2C4840F2312127F09DFEFEE7828B7A
S31508006A90A8BF5D1A114489B2A8BFADB24B2910D858
S31508006AA0C1F14C04A4B2AC4228BF2C463430084489
S31508006AB0224639462D1B16F0D9FAADB227440020D6
S31508006AC003E0A1F14C0080B20024D6F800807B28B0
S31508006AD022D9B8F1000F05D1164840F2562127F001
S31508006AE072FEFEE77C38D8F8008080B2EFE7C0F186
S31508006AF07C06B6B2AE4228BF2E4608F104033946D4
S31508006B001844324616F0B2FAAD1B3444D8F8008061
S31508006B10ADB2A4B23744002045B1B8F1000FE6D1B2
S31508006B20044840F25F2127F04EFEFEE72046BDE806
S31508006B30F08100BFF42A03082DE9F041C68B884688
S31508006B40B11889B2074614461AF0B2FC054668B968
S31508006B503846314622464346FFF78AFFA04205D00B
S31508006B6004484FF4D07127F02EFEFEE72846BDE80C
S31508006B70F08100BFF42A03083F2908B505D909485A
S31508006B804FF42A7127F01FFEFEE700EBD10090F8BC
S31508006B90242001F0070180230B411A4214BF01206B
S31508006BA0002008BDF42A03083F2908B505D9094875
S31508006BB040F2AE2127F007FEFEE700EBD10090F881
S31508006BC0242001F0070180230B4122EA030380F801
S31508006BD0243008BDF42A03083F2908B505D9094811
S31508006BE04FF42D7127F0EFFDFEE700EBD10090F88A
S31508006BF0242001F0070180230B41134380F8243039
S31508006C0008BD00BFF42A0308F8B507461D4608461E
S31508006C10D118FB8B994205DD214840F2CE2127F099
S31508006C20D2FDFEE7BC8B1444A4B24B2C0FD8C4F19A
S31508006C304C06B6B2AE4228BF2E4607F134012144AF
S31508006C403246AD1B1BF0E7FDADB2002401E04C3C1B
S31508006C50A4B23F687B2C19D92FB9114840F2ED210F
S31508006C6027F0B1FDFEE77C3C3F68A4B2F2E7C4F129
S31508006C707C06B6B2AE4228BF2E46391D214432469E
S31508006C801BF0C9FDAD1B3F68ADB200243DB1002F16
S31508006C90EDD1034840F2F62127F095FDFEE7F8BD51
S31508006CA0F42A030870B58C0013195D689DB9DD6870
S31508006CB08DB9056815B95A60DA600AE025446D6829
S31508006CC05D60066805EB8105DE60EA6003681C44C2
S31508006CD06260026070BD03484FF4487127F073FD87
S31508006CE0FEE700BFF42A030870B58C0013195D6827
S31508006CF0BDB1DD68ADB10668B24205D1AA4208BF8A
S31508006D000022056008BF0260D8685A6804446260B9
S31508006D105A68D86802EB8102D0600022DA605A60AD
S31508006D2070BD034840F2373127F04DFDFEE700BF3E
S31508006D30F42A0308F8B5D0F8503116461344D0F8AB
S31508006D404C210446934202D80D468F191EE01B4873
S31508006D50A52127F038FDFEE7B4F85C31102B08D1E1
S31508006D6004F58C7120460A461AF04BFF0023A4F856
S31508006D705C31B4F85C315A1CA4F85C21234415F83C
S31508006D80011B93F818214A4083F81821BD42E3D124
S31508006D90D4F85021D4F84C3132449A42C4F85021E0
S31508006DA00BD1B4F85C312BB104F58C7120460A4638
S31508006DB01AF027FF0023A4F85C31F8BD652B0308F9
S31508006DC02DE9F0471E46D0F858319046D0F85421A0
S31508006DD03344934204460F469DF8209004D93E4812
S31508006DE0C72127F0F0FCFEE70025B54255D0B4F8D8
S31508006DF05E31102B18D104F59C710A4694F848E1C7
S31508006E000F20704505DD11F8013D0133DBB20B702B
S31508006E1043B1204604F594711AF0F3FE0023A4F852
S31508006E205E3101E00138ECE7B4F85E31B9F1000FE4
S31508006E300CD05A1C234417F805A093F83831A4F847
S31508006E405E218AEA030308F805300BE05A1C23443E
S31508006E5018F805A093F83831A4F85E218AEA030ADF
S31508006E6007F805A0B4F85C31102B08D104F58C712D
S31508006E7020460A461AF0C5FE0023A4F85C31B4F889
S31508006E805C3101355A1C2344A4F85C2193F8182177
S31508006E908AEA020A83F818A1A7E7D4F858311D44EC
S31508006EA0D4F85431C4F858519D4213D3B4F85C3120
S31508006EB02BB104F58C7120460A461AF0A2FE94F806
S31508006EC048310133DBB20F2B04D8E218002182F8CF
S31508006ED02811F6E7BDE8F087652B030870B5D0F8EA
S31508006EE054311546D0F8582104469A420E4605D024
S31508006EF012484FF4817127F066FCFEE790F860317E
S31508006F000BB9B5B970BD00F5947100F59C721AF00D
S31508006F1078FE314604F2171394F860018A1B824200
S31508006F20EFDA013393F820001A78424001F8012B72
S31508006F30F2E794F860312B7070BD00BF652B03082B
S31508006F4008B5D0F880308B4201D0CA682AB1074804
S31508006F504FF4B97127F037FCFEE70BB9C16700E0BB
S31508006F60D960C0F88010002008BD00BFE52B0308D3
S31508006F7070B504464B68002503F5034304330360E4
S31508006F80564B574A4360A060C560056160614B680F
S31508006F9004F1530603F5034304338361514BC3617C
S31508006FA000F118032062C3624B68456203F5034388
S31508006FB0043303634C4B8562436300F13003A063DB
S31508006FC0436481644968234601F50241FC31C5637F
S31508006FD00564A4301AF00AFD04F1B4001DF004FAA1
S31508006FE004F1C00020F03DF904F2012020F019F95F
S31508006FF00B2384F88C3084F858304FF6FF73A4F8C6
S3150800700056304FF6FE73FF22C4F890207F2284F88C
S31508007010845084F8875084F8885084F8895084F816
S315080070208A5084F88B50A4F89450C4F89850C4F841
S315080070309C506567A567E567C4F8805084F8595081
S3150800704084F8A020A4F8543004F14B0527F0D3FBAC
S3150800705005F8010FB542F9D194F84C307C2223F09B
S31508007060010343F0020384F84C3004F54A7000210A
S3150800707027F050F920461D491AF07DFE20461C4986
S315080070801AF05BFEB4F8561020461AF068FE204641
S3150800709004F14C011AF02DFE4FF6FE7120461AF047
S315080070A041FE27F0A8FB84F8850027F0A4FB0025FD
S315080070B084F88600C4F8B850C4F8BC5020461AF0C4
S315080070C0E0FD19F049FD20461AF0DBFDFFF7E2F96D
S315080070D0C4F8A453C4F82403204670BD4B22020802
S315080070E0EF1C02083D220208311F0208982D0308EA
S315080070F0DA2B03082DE9F0410C46E2B000230546D9
S3150800710009A804931AF075FD20461BF075F90028A6
S3150800711000F0B08020460DF10E011BF076FA9DF8BE
S315080071200E30082B17D0102B31D0002B46D1627A9F
S31508007130AB6C510703F5056605F14C0844D4D3F842
S315080071406018204600F0DAFEAA6CD2F860380133DF
S31508007150C2F8603838E0627AAB6C520703F2EC7614
S3150800716005F14C0830D4D3F81C18204600F0C6FEAA
S31508007170A86C00F5F8601DF007F9AB6C2046D3F84B
S31508007180D81701F07F01013100F0EAFE1CE03C4B04
S31508007190D5F8A413186801310590C5F8A41320463C
S315080071A000F0ACFE204605A900F0BEFE2046FF21F1
S315080071B000F0D6FEDFF8D480324E05E0324840F2C1
S315080071C0C72127F000FBFEE70DF10D0120461BF055
S315080071D00FFA05AF04A920461BF024FA9DF80D30D6
S315080071E028464146049A00971AF007FE31461022AF
S315080071F009A81AF046FC20461BF043FA02388DF817
S315080072000F0020461BF0B7FA054620461BF0C8FAC1
S315080072100D219DF80F300246019109A829460097CD
S315080072201AF036FC20461BF04EFA054620461BF09F
S31508007230A2FA2946024609A8FFF77CFD20461BF05C
S3150800724044FA064620461BF040FA054620461BF03F
S31508007250A7FA012203463146009209A82A46FFF7F3
S31508007260AFFD20461BF0B7FA0DF10F02014609A83B
S31508007270FFF734FE09A81AF0CDFC62B0BDE8F0812C
S31508007280D62B0308882D0308E52B0308802D030851
S315080072902DE9F0470D46E6B081460DA898461746F3
S315080072A01AF0A7FC6B7A28466FF300036B721BF083
S315080072B0A3F8002800F0E28003A928461BF098F9F5
S315080072C004A928461BF0AEF928460DF10D011BF05E
S315080072D09CF99DF80D40082C0AD0102C53D0002C90
S315080072E040F0CE80D9F8486016F5056649D1C7E062
S315080072F0B8F1000F00F0C48028460DF10F011BF00D
S31508007300AEF9D9F848009DF80F30D0F8D847013BB8
S31508007310DBB204F07F0293428DF80F3002D100F2FF
S31508007320EC7619E004F1FF3A0AF07F02934207D19E
S3150800733000F5F86051461DF016F8544606460BE06F
S31508007340013404F07F02934240F09A8000F5F86019
S3150800735021461DF008F8064698F81C3003F0070386
S31508007360062B0ED1D8F818309C42C0F0898008D177
S31508007370049BD8F80C2001339342C0F0818000F0BA
S315080073808180B91C02E04349434E002405AF9DF8AD
S315080073900C30049A009748461AF02FFD28461BF031
S315080073A070F90238314610228DF80E000DA81AF031
S315080073B068FB28461BF0DFF9064628461BF0F0F95D
S315080073C00D219DF80E300246009701910DA8314611
S315080073D01AF05EFB28461BF076F9064628461BF08F
S315080073E0CAF9314602460DA8FFF7A4FC28461BF049
S315080073F06CF9074628461BF068F9064628461BF02E
S31508007400CFF90022034600920DA839463246FFF707
S31508007410D7FC09A90DF10E020DA8FFF75FFD284656
S315080074201BF0D9F99DF80E20014609A826F030FF71
S3150800743030BB9DF80D30082B1CD198F81C3003F092
S315080074400703062B16D1D8F81830A34203D0C8F87C
S315080074501840C8F81000049BD9F848000133C8F84A
S315080074600C30D0F8D8379C4204D900F5F86021468C
S3150800747001F004F96B7A43F001036B72002402E011
S31508007480082400E01F240DA81AF0C4FB204666B0A5
S31508007490BDE8F087802D0308882D03082DE9F04301
S315080074A090F889300C2903F1010393B004460D4680
S315080074B0D0F8246380F8893009D003D8002900F071
S315080074C0B480ACE0A1F11003012B00F2A88030468D
S315080074D00FA91AF0C6FF9DF83C30022B02D0082BE4
S315080074E02CD06BE020461AF0CCFB19F0C7FB02281B
S315080074F040F28B800320FFF7B3F907460720FFF712
S31508007500BBF981462846FFF7C5F9804630461AF08A
S315080075108CFF94F889300390CDF80090CDF804805C
S3150800752002950493337A03200593BDF83E3007216C
S315080075300693744A3B4627F048F966E020461AF057
S31508007540A0FB19F09BFB02285FD90320FFF788F9F7
S3150800755007460720FFF790F981462846FFF79AF96C
S31508007560804630461AF061FF94F889300390CDF8CA
S315080075700090CDF8048002950493337A032005938E
S315080075809DF83E30072106939DF83F305E4A0793E3
S315080075909DF8403008939DF8413009939DF8423094
S315080075A00A939DF843300B939DF844300C939DF84D
S315080075B045300D933B4627F008F926E020461AF099
S315080075C060FB19F05BFB02281FD90320FFF748F977
S315080075D007460720FFF750F981462846FFF75AF96C
S315080075E0804630461AF021FF94F889300390CDF88A
S315080075F00090CDF8048002950493337A032005930E
S315080076000721424A3B4627F0E0F820461AF0A2FC3A
S3150800761058B994F88920337A9A4267D305E03C48EA
S3150800762040F2134127F0CFF8FEE7002384F88930AB
S3150800763084F8883030461AF0E4FE58B1D4F834336A
S315080076400133C4F8343355B9D4F838330133C4F8A0
S31508007650383304E0D4F83C330133C4F83C3394F8A7
S315080076608430032B0ED0042B12D0012B38D1D4F83A
S315080076704C3320460133C4F84C33B4F894101AF04E
S31508007680F3FA3BE0D4F848330133C4F8483323E02F
S31508007690626C04F130039A4215BFD4F84433D4F827
S315080076A040330133013314BFC4F84433C4F84033BC
S315080076B0636FDA68626702B9A2670022DA60727AD3
S315080076C0314652075EBF94F88620013284F8862038
S315080076D05F6898682A46B84720461AF081FC0DE08C
S315080076E00B4840F2544127F06EF8FEE720461AF0A0
S315080076F039FCD4F854330133C4F8543313B0BDE815
S31508007700F08300BF4F2C0308A42C0308142D03088C
S31508007710E52B0308F0B504460F4685B000682146F8
S3150800772016461D4623F0E1FCD4F8283338460133C3
S31508007730C4F8283301A91AF094FE4FF6FF73BDF872
S3150800774006209A420BBFD4F83033D4F82C330133D1
S3150800775001330CBFC4F83033C4F82C330C2D05D1D3
S31508007760D4F85C330133C4F85C3306E0112D02BF4C
S31508007770D4F858330133C4F8583320461AF0DFFBDF
S3150800778060B9112D0AD194F88830032B06D8013335
S3150800779084F8883020461AF0E5FB1DE0002384F8BB
S315080077A0883094F88430032B04D120462946FFF705
S315080077B075FE11E0042B07D1002EF6D004F1300037
S315080077C064211AF051FAF0E7012BEED0034840F293
S315080077D07E3126F0F8FFFEE705B0F0BDE52B03087D
S315080077E070B5B0F888600446D0F82453002E53D1FB
S315080077F090F85930AB7190F88430032B16D0042BCF
S3150800780025D0012B36D11AF03CFA4FF6FF71FEF758
S31508007810F3FD94F88C3020466B7129461AF0FEFA6F
S31508007820284631461AF004FE08230EE090F8583030
S3150800783029466B711AF00AFB94F8851028464B1CEA
S3150800784084F885301AF0F4FD02232B7218E090F8BC
S31508007850583029466B71436F1A6898689047002814
S3150800786053D16B7A5A070BD4284694F886101AF027
S31508007870DFFD05E02A4840F2093126F0A4FFFEE7BD
S3150800788029462046FFF736FC94F8593095F9061034
S315080078905AB29142C8BFAB7120461AF0F2F969791B
S315080078A0FEF7E4FD28B11E4840F2173126F08BFF9B
S315080078B0FEE720461AF0E5F92946FEF715FE28B137
S315080078C0174840F2193126F07EFFFEE728461AF0DF
S315080078D098FD30B120461AF0D4F9FEF729FEC30701
S315080078E00ED5D4F8B830CBB16B7A284643F00203EC
S315080078F06B72D4F8B830D4F8BC10BDE8704018479D
S31508007900204610211AF0B0F9EBE72046D4F82413E4
S315080079103246BDE870400C23FFF7FCBE70BD00BFC1
S31508007920E52B03082DE9F041D0F860338AB001331E
S3150800793004460E46C0F860331546002A40F03181E9
S31508007940002900F02D814B7A62F300034B72D0F8C0
S31508007950B8304BB14B7A62F341034B72D0F8B8306A
S315080079600846D4F8BC10984730461AF0D7FC0546A6
S31508007970002840F0168104A930461AF0E1FDA06CF3
S3150800798004A900F6FC4020F025FD9DF810300746B6
S31508007990022B05D0082B0FD0002B40F076810BE088
S315080079A0002800F0768108238DF810300368CDF89A
S315080079B012304368CDF8163004F14C080DF1120068
S315080079C04146082226F064FC002800F05E819DF8F6
S315080079D01030ABB194F8003293B104F1C0050DF143
S315080079E0120128461FF075FC0146002800F0538155
S315080079F0284603AA1FF0B3FC10B99DF80C30B371E2
S31508007A009DF8103053B9304607A91AF02AFD9DF89B
S31508007A101C50022D08D0082D25D039E094F82133C2
S31508007A20002B40F01F81EEE730460DF10E011AF0EB
S31508007A300AFD4FF6FF72BDF80E30934204D0B4F833
S31508007A4056209A4240F0238194F88720BDF81E30CC
S31508007A501AB14FF6FF7293421AD0B4F854209342E3
S31508007A6040F0158114E030460DF10E011AF0EBFCDA
S31508007A70BDF80E20B4F856309A4240F008810DF150
S31508007A801E0041462A4626F003FC002840F0FF80E7
S31508007A904FF6FF73BDF81E2020469A420BBFD4F856
S31508007AA06833D4F86433013301330CBFC4F8683340
S31508007AB0C4F86433314604AA3B46FFF7E9FB05469A
S31508007AC000286ED13FB307F11E0004F1B40196F900
S31508007AD006201CF0EFFC30461AF08EFCD8B13B7F2E
S31508007AE003F00703052B04D0062B14D0012B40F016
S31508007AF0D08030461AF07BFC032801D0022550E0DE
S31508007B0030460DF10D011AF01FFE0028F6D19DF83A
S31508007B100D30042BF2D194F88430012B0FD1304666
S31508007B201AF065FCB0BBD4F87433D4F89800013366
S31508007B30C4F874333146D4F89C309847ADE094F8CD
S31508007B40873063B99DF81C304BB1206B04F13001C6
S31508007B5023F0CBFA20461AF094F8FEF777FC304665
S31508007B601AF045FC01280FD008D3032812D1204665
S31508007B7031461AF02DFB02287FD18EE0D4F87433F3
S31508007B800133C4F8743378E0D4F86C330133C4F89D
S31508007B906C3372E0D4F87C330133C4F87C337CE070
S31508007BA0142520461AF06DF819F068F8012812D93C
S31508007BB00220FEF755FE06460720FEF75DFE07463D
S31508007BC02846FEF767FE0097019007210220344AEF
S31508007BD0334626F0FAFD083D172D3DD8DFE805F0B7
S31508007BE00C3C3C3C3C3C3C3C3C3C3C12181E242A8D
S31508007BF0303C3C3C3C3C3C36D4F898330133C4F822
S31508007C0098334AE0D4F89C330133C4F89C3344E0F3
S31508007C10D4F88C330133C4F88C333EE0D4F890336F
S31508007C200133C4F8903338E0D4F894330133C4F8F8
S31508007C30943332E0D4F880330133C4F880332CE02F
S31508007C40D4F884330133C4F8843326E0D4F888336F
S31508007C500133C4F8883320E0D4F8A0330133C4F8DC
S31508007C60A0331AE004F201200DF112011FF0E5FA23
S31508007C7000283FF4C8AE1B2593E7E46F6CB1236870
S31508007C80A06831469847E468F8E7162589E7182575
S31508007C9087E7152585E7172583E70AB0BDE8F0814C
S31508007CA0552D03081FB590F884300446022B33D0AF
S31508007CB0042B36D0012B5AD1D0F8902090F88C306E
S31508007CC001335208DBB21BD1C4F8902084F88C30FB
S31508007CD0204619F0D6FF94F85810FEF7C7FB204641
S31508007CE019F0CFFFB4F85610FEF786FBD4F89800C3
S31508007CF0D4F89C300021984720461AF071F93CE0E8
S31508007D001A2BE1D8D107DBD5C4F8902084F88C303B
S31508007D1020461AF027F930E090F9A0101AF0BBF9BE
S31508007D202BE019F0AEFF94F85810FEF79FFBD4F835
S31508007D30283301A90133C4F82833D4F824031AF0E8
S31508007D4090FB4FF6FF73BDF8062020469A420BBFFC
S31508007D50D4F83033D4F82C33013301330CBFC4F8CC
S31508007D603033C4F82C331021FFF798FB05E004489C
S31508007D7040F2BF3126F027FDFEE704B010BD00BF74
S31508007D80E52B030830B503780D46022B89B0044667
S31508007D90114615D0082B19D1C2788378009202793A
S31508007DA001924279029282790392C2790492027A06
S31508007DB00592427A28460692084A26F02DFA09E0E4
S31508007DC02846074A638826F027FA03E02846054A24
S31508007DD026F022FA284609B030BD00BFA72D0308B1
S31508007DE0A02D0308CF2D030810B50C461AF023FB67
S31508007DF028B9054840F28F1126F0E5FCFEE7047025
S31508007E0024124470002010BDD72D030808B5026857
S31508007E1053781B0203F44063B3F5006F05D0054899
S31508007E204FF4E67126F0CFFCFEE751710912917105
S31508007E30002008BDD72D030808B503685A78120232
S31508007E4002F44062B2F5406F05D008484FF4EE716F
S31508007E5026F0B9FCFEE701F10802043312F8010D19
S31508007E608A4203F8010FF9D1002008BDD72D03086F
S31508007E7010B503680C465B781B0203F44043B3F560
S31508007E80004F05D0094840F26A2126F09CFCFEE71F
S31508007E901AF040FB28B9054840F26D2126F093FCFC
S31508007EA0FEE7047024124470002010BDD72D030885
S31508007EB010B503680C465B781B0203F44043B3F520
S31508007EC0404F05D00C4840F27A2126F07CFCFEE7AC
S31508007ED01AF020FB28B9084840F27D2126F073FCE9
S31508007EE0FEE704F10803013813F8012DA34200F850
S31508007EF0012FF9D1002010BDD72D030810B50C4667
S31508007F001AF04CFB28B9074840F2EB2126F05BFC37
S31508007F10FEE7230A44708370230C240EC370047191
S31508007F20002010BDD72D030838B50D461AF036FBCC
S31508007F3028B90A4840F2253126F045FCFEE70446F2
S31508007F4014F8050B00F018001AF080FB29460246C3
S31508007F502046BDE8384015F089B800BFD72D03087C
S31508007F6038B50D461AF01AFB044628B9074840F2F8
S31508007F70463126F028FCFEE7007800F018001AF0D3
S31508007F8065FB20444571002038BD00BFD72D030886
S31508007F9038B5036805460812587001F44060B0F514
S31508007FA0006F197008D0B0F5406F0AD038B125486F
S31508007FB06B2126F008FC01E0072403E0FEE7032412
S31508007FC000E00D2401F44040B0F5004F08D0B0F5AC
S31508007FD0404F0BD090B11B48872126F0F4FB0CE0EC
S31508007FE048065CBF0234E4B2023404E048065CBFCB
S31508007FF00234E4B20834E4B200E0FEE7080713D519
S315080080001A55530718BF053402F0180218BFE4B210
S31508008010102A05D0182A05D0082A05D1013402E00D
S31508008020053400E00934E4B201F00701032908BF6A
S315080080300134284608BFE4B21AF023FB204428710D
S31508008040002038BDD72D030870B5044601461BF03D
S3150800805045FD214604F1080023F07BFE214604F184
S3150800806014001BF0CAFE04F50246214604F120005E
S3150800807000F00EF9FC36A4F5D87104F1E00019F009
S31508008080CAFA304619F0B8FC04F50340043023F068
S3150800809009F848F20833002504F50340E5540C3086
S315080080A019F0B3FA04F5034023463146084A1C3052
S315080080B019F09CFC48F22C33E55048F23033E55071
S315080080C048F23433E55448F238332046E55070BD5B
S315080080D09D330208F0B585B01F469DF82830044642
S315080080E00D461646002B6ED148F22C33C358002B8A
S315080080F04ED048F23433C35CA3B110461BF0E8F9FE
S31508008100002845D106F110001BF0E2F900283FD1FE
S31508008110112F1BD130461BF069F938BB30461BF0CE
S3150800812022FA18BB2846E98B19F005FC064688B3DF
S31508008130314620461AF0DBFB48F2303248F22C333F
S315080081403046E358A1589847002053E03A2FE9D122
S31508008150A37B002BE6D008220DEB02032846298CC8
S31508008160FEF726FC9DF80830802B10E008220DEB60
S3150800817002032846298CFEF71BFCBDF80A20C2F329
S31508008180072343EA022344F64C529BB29342C9D1D1
S3150800819004202FE0A4F5D87018F070FD02284FF0DF
S315080081A0030027D9FEF75CFB04460620FEF764FBAE
S315080081B0EB8B00900193032006210F4A234626F0F5
S315080081C004FB032016E0A0F5D87018F057FD022826
S315080081D00FD90320FEF744FB04460620FEF74CFBA6
S315080081E0EB8B0090019303200621044A234626F0D0
S315080081F0ECFA022005B0F0BD472E0308952E0308B9
S315080082003C289ABF024B53F820000248704700BF2B
S3150800821040EF0208CF2D030830B5038845880C4681
S31508008220190A41EA0323290A41EA052189B089B2D4
S31508008230009185889BB2290A41EA052189B20191F4
S31508008240C588290A41EA052189B202910589290AC0
S3150800825041EA052189B203914589290A41EA05219E
S3150800826089B204918589290A41EA052189B20591CD
S31508008270C089010A41EA002189B2069120461146C1
S31508008280024A25F0C9FF204609B030BD142F03085D
S3150800829038B50446134B016001F503418360043188
S315080082A0031D4160E06083610F4B0025036200F106
S315080082B01C0305614561C161606203638562C5622D
S315080082C080F8345080F83550C5868563BC3019F07F
S315080082D095F904F13C002946802226F01BF8204631
S315080082E038BD00BFD93A0208A93A020838B504468B
S315080082F0154B0025416001F5024103608560C560A4
S3150800830005610275457585752346FC310F4A183097
S3150800831019F06CFB04F13003636404F14803E36568
S3150800832004F16003636704F17803C4F88C3004F140
S315080083309003C4F8A03004F1A403A562E562C4F86A
S31508008340B430204638BD00BF10EA0208F33D0208E3
S31508008350034601600A68011D526802F503420432A9
S3150800836042600D4A8260D860816190F8241000222C
S3150800837001F0F00162F3071180F8241090F8251037
S31508008380026101F0F00162F307114261C261026203
S3150800839080F82510704700BF3542020890F824304F
S315080083A0F7B5DB07044633D503681B6893F8F3383B
S315080083B073BB4068211D22F098FE2068543019F0DE
S315080083C05EF9064648B196F8303003F00303022BEF
S315080083D038D0304619F05DF9F3E7236802211B68A7
S315080083E032465868E03019F07FFA074680B32068AD
S315080083F039461CF0CDF9054638B1384619F054F817
S315080084000E2D05D01A2D24D11CE02046314628E031
S3150800841020461BF068FE18F031FC01280DD9022011
S31508008420FEF71EFA05460720FEF726FA07210090F2
S315080084300E4A02202B4626F0C8F920461BF056FEA7
S315080084400E2510E0204600211BF09BFE1A250AE0A7
S315080084500325204694F82430012143F0080384F8C4
S3150800846024301BF08EFE284603B0F0BD2C2F0308DF
S3150800847037B590F824200446D3072DD5C2F3031345
S31508008480013303F00F0363F30712052B80F824204A
S3150800849004D803B0BDE83040FFF780BF1BF023FEC9
S315080084A018F0ECFB022811D90320FEF7D9F9054686
S315080084B00720FEF7E1F994F82420009012090192AA
S315080084C003200721054A2B4626F07FF994F8243025
S315080084D06FF3071384F8243003B030BD702F0308F8
S315080084E037B590F824200446D50750D590F825309E
S315080084F0D9B913F0F00108D0F03313F0F00F80F873
S3150800850025300CBF0123002300E00B46520736D561
S3150800851094F824306FF3820384F8243094F82530D5
S315080085206FF3030384F825302AE0591C01F00F0184
S3150800853061F30303042980F8253006D8530726D4A7
S3150800854042F0040280F824201AE01BF0CCFD18F053
S3150800855095FB0128DCD90220FEF782F9054607209B
S31508008560FEF78AF994F82520009002F00F0201928E
S3150800857002200721074A2B4626F027F9C8E733B118
S315080085802046012103B0BDE830401BF0FABD03B018
S3150800859030BD00BFAB2F03080346002202750160F9
S315080085A0496810B501F50341043181674FF4287411
S315080085B00E49C4664FF41C748261C265026642663F
S315080085C0826680F87420C167046700F17801C3F8F1
S315080085D08000C0F88420C0F88820C0F8A020FF22B8
S315080085E0C0F88C1080F8A42010BD00BFE54302082F
S315080085F038B5002380F87430C56E084B04465D43D1
S3150800860026F0D7F8C4F88850C4F8840004F1780135
S31508008610A06FBDE8384022F0BABD00BF80EE360034
S315080086207FB505460C46164601A819F0F9FA01A8C1
S31508008630291D2A7D19F008FB230E8DF80030230C1E
S315080086408DF8013001A8230A694604228DF8023004
S315080086508DF8034019F0FAFA062201A8064919F01E
S31508008660F5FA01A8314619F0F3FA01A819F0E6FA65
S31508008670002004B070BD00BFE52F0308836970B5FC
S31508008680994204460D4648D00133994200F17806CE
S315080086901ED0A5612046294604F11C02FFF7C0FF3B
S315080086A00023E3652366D4F88C30B3421BD001233C
S315080086B084F87430E56E194B5D4326F07AF8C4F8F1
S315080086C08850C4F884003146A06F22F060FD0AE0A5
S315080086D0036F002BDDD0D0F88C30B342D9D090F898
S315080086E0743033B9D5E720682021BDE870401BF007
S315080086F0BFBA26F05EF8D4F88420236F074901FB39
S315080087000323934204D2904207D89842C1D270BD3F
S315080087109042BED99842BCD270BD70BD80EE36007C
S3150800872002299FBF0A4B0B4A5B5C525C89BF142126
S3150800873016210A220223884206D8904206D8984271
S3150800874094BF00200120704703207047022070471D
S31508008750EB2F0308EE2F030870B504463D4B216046
S3150800876043603D4B002583603C4BE06043613C4BD6
S315080087700561836148F20433E06105624A680E4682
S315080087801A444262374A826200F12402E062826336
S315080087904A6805631344C363334B4563036400F1B6
S315080087A03C03606403658564C564543018F02DFF86
S315080087B004F1640018F022FF04F1680018F01EFFA7
S315080087C0082384F879304FF6FE73656784F87A5083
S315080087D084F87B507168254A01F50241A4F8903067
S315080087E0A4F89230A4F86E502346256784F878508A
S315080087F084F8945084F8955004F19800FC3119F0E7
S31508008800F5F84FF6FF732146A4F8B23084F8A8505D
S31508008810C4F8AC5084F8B05084F8B15084F8B45019
S3150800882004F1B800FFF794FD214604F1E0001EF0BC
S3150800883091FB25F0E0FF2146A4F86C0051F8040BE3
S3150800884000F66C00FEF77CFB84F87C5084F88650B2
S31508008850204670BD8150020825450208334E02089D
S3150800886053500208C34E0208FF4F0208634D020820
S31508008870F0B592F87B308BB004460F46154663B1C7
S31508008880012380F87830136F036792F87A3080F8FE
S315080088907A3092F87C3080F87B30B5F87810384614
S315080088A0FEF75AF897F83060C6F30106F1B231B30D
S315080088B0012950D168461BF049FE3946684624F01E
S315080088C012FB84F89460BDF80420C2F3072343EA38
S315080088D002239BB2A4F89230BDF80210C1F3072216
S315080088E042EA0122A4F890202168022284F87C201A
S315080088F0B1F8C01884F88620A4F87E1028E028224B
S315080089006B463846FEF754F884F89460204602A968
S3150800891004F17C021CF07FF806A81AF067FD30B156
S31508008920204606A904F186021CF08FF819E095F88E
S315080089307F309B0604D5022384F88630AB8A07E08D
S31508008940082384F8863028686968883403C408E0F0
S31508008950A4F8883005E0044840F21B2125F033FFCF
S31508008960FEE70BB0F0BD00BFF12F03082DE9F0417B
S3150800897000F154070646384618F081FE04460025DD
S31508008980002C3CD0204618F084FE94F830308046FF
S315080089909A0632D503F00303012B08D002D3022B23
S315080089A02DD009E0304621461CF088F803E0304611
S315080089B021461BF0BEFF0546092D18D8DFE805F04D
S315080089C01F170F0F1717171717052146384618F0E0
S315080089D029FF06F16800214618F0A3FE0DE0384687
S315080089E0214618F01FFF204618F05EFD05E00548F1
S315080089F04FF4E17125F0E7FEFEE74446C0E720465E
S31508008A00BDE8F081F12F03087FB514464FF6FE72D4
S31508008A100E4601680546B1F8C0389342ADF80630EF
S31508008A2003D002238DF8043008E008220DF1060071
S31508008A3001F6B8018DF8042014F018FB49F6430333
S31508008A404DF643429DF80410204602290CBF1946EC
S31508008A5011460D2241F02801FFF79AFA2B682046A5
S31508008A60B3F8C218FFF7C0F9286800F6FC401DF0F5
S31508008A7035FC014628B9124840F2D13125F0A3FE4B
S31508008A80FEE79DF804302046022B08D1898AFFF7B5
S31508008A90BDF92046BDF80610FFF7EAF906E0FFF72C
S31508008AA0CBF920460DF10601FFF702FA204604210C
S31508008AB019F056FEF38B0020A5F86E3004B070BD91
S31508008AC0F12F0308F8B5064614460D46104649F632
S31508008AD069010D22FFF75CFA33682046B3F8C2181D
S31508008AE0FFF782F9B6F888102046FFF78FF9B6F82F
S31508008AF07E102046FFF7BCF92046EF8B19F043FE9F
S31508008B0080B2874205D90C484FF47D7125F05BFE8B
S31508008B10FEE72046EF8B19F0D8FD3A4603460021BA
S31508008B202846FDF745FF2046A97F19F046FEEB8B40
S31508008B300020A6F86E30F8BDF12F03082DE9F04F96
S31508008B4004468BB002A80D4690461BF0FFFC94F82D
S31508008B5094306BB102238DF81C30B4F890208DF850
S31508008B601030B4F89230ADF81E20ADF812300DE092
S31508008B70224652F8860F04AB5168128903C31A803D
S31508008B8007AB04F17C0207CA03C31A8094F886303F
S31508008B9094F87C20022B0CBF4FF400614FF440611F
S31508008BA041F48051022A0CBF4FF400424FF4404270
S31508008BB041F00101082B41EA020105D04FF6FF7387
S31508008BC0B4F888209A4201D041F0200195F8303057
S31508008BD0C3F380126AB1C3F38202012A41F0080185
S31508008BE004D0042A0CBF0022082200E0102242F01A
S31508008BF005022068C3F38203012BB0F8C26804D0CB
S31508008C0009D3032B07D8EE8D05E04FF6FF7695F8C6
S31508008C102E3088F8053023684046B3F8C238B34288
S31508008C2008BF41F04001FFF7B3F931464046FFF768
S31508008C30DBF823684046B3F8C21819F05FFC94F8CD
S31508008C4086304046022B04D1B4F88810FFF7DEF8C8
S31508008C5003E004F18801FFF7EFF894F87C3040460A
S31508008C60022B04D1B4F87E10FFF702F903E004F1F1
S31508008C707E01FFF71DF9404619F027FD94F8947018
S31508008C800646002F4ED0206890F80B3D022B1ED0CA
S31508008C90B4F8921000F6FC401FF046FC1028074670
S31508008CA0B4F8921020680CD000F6FC4948461FF02C
S31508008CB056FCC0F3872148461FF07DF83844C0B2F9
S31508008CC006E0890A00F6FC401FF075F800E011205E
S31508008CD0B4F89230C3F308020AB10130C0B20130C9
S31508008CE0C0B20E2800F2F98060F04F008DF8080037
S31508008CF0B4F8901002A8C1F3072242EA0122ADF89F
S31508008D000A201A0A42EA03233146ADF80C301BF052
S31508008D1025FC9DF8087007F00F070F2F14BF0527CD
S31508008D2006273E442A8C002A40F088802068009650
S31508008D3000F66800294607AA04AB23F096FBB0F1B3
S31508008D40000A05DC694840F29A4125F03CFDFEE739
S31508008D50EB8BB5F820904046C9EB030919F013FDD3
S31508008D605744FFB21FFA87FBCBEB00001FFA89F9BD
S31508008D7080B281454CD995F83090C9F38019B9F17C
S31508008D80000F09D1284618F0C2FB28B128464946E3
S31508008D90FDF7E2FD1D20A6E06B8C5BB9B4F86C30DC
S31508008DA013B90123A4F86C30B4F86C305A1CA4F833
S31508008DB06C206B8431463A46301D25F0F2FA40465F
S31508008DC019F0E1FC6FF03F03337000237370EB8BEF
S31508008DD0CBF57F49C3F30A036FEA83436FEA9343EC
S31508008DE09AB2120A42EA032333806A8C09F1FC0913
S31508008DF0C2F30723484443EA022320F00709738095
S31508008E0030461BF0BBFB07441FFA89F90644FFB23C
S31508008E104A46298C06EB0A032846FDF7C9FD07EBE7
S31508008E2009014046C9B219F0C8FC288C00218144C2
S31508008E30A4F86E902846FDF78FFD43E0EB8BC2EB56
S31508008E4003096FF03F03337000237370EB8B1FFA2F
S31508008E5089FAC3F30A0343F440431A0A42EA03228F
S31508008E603280698CC1F3072242EA012272802A8C79
S31508008E703AB143F40053190A41EA0323D210338066
S31508008E80327130461BF07AFB06440744404619F017
S31508008E907AFCFFB2C01B20F007091FFA89F9D145F1
S31508008EA028BFD14633464A46298C2846FDF780FD19
S31508008EB007EB09014046C9B219F07FFC2B8C99448F
S31508008EC0A4F86E90B4F86E20EB8B9A4203D2404613
S31508008ED0012119F0A0FA002005E0BF228DF808202C
S31508008EE08DF8090004E70BB0BDE8F08FF12F0308F1
S31508008EF07FB590F8A83004460D46002B00F0B980DF
S31508008F00466F012280F8952046B91BF02CFF6B7A34
S31508008F1066F382036B7208232B72A8E096F830304A
S31508008F2003F00301012965D006D302296DD1314624
S31508008F302A46FFF769FD61E0C3F38203022B3DD1A0
S31508008F4090F8B4306BB90B2380F8B030036893F807
S31508008F50C41880F8B110B3F8C23880F8B420A0F865
S31508008F60B230D4F8AC3094F8B01013F0010F06D133
S31508008F705B080131C4F8AC3084F8B010F1E720681A
S31508008F8000F66C0018F02FFF4FF6FF7294F8B03019
S31508008F906B71636FDB8D934210D12268B2F8C228D9
S31508008FA09A420BD125F027FC4FF6FF7381B29942FE
S31508008FB0F8D0206800F66C0018F0D1FE2046616FE4
S31508008FC02A46FFF7BBFD1D280BD1626F204692F893
S31508008FD0303043F0400382F83030616F2A46FFF79D
S31508008FE0ADFD2B79072B09D1264840F27B3125F0B8
S31508008FF0EAFBFEE731462A46FFF764FD28B1214819
S3150800900040F2873125F0DFFBFEE701A9284619F073
S3150800901028FA206801A900F6FC401FF029F940B19A
S31508009020037F5B0605D4B0F87E30C3F30C03012B2F
S3150800903021D894F878206B7A62F382036B7294F8DD
S3150800904079302B7294F878308BB1284694F87B10D7
S3150800905019F0EEF9284619F0CFF940B1216F2846E4
S31508009060FEF74CFF284694F87A10FEF779FF0020A1
S3150800907006E00C2004E02846012119F0CCF9D8E7CF
S3150800908004B070BDF12F03082DE9F04F92F8304077
S31508009090A3B014F0030480468A4615469B469DF8FD
S315080090A0B07040F0BC801046214628220EABFDF772
S315080090B07FFC2828014640F0B2809DF8383003F03E
S315080090C0F003602B40F0AB809DF83E90B9F1060F97
S315080090D00DD0B9F1110F19D12846082218ABFDF7A2
S315080090E067FC082840F09B80BDF8664009E02846E2
S315080090F0142218ABFDF75CFC142840F09080BDF8EC
S315080091007040C4F3072343EA0424A4B240461BF084
S3150800911046FA17F0B3FD022843D90320FDF7A0FB52
S315080091200B900720FDF7A8FB0C90BAF1000F05D0AD
S315080091303C4B3D4E002F18BF1E4600E03B4E4846AE
S31508009140FFF75EF8EB8B3A4A0D933A4B8146BAF134
S31508009150000F0CBF92469A46584618A92822FEF7D1
S3150800916011FE95F83030834613F0400F324B334DDD
S3150800917008BF1D46002F4DD1314B18460C9A08934F
S315080091808DE844020D9A099003920494CDF814A030
S31508009190CDF818B00795032007212A4A0B9B25F01E
S315080091A014FB40461BF0FBF917F068FD022814D99A
S315080091B00320FDF755FB04460720FDF75DFB18A9BC
S315080091C00546282210A8FFF727F8009501900721E1
S315080091D003201D4A234625F0F8FA40461BF0DFF91E
S315080091E017F04CFD02281AD90320FDF739FB04466F
S315080091F00720FDF741FB18A90546282214A8FFF702
S315080092000BF80095019007210320104A234625F004
S31508009210DCFA04E03846FDF73DFB0D4BAEE723B01C
S31508009220BDE8F08F6C300308763003086930030810
S31508009230793003087E300308853003088130030837
S315080092407D58030891300308D1300308E23003083B
S3150800925088300308F0B5002380F8953090F8A830D8
S3150800926089B004460F461646002B00F0FF80406F73
S3150800927018B1B4F86E10FDF76FFB05A9384619F05A
S31508009280F0F8206805A900F6FC401FF0A3F805468B
S3150800929030B30C2E24D001D82EB11BE0102E08D0E6
S315080092A0112E1DD016E0384619F0ABF8C0B16E770E
S315080092B016E0437F828A0133DBB2C2F308024377A2
S315080092C072B9032B0CD92068294600F6FC401FF01A
S315080092D0D3F905E0704840F2625125F074FAFEE7CA
S315080092E0206805A900F6FC401EF0C2FF05460028C6
S315080092F065D0037F6FF3C7130377636F002B00F006
S31508009300B580426F93422DD116B980F87B6029E06B
S3150800931090F87B300133DBB2032B80F87B301AD808
S31508009320384619F069F8002800F0A08004A93846E4
S3150800933019F078F9049B0DF10F012B67384619F0DF
S315080093408EF99DF80F30384685F87A3019F06DF8A1
S3150800935085F87C008AE0002380F87B30636FDB8B1E
S31508009360A4F86E30636FB4F86E10D88B884204D9AF
S31508009370934224D1A5F8781021E093420AD100231C
S31508009380A5F878306B672EB904F1E000294601226A
S315080093901DF0B2FE2068294600F6FC401EF075FF57
S315080093A00746606F3946FDF7E7FB40B1606F3946FF
S315080093B0FDF7FAFB04F1E000294603F0B9F9606FFE
S315080093C0002853D090F8303099061DD5B4F86E10A1
S315080093D0C28B8A429FBF6FF3451380F83030606FA7
S315080093E00021FDF7B9FA636F93F83030C3F38203AF
S315080093F0022B09D1012384F8953004F124004FF497
S31508009400967118F031FC31E0636F93F8303003F051
S315080094100303022B15D1254655F8B80B00F6FC4078
S315080094201CF05CFF037F28465A0707D11AF05EFE38
S31508009430206800F6FC401CF064FD02E03146FFF7A8
S315080094404FF8626FB4F86E10D38B994205D3009625
S315080094502046012105ABFFF717FE606F90F8303004
S315080094609B0603D418F0BEF8054638B194F8A83020
S3150800947083B104F1980018F0DCFA0BE0616F04F18F
S31508009480540018F0CFF9606F18F00EF86567A4F865
S315080094906E50EBE709B0F0BDF12F03082DE9F04F48
S315080094A087B09A46109B0E880593B1F80280330A56
S315080094B043EA06264FEA182343EA08281FFA88F3E0
S315080094C0044608460D46174604931BF05EF8804688
S315080094D0DDF84490C6F30A062846B8F1000F6ED1A7
S315080094E01BF04CF822688346506841464246E030F5
S315080094F018F0FAF98046002800F0BF8099F8052090
S3150800950090F83030CBEB070762F3861380F83030DB
S31508009510B9F800305D44C3852068FFB28DE8A00025
S31508009520029600F6680041465246059B23F01BFC4E
S31508009530B0F1000B40F3A380CBEB0707B8F8203057
S31508009540FFB23B449E42C0F29A803146404617F02D
S31508009550AFFF0646002840F09580BDF81030B8F8F1
S315080095602010A8F82230052388F82C303A4605EB57
S315080095700B034046FDF77CFA39464046FDF7D2F91B
S315080095802068414600F2BC701AF034F8002878D0FA
S31508009590236893F8F3381BB998F830305B0654D42F
S315080095A004F16400414618F0BCF8206D04F13C0350
S315080095B098424ED14FF47A7118F056FB49E01AF0EA
S315080095C0DDFF834604F1640018F01BF88046D8B125
S315080095D0B8F81E30B34213D1B8F82230049A934231
S315080095E00ED128461AF0D1FFB8F82030834207D1A9
S315080095F098F8303099F80520C3F38013934203D0C6
S31508009600404618F046F8E1E7236893F8F3384BB973
S31508009610B8F1000F09D199F8053093B320461BF02D
S31508009620B0FC2EE0B8F1000F2BD0CBEB0707FFB24A
S31508009630B8F8201040463A4605EB0B03FDF718FA32
S3150800964040463946FDF76EF903E020461BF099FCC3
S31508009650A6E7B8F82020B8F81E309A4235D3414616
S3150800966004F1640018F0A1F8204641464A465346DC
S3150800967007B0BDE8F04F1BF0EEBC032602E0062655
S3150800968000E0022620461AF08AFF17F0F7FA0128AA
S3150800969012D90220FDF7E4F804460720FDF7ECF896
S315080096A005463046FDF7F6F8009501900721022099
S315080096B0074A234625F089F8B8F1000F05D0404639
S315080096C007B0BDE8F04F17F0EFBE07B0BDE8F08F62
S315080096D0F33003082DE9F04F9846036806465868A4
S315080096E08946002185B01546E0300A46DDF838A0DF
S315080096F00F9F18F0F9F8044600283DD07B7990F8BA
S315080097003020214663F3861280F830203B88424693
S31508009710C385306800230293CDF80090019500F6C2
S315080097206800534623F01FFBB0F1000B27DDE18BE1
S31508009730CBEB0505EDB22944204689B217F0B8FEF1
S315080097408246F0B9218C20462A4609EB0B03FDF721
S315080097508FF93068214600F2BC7019F04BFF10B93A
S315080097604FF0020A0DE0304621463A46434605B018
S31508009770BDE8F04F1BF06FBC4FF0030A01E04FF055
S31508009780060A30461AF00BFF17F078FA012812D9A4
S315080097900220FDF765F805460720FDF76DF8064631
S315080097A05046FDF777F80096019007210220074AF0
S315080097B02B4625F00AF82CB1204605B0BDE8F04F37
S315080097C017F072BE05B0BDE8F08F00BF213103085F
S315080097D02DE9F047884616468AB0074602A89A46F3
S315080097E0DDF848901AF0B2FE02A84146324623F048
S315080097F05AFB002840F0CC8099F8054034B19DF812
S31508009800085005F03003302B22D004460825384688
S315080098101AF0C5FE17F032FA012812D90220FDF710
S315080098201FF806460720FDF727F807462846FDF7DE
S3150800983031F800970190072102205C4A334624F04C
S31508009840C4FF002C00F0AE80204617F02DFEA9E0DC
S31508009850BDF80A100222C1F307238DF81C208DF8E3
S315080098601020BDF80C2043EA0123ADF81E30C2F3E0
S31508009870072343EA02223B6892B2B3F8C018ADF850
S315080098801220914205F00F0524D10F2D14BF052390
S31508009890062308EB03010D88F21A2D0205F4584534
S315080098A0B5F5404FD2B207D104AB8DE80802384669
S315080098B007ABFFF7F3FD75E018F8033003F0E00394
S315080098C0602B68D104AB8DE80802384607ABFFF772
S315080098D001FF67E0ECB20F2C08BF9DF80940002C89
S315080098E060D003F6FC40BAF8021005F03BFA04AB68
S315080098F0009338464146324607AB1BF0E4FA054664
S3150800990000284BD19DF8083003F00F010F2914BF2A
S315080099100A469DF80920013AD2B20E2A31D80F29F3
S315080099202FD023F00F0313438DF8083002A84146C1
S315080099301AF014FE3B68012158680022E03017F03F
S31508009940D3FF044660B3B6B2314617F0B1FD0546FB
S3150800995000287FF45CAF2946324643462046FDF789
S3150800996087F899F8052094F83030384662F386135C
S3150800997084F83030B9F800302146E3851AF008FF3C
S3150800998010E043F00F038DF808308DF80920CDE775
S31508009990002402253BE70446062538E7002436E777
S315080099A0032534E70AB0BDE8F08700BF5031030845
S315080099B02DE9F04190F8A8308EB005460C46002BEC
S315080099C07BD008460BA918F0BBFD0646002875D1C2
S315080099D008AB20461946039318F043FD002840F0CB
S315080099E087800DF118084146204618F079FD6279FE
S315080099F020468DF81A20A2798DF81B20E2798DF879
S31508009A001C2018F0F9FC8DF81D00204618F05DFEA4
S31508009A100746204618F0C4FE2146064605F1B8005A
S31508009A201AF0F4FB204618F0E2FC0128039B02D04A
S31508009A3003281CD05CE0052E31D93A7802F0C00222
S31508009A40802A23D03A88120202F45842B2F5404FCF
S31508009A5028D03A7802F0E002602A49D18DE8080158
S31508009A602846394632460BABFFF734FE40E020461F
S31508009A700DF1170118F068FE9DF81730042B37D141
S31508009A8028460BA942461BF0BCFA31E0CDF8008007
S31508009A902846394632460BABFFF79AFE28E0042ED5
S31508009AA009D9CFE78DE808012846394632460BAB77
S31508009AB0FFF7F4FC1CE0DEB1CBE70E2628461AF0C9
S31508009AC06EFD17F0DBF8012812D90220FCF7C8FE54
S31508009AD004460720FCF7D0FE05463046FCF7DAFEBA
S31508009AE00095019007210220034A234624F06DFEC3
S31508009AF00EB0BDE8F08100BF552D030830B587B01C
S31508009B0005460021102201A824F004FC00238DF844
S31508009B10163044F64C5305F1CC04204606492A462D
S31508009B20ADF814301AF07BF918B9204601A91AF0D5
S31508009B30BCF907B030BD00BF87620208C37B37B5E2
S31508009B40012B044603D0006808211AF091F8E37B3C
S31508009B50042B04D1206804F594711AF0A5F820683E
S31508009B60002500F5BE701DF04FFE012304F14401E7
S31508009B70E373606C84F8405021F0B7FA206800F669
S31508009B8014401AF027FF206800F6FC401EF01AF869
S31508009B9048F20832236820465B689D5483F854507F
S31508009BA01BF080FA17F06AF802280DD90320FCF793
S31508009BB057FE04460220FCF75FFE02210090044A85
S31508009BC00320234624F001FE002003B030BD00BF69
S31508009BD084310308C37B37B5022B04460D4603D0F0
S31508009BE0006808211AF044F8E37B042B04D12068A6
S31508009BF004F594711AF058F8204629461BF038FBEC
S31508009C000223E373002384F8403084F89A3094F8EA
S31508009C1034301A0709D5D4F804114FF47A73890831
S31508009C2004F14400594318F01FF894F834309B07A0
S31508009C3006D5206894F8951000F6FC401FF026F922
S31508009C40206800F5215008301CF05EFE48F2083105
S31508009C50236800225B685A5483F854204FF6FF7332
S31508009C60B4F824219A420BD02068A4F8243194F839
S31508009C70223100F5315001213C30994022F026F975
S31508009C8020461BF00FFA16F0F9FF02280DD903201B
S31508009C90FCF7E6FD04460220FCF7EEFD02210090E3
S31508009CA0034A0320234624F090FD002003B030BD6C
S31508009CB09E3103082DE9F74F04460E46002521601C
S31508009CC000F110078573C5732E301AF08DFB0C232F
S31508009CD084F8365084F8375084F834307368E4646E
S31508009CE003F5034304336364A74B84F83550A36430
S31508009CF004F14403A365736884F8405003F50343ED
S31508009D000433E365A14B84F84150236604F15C03F0
S31508009D102367782384F8743025656565A566E56646
S31508009D2084F8755084F87650A567646604F1800057
S31508009D3017F064FC84F8955084F8965084F8975088
S31508009D4084F8985084F8995084F89A5084F8A55065
S31508009D5004F1C6001AF048FB716804F1CC0014310E
S31508009D601AF049F87168F02301F50241C4F8043184
S31508009D70FC31874A234604F5847017F037FE0B2317
S31508009D8084F821314FF6FF732946A4F82431C4F824
S31508009D901851C4F81C5184F8205184F82251C4F88B
S31508009DA0B051C4F8B451C4F8B8510A22201D24F0A1
S31508009DB0B1FA29460A2204F19B0024F0ABFA294697
S31508009DC03846242224F0A6FA04F5A0792946092261
S31508009DD004F1840024F09EFA29464846182224F005
S31508009DE099FA04F5B8782946182204F5AC7024F0D7
S31508009DF091FA04F5C47729461822404624F08AFACF
S31508009E0004F5CE7629461422384624F083FA2946E4
S31508009E101422304624F07EFA04F1A80A29461822AC
S31508009E2004F5947024F076FA24222946504624F044
S31508009E3071FA6FF00103216884F840316FF07F03EF
S31508009E40484684F8413101F6B80119F06BFB402306
S31508009E5084F8503194F85131494643F0030384F8A5
S31508009E605131206819F00AFF802384F8383194F8B4
S31508009E703931216803F0800343F01F0384F8393130
S31508009E800DF10100FD2301F6D70105228DF80030FA
S31508009E9004F2671913F0EAF88DF806508DF80750A2
S31508009EA004F25F1524F0A7FC05F8010F4D45F9D11A
S31508009EB094F869314FF0030943F0030369F3C603C5
S31508009EC0DBB24FF0400A43F0040384F8693169466F
S31508009ED084F868A120461BF016FB09FA09F96FF009
S31508009EE00103002584F87C314FF0FF3B236849F0D5
S31508009EF0870984F8785184F8795184F87A5184F876
S31508009F007BB184F87D5184F880A184F881915B68DF
S31508009F103946C3F8588032234FF0010884F889314E
S31508009F2084F888B184F8945184F8955184F8965148
S31508009F3084F89781206819F046FE31462646332371
S31508009F4084F89D3184F89CB184F8A85184F8A95105
S31508009F5084F8AA5184F8AB81206819F034FE0D4BB9
S31508009F6056F8380BC4F8B03104F5D871C4F8B441C2
S31508009F7019F0F6FD30462946082224F0CBF920468A
S31508009F8003B0BDE8F08F00BF0B620208D55C02087B
S31508009F90895F02081F5B02082DE9F04389B000219A
S31508009FA01422064603A824F0B5F924F002FC06F1AB
S31508009FB080080746404617F024FB04464FF0FF3555
S31508009FC0002C3FD0204617F064FBE18B142214398D
S31508009FD003AB814689B22046FCF7EAFC079BFA1ACE
S31508009FE0002A04DADB1B9D4228BF1D4628E02146CD
S31508009FF0404617F0DAFBE18B2046143989B217F090
S3150800A00057FA3046214603AA1BF08EFDA8B93046FA
S3150800A0101BF048F816F032FE022811D90320FCF787
S3150800A0201FFC04460220FCF727FC022100900A4A7E
S3150800A0300320234624F0C9FB02E0204617F034FA31
S3150800A0404C46BDE76B1C04D006F15C00294617F0A8
S3150800A0500BFE09B0BDE8F083D53103082DE9F041C0
S3150800A060044686B000F18C0500F1940624F0C3FB83
S3150800A07005F8010FB542F9D194F84030032B07D003
S3150800A080042B0ED04A4840F2FC5124F09CFB07E012
S3150800A09094F89530013B012B8CBF8027C02701E03F
S3150800A0A0FEE7C02720461BF09EFA07F04008064642
S3150800A0B008B9002567E02046314609221BF0A8FAB0
S3150800A0C0054600285FD12046314694F834201BF017
S3150800A0D0EEFA0546002856D12046314604F18D028F
S3150800A0E008231BF008FB054600284CD120463146BC
S3150800A0F03A461BF0BCFB0546002844D120463146AB
S3150800A1001BF0D7FB054600283DD12946102202A898
S3150800A11024F000F940F2FF232046ADF80830314616
S3150800A1204FF4007302AAADF816301BF0FDFC054685
S3150800A13048BB2046B8F1000F11D11AF0B3FF16F04C
S3150800A1409DFD0228B5D90320FCF78AFB07460220A5
S3150800A150FCF792FB02210090164A032010E01AF041
S3150800A160A1FF16F08BFD0228A3D90320FCF778FB84
S3150800A17007460220FCF780FB0F4A009002210320C5
S3150800A1803B4624F022FB04F14400B8F1000F02D14B
S3150800A19040F2EE2101E040F2E24117F065FD1DB103
S3150800A1A016B1304617F080F9002006B0BDE8F081F8
S3150800A1B0F4310308613203088932030870B55B4B32
S3150800A1C088B01A889B780546ADF80C208DF80E30B5
S3150800A1D01BF009FA0646002800F09F8028463146FB
S3150800A1E00B221BF015FA0446002840F098802846F2
S3150800A1F0314605F1840295F88C301BF092FA044634
S3150800A200002840F08C80284631461BF0A1FA044607
S3150800A210002840F08480284631461BF0AFFA0446F1
S3150800A22000287CD12846314695F834201BF03FFAA1
S3150800A2300446002873D128463146D5F804211BF078
S3150800A24046FA044600286AD1284631461BF031FBF7
S3150800A2500446002863D195F834309B0709D528466B
S3150800A260314603AA03231BF0ECFA0446002856D10C
S3150800A27007E0284631461BF02FFB044600284ED13E
S3150800A280EDE72846314601221BF095FB04460028D7
S3150800A29045D1284631461BF0BCFB044600283ED172
S3150800A2A02146102204A824F035F848F2FE0304A833
S3150800A2B005F1A801ADF8103019F034F928463146F1
S3150800A2C004AA1BF031FC044648BB28461AF0EAFEED
S3150800A2D016F0D4FC02280DD90320FCF7C1FA04466F
S3150800A2E00220FCF7C9FA02210090114A03202346EE
S3150800A2F024F06BFA95F8343003F0080303F0FF04F2
S3150800A3005BB92868012100F6CC4019F09DFF286842
S3150800A310214600F614401AF06BFB002402E0304692
S3150800A32017F0C2F8204608B070BD00BF8031030898
S3150800A330B53203082DE9F04786B0054688469246A9
S3150800A34099461BF050F90646002878D0284631462B
S3150800A3500E221BF05DF90446002872D128463146C4
S3150800A3601BF07CF9044600286BD1284631461BF0C1
S3150800A3702FFA0446002864D14746C8EB070353451D
S3150800A38033DA17F8013B052B22D00CD8022B0FD055
S3150800A390042BF2D12846314609F1020299F8013018
S3150800A3A01BF0BFF91DE0082B17D0132B07D0E4E7E5
S3150800A3B028463146D5F804211BF089F911E095F8AD
S3150800A3C034309B07D9D4284631461BF085FA08E075
S3150800A3D0284631461BF0BCF903E0284631461BF0F7
S3150800A3E0CDF904460028C8D02BE01022002102A887
S3150800A3F023F090FF48F2FE0302A805F11001ADF81C
S3150800A400083019F08FF82846314602AA1BF08CFB53
S3150800A4100446B0B928461AF045FE16F02FFC022865
S3150800A4200DD90320FCF71CFA04460220FCF724FA8F
S3150800A43002210090064A0320234624F0C6F9002488
S3150800A44002E0304617F030F8204606B0BDE8F0873F
S3150800A450D43203082DE9F0438DB006468846914666
S3150800A4601BF0C1F80546002800F0978090F83030B8
S3150800A470012243F0400362F3840380F8303080F809
S3150800A4802E80294630460F221BF0C2F804460028C3
S3150800A49040F0858014238DF80C3003238DF80D3099
S3150800A4A033688DF80E0093F8C43807461B02284611
S3150800A4B003A90522ADF80F30FCF73EFB0446002839
S3150800A4C06DD1B9F1000F38D016238DF814300DF17F
S3150800A4D0160008238DF815301AF0D4FD4FF4807352
S3150800A4E0284605A90A228DF81B408DF81A708DF8A2
S3150800A4F019708DF818708DF817708DF81670ADF8FC
S3150800A5001C30FCF719FB0446002848D115238DF8A2
S3150800A510083033680227B3F8C2282846C2F307234F
S3150800A52043EA022302A904228DF80970ADF80A301D
S3150800A530FCF702FB044690BB05E030462946224656
S3150800A5401BF039FADFE72146102208A823F0E2FEBD
S3150800A55040F2FF233046ADF8203029464FF4807389
S3150800A56008AAADF82E301BF0DFFA0446B8B9304613
S3150800A5701AF098FD16F082FB02280ED90320FCF784
S3150800A5806FF904463846FCF777F939468DE8010134
S3150800A590064A0320234624F018F9002402E0284638
S3150800A5A016F082FF20460DB0BDE8F083023303089B
S3150800A5B02DE9F34705460F4692469946BDF8288089
S3150800A5C01BF011F8064600284CD0284631460722CB
S3150800A5D01BF01EF80446002846D128463146524646
S3150800A5E04B461BF02EF9044600283DD12246284644
S3150800A5F031461BF0E0F90446B0BB284631461BF04D
S3150800A60008FA044680BB284631463A46B8F1000F98
S3150800A61005D043461BF092FB044628BB0DE01BF011
S3150800A62083FA044600BB95F834301B0705D428681E
S3150800A630082100F6CC4019F01AFE28461AF032FD19
S3150800A64016F01CFB02280DD90320FCF709F904466D
S3150800A6500220FCF711F902210090074A032023463D
S3150800A66024F0B3F8002402E0304616F01DFF204619
S3150800A67002B0BDE8F08700BF273303082DE9F04193
S3150800A6800C2394B08DF8083004460E460846174643
S3150800A690002104226B4420F0D8FD0546002840F02E
S3150800A6A0BA809DF80D50022D01D00625B3E030463C
S3150800A6B00B210A2206AB20F0C8FD002840F0AA802C
S3150800A6C09DF81930082BF0D120461AF0EBFC16F04D
S3150800A6D0D5FA022815D90320FCF7C2F88046284681
S3150800A6E0FCF7CAF8BDF80E100090C1F3072242EA3B
S3150800A6F0012292B2019203202946564A434624F083
S3150800A70064F8E37B012B0CD107F1100504A8294650
S3150800A71017F0F5FDE37B022B0ED079D3042B42D933
S3150800A72076E02068314600F6FC403A461EF084FC86
S3150800A730054600286FD1E7E704F1100004A90822AE
S3150800A74023F0A6FD002863D1BDF80E20C2F3072327
S3150800A75043EA0223A28C9BB29A4220D106A81AF099
S3150800A7609BFC0746201D1AF097FC87429DF821306E
S3150800A77002D1627B934212D0204639469DF81E20AC
S3150800A7801AF04DFE94F834309B0706D53046092159
S3150800A7902B2209AB20F059FDF0B10123A37324F055
S3150800A7A008F8A0610BE0206804A900F6FC401DF03B
S3150800A7B0C9FD68B3037F03F00703062B28D1A37BE3
S3150800A7C0B3B942F6652221689DF81F308A5C9B1A48
S3150800A7D05BB2002B0CDC1BE09DF82530093B202BD7
S3150800A7E0DBD8206809A900F6FC401DF01DFBD4E75C
S3150800A7F024F001F84FF47A73B0FBF3F202FB13006E
S3150800A80080B200902946204602AA0123FFF7D0FE0F
S3150800A81000251AE0054620461AF044FC16F02EFAE2
S3150800A820012812D90220FCF71BF804460720FCF77A
S3150800A83023F806462846FCF72DF8009601900721CE
S3150800A8400220054A234623F0C0FF284614B0BDE877
S3150800A850F08100BF423303086C3303082DE9F04149
S3150800A8600023CEB0ADF80C30ADF80E3004460D46D8
S3150800A870084617460B210A2204AB20F0E6FC0646DA
S3150800A880002840F00E819DF81130082B01D00626CD
S3150800A89007E104A81AF000FC8046201D1AF0FCFB0C
S3150800A8A0804509D19DF81620A37A9A4204D19DF8CD
S3150800A8B01920637B9A420ED0E37B022B40F0E98095
S3150800A8C09DF81930204641469DF816201AF0A7FD36
S3150800A8D00123A37316E0A37BA3B994F83430226846
S3150800A8E013F0010F15BF42F6652142F664219DF863
S3150800A8F017309DF81830525C9B1ADBB25BB2002BFE
S3150800A90040F3CF80284616210A2207AB20F09DFC8B
S3150800A910C8B99DF81D30082BB9D1206800F57F709D
S3150800A92020F06CFE40B92846182103AA20F053FCF3
S3150800A930002840F09880AEE00DF11E0121F0BFF925
S3150800A9400028F0D1A7E04FF000088DF81D802846B2
S3150800A95017210A220AAB20F078FCC8B99DF82930DD
S3150800A960082B7CD1206800F5CA6020F047FE40B964
S3150800A970284619210DF10E0220F02DFC002872D16F
S3150800A9808CE00DF12A0121F09AF90028F0D185E032
S3150800A99000238DF8293028460C2140F201120DAB10
S3150800A9A020F053FCC0B99DF83500FF2857D094F81D
S3150800A9B034300190206803F001030DF1360E00F5DE
S3150800A9C025509DF817109DF81820CDF800E018308E
S3150800A9D083F001031CF094F99DF81D10B9B1BDF878
S3150800A9E00C10C9B102AB28460222FBF7E1FFBDF8FD
S3150800A9F00C309DF809202068023300920DF11E01E3
S3150800AA002A469BB200F53D7021F053F804E0206811
S3150800AA1000F53D7021F027F89DF82910B9B1BDF869
S3150800AA200E10C9B102AB28460222FBF7C1FFBDF8DA
S3150800AA300E309DF809202068023300920DF12A0194
S3150800AA402A469BB200F5A96021F0D0F804E02068F8
S3150800AA5000F5A96021F0ADF80023A37300E00626EF
S3150800AA60B8F1000F1DD0384618F0CDFC40B123F0E0
S3150800AA70C2FE4FF47A73B0FBF3F202FB130080B206
S3150800AA80009007F110012046084A0123FFF790FDC0
S3150800AA9007E0022605E04FF0010858E74FF00108E5
S3150800AAA079E730464EB0BDE8F08100BF8331030830
S3150800AAB0F7B50E46144605461AF0F4FA16F0DEF80F
S3150800AAC002280DD90320FBF7CBFE07460220FBF729
S3150800AAD0D3FE02210090144A03203B4623F075FE5C
S3150800AAE0224628463146FFF7B9FE0446C8B128462D
S3150800AAF01AF0D8FA16F0C2F8012812D90220FBF784
S3150800AB00AFFE05460720FBF7B7FE06462046FBF7CD
S3150800AB10C1FE0096019007210220044A2B4623F025
S3150800AB2054FE204603B0F0BD9F330308BF33030825
S3150800AB30F0B590F89A3087B0032B044605D9002360
S3150800AB4080F89A301BF0DDF9A8E044304FF47A71AA
S3150800AB5017F08AF894F89A302046013384F89A3028
S3150800AB601AF041FD0646002800F098802046314636
S3150800AB700D221AF04DFD0546002840F0918020462A
S3150800AB80314694F834201AF092FD0546002840F024
S3150800AB90878094F834309B0707D5E37B042B3CD891
S3150800ABA0DFE803F0350B1D353500204631461AF02F
S3150800ABB093FE0546002873D1EFE704F18C0504F1EE
S3150800ABC0940723F018FE05F8010FBD42F9D1204677
S3150800ABD0314604F18D0208231AF08DFD13E0204654
S3150800ABE031461AF03BFD0546002859D12046314624
S3150800ABF01AF0EEFD0546002852D120463146D4F813
S3150800AC0004211AF064FD0546002849D105E02748C5
S3150800AC1040F2BE6123F0D7FDFEE71022002102A80C
S3150800AC2023F078FB48F2FE0302A804F11001ADF800
S3150800AC30083018F077FC2046314602AA1AF074FF4D
S3150800AC40054668BB20461AF02DFA16F017F80228B2
S3150800AC500DD90320FBF704FE05460220FBF70CFE80
S3150800AC6002210090124A03202B4623F0AEFD94F8E9
S3150800AC703430206803F0080303F0FF054BB900F6EB
S3150800AC80CC40012119F0E0FA2068294600F6144064
S3150800AC9002E000F61440012119F0AAFE002502E0A0
S3150800ACA0304616F001FC284607B0F0BDF43103081B
S3150800ACB0F23303082DE9F04F97B00F4692460293F8
S3150800ACC0D2F8288004461AF0EDF915F0D7FF0228C5
S3150800ACD00DD90320FBF7C4FD05460220FBF7CCFD82
S3150800ACE002210090944A03202B4623F06EFD384635
S3150800ACF004210A220AAB20F0A8FA054610BB9DF8E3
S3150800AD002920082A40F0AA810DF12A0004F18D01B4
S3150800AD1023F0BEFA002840F0A181294638460422CD
S3150800AD2005AB20F092FA054660B99DF81530022B5E
S3150800AD3040F0948138460B210A220DAB20F085FAA3
S3150800AD400546D8B120461AF0ADF915F097FF012847
S3150800AD5040F286810220FBF783FD04460720FBF7B5
S3150800AD608BFD06462846FBF795FD009601900721C0
S3150800AD700220724A234623F028FD71E19DF83530FA
S3150800AD80082B40F06B811021384603220DEB010396
S3150800AD9020F05BFA05460028D4D19DF81130012B26
S3150800ADA040F05C81206898F9031000F5126019F0EC
S3150800ADB056FB9DF81230984228BF1846C0B219F0C3
S3150800ADC043FB94F840308346032B02D1032840F016
S3150800ADD0478138460F210C2213AB20F036FA00289B
S3150800ADE040F038819DF84D300A2B40F0378194F8B1
S3150800ADF034309A075CD5E37B012B59D0D4F8009000
S3150800AE009DF8533099F8446F9E1B94F89530F6B226
S3150800AE10032B4DD8DFE803F0020E0E2B0DA81AF00F
S3150800AE203BF98146201D1AF037F9814540D176B2A3
S3150800AE30002E3BE00DA81AF02FF90390201D1AF0FA
S3150800AE402BF9039B834240F00B8173B2002B2FDC56
S3150800AE50002E40F0058109F6FC401CF081FE42F602
S3150800AE6038032268D35C984280F0FA8020E00DA867
S3150800AE701AF012F9261D039030461AF00DF9039BB5
S3150800AE80834200F0ED809DF8543009F6FC40012B12
S3150800AE908CBF0023012303931DF00AF8039B024687
S3150800AEA00DA9184633461DF038F8002840F3D88017
S3150800AEB094F8C43003F00703062B22D194F83430F3
S3150800AEC09B070DD4BDF816102046C1F3072343EAA5
S3150800AED0012189B25A4613AB1AF067FF88B9BFE059
S3150800AEE09DF854000DA901288CBF0020012094F874
S3150800AEF0A52004F19B031DF010F80028C0F2B080CD
S3150800AF00E0D038460521062206AB20F09EF9002837
S3150800AF1040F0A0809DF81930042B40F09F803846F9
S3150800AF200821062208AB20F090F948B99DF821308F
S3150800AF30042B40F095800BE01F34030841340308C6
S3150800AF40DDF81A0016F08EFE16F08CFECDF82200FB
S3150800AF50384603210A2210AB20F077F90646002866
S3150800AF607AD19DF84120131F042B77D80DF14201A1
S3150800AF7004F1840012F07AF89DF841300AF11001C4
S3150800AF8084F88C3004F1A80017F0B9F9BDF816203A
S3150800AF90DDF81A00C2F3072343EA0223A4F8BC30FB
S3150800AFA016F060FEC4F8B400DDF8220016F05AFE6A
S3150800AFB094F8C43004F1C60743F0780384F8C43023
S3150800AFC0C4F8B800384619F01CFA216898F9032025
S3150800AFD001F51261384619F06DFA84F8C5609DF8D6
S3150800AFE0120019F031FA94F8CB30062260F3010307
S3150800AFF084F8CB3094F8C43062F3020384F8C43082
S3150800B000029BC4F8C0309DF84E30D34084F8963081
S3150800B0109DF84F3084F897309DF8503084F8983072
S3150800B0209DF8513084F899309DF8523084F87C3078
S3150800B0300DAB03CB1B88C4F89B00A4F8A3309DF87E
S3150800B0405430C4F89F10012B8CBF0023012384F8C9
S3150800B050A53005E0054675E6054673E6062571E65C
S3150800B060284617B0BDE8F08F70B5DAB00E4604462C
S3150800B0701AF018F815F002FE02280DD90320FBF77E
S3150800B080EFFB05460220FBF7F7FB02210090AA4AD0
S3150800B09003202B4623F099FB94F84030052B01D06A
S3150800B0A0002546E130460B210A2205AB20F0CDF8F3
S3150800B0B00546002840F01B819DF81530082B01D065
S3150800B0C0062514E129463046042203AB20F0BDF8D4
S3150800B0D00546002840F00B819DF80D30022BEFD174
S3150800B0E030460A21042204AB20F0AFF805460028B2
S3150800B0F040F0FD809DF81130022BE1D130460C213D
S3150800B10040F2011219AB20F0A0F80546002840F0DD
S3150800B110EE80304616210A2208AB20F096F878BB56
S3150800B1209DF82130082BCBD1304618210DF10A02A3
S3150800B13020F051F8B0B9BDF80A1002AB3046022229
S3150800B140FBF736FCBDF80A3020689DF80920023363
S3150800B15000920DF1220132469BB200F53D7020F0B7
S3150800B160A8FC0DE0206800F57F7020F047FA38B992
S3150800B170206800F53D7020F041FA002840F0D280A2
S3150800B18094F84130032B05D12068012100F5A96008
S3150800B19020F00FF9304617210A220BAB20F055F89C
S3150800B1A008BB9DF82D30082B8AD1304619210DF1A0
S3150800B1B00A0220F010F8E0B9BDF80A1002AB3046D2
S3150800B1C00222FBF7F5FBBDF80A3020689DF8092036
S3150800B1D0023300920DF12E0132469BB200F5A960AA
S3150800B1E020F004FD05E02068012100F5A96020F0A3
S3150800B1F0E0FC04F14401606C1FF077FF002384F83B
S3150800B20041302046FEF79AFC05A819F045FF9DF83F
S3150800B2101D3001469DF81A2020461AF000F994F8C8
S3150800B2203430206803F0080303F0FF054BB900F635
S3150800B230CC40294619F008F82068294600F614403B
S3150800B24002E000F61440012119F0D2FB304609212C
S3150800B2502B220EAB1FF0F9FF00283BD004F1100596
S3150800B26004F1A8060FCE0FC50FCE0FC533682046CA
S3150800B2702B601AF0DCFDBDF80E202068C2F3072308
S3150800B28043EA0223A3840DF1660594F83430009549
S3150800B2909DF8655003F0010300F525509DF81B1035
S3150800B2A09DF81C2083F00103019518301BF028FD3A
S3150800B2B0206800F53D7020F0B9FABDF81210204656
S3150800B2C0C1F3072343EA012189B2FEF783FC054649
S3150800B2D068B9E5E694F834309B07BFD520680EA90F
S3150800B2E000F6FC401CF0A0FD05460028B6D0204616
S3150800B2F019F0D8FE15F0C2FC01281AD90220FBF76E
S3150800B300AFFA04460720FBF7B7FA06462846FBF7C6
S3150800B310C1FA0096019007210220084A234623F025
S3150800B32054FA06E0206800F53D70014620F0A4FBBB
S3150800B33026E728465AB070BD763403089A340308BF
S3150800B3402DE9F0410C23D0B08DF8083004AE002367
S3150800B3500F46904633603371054619F0A3FE15F083
S3150800B3608DFC02280DD90320FBF77AFA0446022041
S3150800B370FBF782FA02210090584A0320234623F05D
S3150800B38024FA38460021042203AB1FF05EFF044668
S3150800B390002840F09F809DF80D40022C01D006241D
S3150800B3A098E0BDF80E20C2F3072343EA0223AA8CCD
S3150800B3B09BB29A4240F08E8038460B210A2206AB91
S3150800B3C01FF043FF002843D19DF81930082BE6D11A
S3150800B3D006A819F061FE9DF81E2001469DF8213049
S3150800B3E028461AF01CF895F83430384613F0010F41
S3150800B3F014BF42F6652142F664212B6818BF9DF8F2
S3150800B4001F205B5C08BF9DF820200C219A421CBFB8
S3150800B4100123AB7340F201120FAB1FF016FFB8B948
S3150800B4209DF83D40FF2CBAD00DF13E0095F834301A
S3150800B4308DE81100286803F0010300F525509DF8F2
S3150800B4401F109DF82020183083F001031BF058FCCC
S3150800B45038460D210A220CAB1FF0F7FE58B99DF8A5
S3150800B4603120052A9BD830460DF1320111F0FEFD38
S3150800B4709DF8314000E00024384603210A2209AB32
S3150800B4801FF0E3FE90B99DF82530043B042B86D8BF
S3150800B490022C1EDC0423621C3355D2B2A31C0821DD
S3150800B4A0B154DBB203340522E4B2F25422462846EC
S3150800B4B0314609ABFEF73EFF044658B9AB7B4BB1A4
S3150800B4C0009008F11001284602AA0123FFF770F838
S3150800B4D000E00324204650B0BDE8F081D1340308CB
S3150800B4E02DE9F0418EB00E469046044619F0DAFD75
S3150800B4F015F0C4FB02280DD90320FBF7B1F9054660
S3150800B5000220FBF7B9F902210090814A03202B4655
S3150800B51023F05BF930461121032202AB1FF095FE9A
S3150800B52018B920461AF0EDFCD1E030460121032275
S3150800B53003AB1FF08AFE0546002840F0CA809DF836
S3150800B5400D30012B01D00625C3E09DF80E2094F896
S3150800B55034309A4201D00225BBE0E37B012B02D0AE
S3150800B560022B4FD0ADE0304604210A220BAB1FF068
S3150800B5706CFE0546002840F0AC809DF82D20082A70
S3150800B580E1D10DF12E0004F18D0122F081FE002893
S3150800B590E1D130460521062205AB1FF056FE0546C9
S3150800B5A0002840F096809DF81530042BCBD1304604
S3150800B5B00821062207AB1FF048FE20B99DF81D306A
S3150800B5C0042BC0D107E0DDF8160016F04BFB16F089
S3150800B5D049FBCDF81E00DDF8160016F043FBE061C6
S3150800B5E0DDF81E0016F03EFB94F82C30062262F3B6
S3150800B5F0020384F82C3023682062B3F8C01820466A
S3150800B600FEF7E8FA30460021042204AB1FF01DFEBF
S3150800B610054600285DD19DF81170022F93D1226846
S3150800B620BDF81230B2F8C028C3F38503B3EB922FE6
S3150800B6307FF477AF204631464246FFF70FF90546B5
S3150800B640002846D130463946062209AB1FF0FDFDD3
S3150800B65050B99DF82530042B7FF475AFDDF8260028
S3150800B66016F000FBC4F8040194F8343004F14405DC
S3150800B67003F0080303F0FF0683B92068314600F695
S3150800B680CC4018F0E1FD2068314600F6144019F068
S3150800B690AFF9606C29461FF028FD0EE0D4F80411B6
S3150800B6A04FF47A7389082846594316F0DDFA20685C
S3150800B6B0012100F6144019F09BF9002384F89A300A
S3150800B6C005E0144840F6BF3123F07DF8FEE7002573
S3150800B6D019E0204619F0E6FC15F0D0FA012812D92F
S3150800B6E00220FBF7BDF804460720FBF7C5F8064617
S3150800B6F02846FBF7CFF80096019007210220064A54
S3150800B700234623F062F828460EB0BDE8F08100BF54
S3150800B71004350308F43103083835030870B588B0D2
S3150800B7200D46044619F0BEFC15F0A8FA02280DD9F4
S3150800B7300320FBF795F806460220FBF79DF8022141
S3150800B7400090334A0320334623F03FF82846142155
S3150800B750052203AB1FF079FD002855D19DF80D3061
S3150800B760032B51D1284616210A2205AB1FF06DFD81
S3150800B770002849D19DF81530082B45D128461521B2
S3150800B780042202AB1FF061FD054600283CD19DF856
S3150800B7900930022B38D1206800F57F701FF02EFF84
S3150800B7A028B10DF1160120F08AFA002825DD204679
S3150800B7B0002119F0FEFC2068BDF80F1090F8C43877
S3150800B7C0090A84F82231B0F8C23800F66C00A4F8E9
S3150800B7D0243116F008FBBDF80A102068C1F30723C8
S3150800B7E043EA012189B200F66C0016F0B8FA204641
S3150800B7F0002101221AF0F2FB06E0BDF80F102046E0
S3150800B800090A2A46FEF726FE002008B070BD00BFCA
S3150800B810733503082DE9F043A3B00D469046976AA1
S3150800B820064619F03FFC15F029FA02280DD903201F
S3150800B830FBF716F804460220FBF71EF802210090D3
S3150800B8406C4A0320234622F0C0FF96F82031002BCD
S3150800B85000F0B1802C8CB5F81E904C452BD202AB6B
S3150800B860284621460222FBF7A3F89DF808301A2B32
S3150800B8709DF8093003D002331C44A4B2EDE7023424
S3150800B880A4B2234413A800213C221FFA83F922F00C
S3150800B89041FD3B8813A8ADF87E30BB7808F110014E
S3150800B8A08DF88230FB788DF883303B798DF88430BB
S3150800B8B016F025FD15E006247EE003AB2846214652
S3150800B8C00222FBF775F89DF80C30082B47D00BD8E9
S3150800B8D0022B25D0032B32D09DF80D3002331C44A1
S3150800B8E0A4B24C45E9D35EE0122B49D0812BF3D1A3
S3150800B8F004AB284621460422FBF75AF89DF8113076
S3150800B900022BD8D19DF812209DF88530111161F3CC
S3150800B9100303C2F3C00262F304138DF88530DBE734
S3150800B9200A222846214606ABFBF742F89DF819205D
S3150800B930082AC0D10DF165000DF11A010CE012229A
S3150800B9402846214609ABFBF733F89DF82520102A2F
S3150800B950B1D815A80DF1260111F088FBBCE7122213
S3150800B960284621460EABFBF723F89DF83920102A06
S3150800B970A1D88DF86D200DF16E000DF13A01EBE7B7
S3150800B98005AB284621460422FBF712F89DF8153028
S3150800B990022B90D1BDF81620C2F3072343EA0223EF
S3150800B9A0ADF8803098E7D6F8183113A8D6F81C11E8
S3150800B9B0984700241AE00224304619F073FB15F064
S3150800B9C05DF9012812D90220FAF74AFF0546072031
S3150800B9D0FAF752FF06462046FAF75CFF00960190F2
S3150800B9E007210220044A2B4622F0EFFE204623B008
S3150800B9F0BDE8F0838E350308B13503082DE9F04F0D
S3150800BA000C46FBB0054621A8164616F0F2F80AAB16
S3150800BA102046218C0C22FAF7CBFF9DF82830FF2B05
S3150800BA2022D0DBB99DF82920152A17D11CE0FF2B57
S3150800BA302BD120460221FAF775FF9DF82830FF2BF7
S3150800BA400CBF9DF829309DF83330102B15D1286886
S3150800BA50214600F6FC40324603F066F821A816F0A7
S3150800BA60D9F87BB0BDE8F08FB26A002ADFD1C648A4
S3150800BA7040F2F37122F0A7FEFEE7112BEED128461D
S3150800BA8021463246FFF7C6FEE8E7EA7B002AE5D0FC
S3150800BA90002BE3D1DDF82E0016F0E4F8804628687E
S3150800BAA0D0F8D837984502D100F2DC7905E000F5E0
S3150800BAB0F860414618F060FC81469DF8283020461B
S3150800BAC0002B14BF01210B21FAF72CFFE18B20462E
S3150800BAD0043989B2042206ABDDF82AA0FAF768FF12
S3150800BAE004288346BAD1E18B2046043989B215F079
S3150800BAF0DFFC0028B2D106F1100C614608A80DAF8C
S3150800BB00CDF80CC016F0FBFB0523284608A95246BB
S3150800BB10009719F057FD4946102221A815F0B1FFE4
S3150800BB20238CE28B0D21D21A01915B4621A82A218A
S3150800BB30009715F0ADFFDDF80CC021A8614610226C
S3150800BB40FBF7F8F821A831461022FBF7F3F821A8ED
S3150800BB500DF129010A22FBF7EDF8B4F82090218CA3
S3150800BB60E38B8B4218D911AB20464022FAF720FF07
S3150800BB70074611A90023009321A80A463B46FBF76E
S3150800BB801FF9218C20463A4611ABFAF771FF204679
S3150800BB903946FAF7C7FEE2E704230DF1160221A893
S3150800BBA007A98DF81630FBF799F99DF81620042A8F
S3150800BBB07FF454AF06A807A922F06AFB00287FF491
S3150800BBC04DAF2868D0F8D837984504D900F5F860FD
S3150800BBD04146FCF753FD49462046FAF7BDFE0DF1EE
S3150800BBE01703218C01222046FAF7E2FE204601219E
S3150800BBF0FAF798FEEB7B013B032B29D8DFE803F025
S3150800BC00060602029DF817300C2B04D1284608A90F
S3150800BC101AF019FB05E0286808A900F6FC401CF094
S3150800BC2091FBA8B1037F03F00703062B10D18369A4
S3150800BC30984503D103699A4506D20FE77FF60EAFFA
S3150800BC400023C0F81880C3600AF10103036106E007
S3150800BC509DF81730022B02D9042B40F0A3809DF8DB
S3150800BC6017300F2B3FF6FAAE01A252F823F000BFA9
S3150800BC70B1BC0008C1BC0008D3BC00085DBA000806
S3150800BC80E5BC00085DBA00085DBA0008F1BC00080A
S3150800BC9001BD00080DBD00081DBD00082BBD00082C
S3150800BCA03DBD000849BD00086DBD000899BD0008E6
S3150800BCB028682146324600F6FC4004F0B3FACDE681
S3150800BCC0286821463246434600F6FC4004F082FDC9
S3150800BCD0C4E6286821463246434600F6FC4004F08E
S3150800BCE0A1FDBBE6284621463246FEF7C7FCB5E667
S3150800BCF028682146324600F6FC4004F047FEADE6C9
S3150800BD00284621463246FEF7D3FEA7E6286821468E
S3150800BD10324600F6FC4003F06BFD9FE628462146B6
S3150800BD2032464346FEF7C6FF98E62868214632465D
S3150800BD30434600F6FC4005F0BFF88FE62846214644
S3150800BD403246FFF791F989E6EB7B033B012B07D8CF
S3150800BD5028682146324600F6FC4003F0F7FE7DE6E9
S3150800BD60284621463246FFF7EBFA77E6EB7B033B9C
S3150800BD70012B0BD8286821463246434600F6FC407C
S3150800BD8004F008FF6AE600BFF43103082846214696
S3150800BD903246FFF7A5FB61E6284621463246FFF7FD
S3150800BDA0BDFC5BE623F00403093B022B3FF656AEC7
S3150800BDB055E700BFF8B504460F461E46154622B994
S3150800BDC00B48482122F0FFFCFEE71046214694F86E
S3150800BDD0FF2011F04BF994F8FF30337037B1204645
S3150800BDE029463246BDE8F8401AF005BDF8BD00BF41
S3150800BDF0E935030838B5044694F8FF3015461A4461
S3150800BE00FF2A084604DC8C4202D8E218914205D97A
S3150800BE10084840F24B2122F0D6FCFEE7621A1A4483
S3150800BE20284422F0BEFA94F8FF2000202A4484F819
S3150800BE30FF2038BDE935030838B590F8FF300446C9
S3150800BE409A42154605D8884203D80A1A50199842C4
S3150800BE5005DD094840F2552122F0B5FCFEE75B1BDB
S3150800BE609A1A0846294422F09CFA94F8FF300020D2
S3150800BE705D1B84F8FF5038BDE9350308F0B5044664
S3150800BE80B3B00F4603A800212C2222F043FA94F8F7
S3150800BE9005314BB122F08DFCD4F80831C01A504B4D
S3150800BEA0984201DD1A2597E002220EA800211EF00D
S3150800BEB090FD0EA8022105F0B9FD4A490EA81EF00C
S3150800BEC0F1FE0EA81EF078FFD4F800010EA900F5C1
S3150800BED08E701EF034FA0646002878D094F804319D
S3150800BEE0B3B10A238DF8083094F8FF3002A902226C
S3150800BEF08DF80930FAF720FE0546002869D1304644
S3150800BF00214694F8FF20FAF717FE0546002860D167
S3150800BF104FF6FE739F4211D002238DF808308DF834
S3150800BF2009303B0A43EA0727304602A90422ADF83E
S3150800BF300A70FAF701FE054600284AD1D4F800012E
S3150800BF4007A900F6FC4019F0A9FAD4F8000103ADD8
S3150800BF5000F6FC4019F079FA034600F110072A4664
S3150800BF6018685968083303C2BB421546F7D14FF221
S3150800BF70BF03D4F80001ADF82E300023009300F576
S3150800BF808E70314603AA1EF097FC054608BB94F846
S3150800BF90043133B122F00DFC0123C4F8080184F8FA
S3150800BFA0053120461AF0F8F914F068FE022813D96C
S3150800BFB00320FAF755FC04460420FAF75DFC042131
S3150800BFC00090094A0320234622F0FFFB04E00325DC
S3150800BFD002E0304615F068FA284633B0F0BD00BFD7
S3150800BFE0DF930400863603085F36030810B5044657
S3150800BFF01A4B1B4A03601B4B4360A06002611A4A36
S3150800C00000234261194AC360A0610262184AC361EB
S3150800C0104262184AA0620263174AC3624263A06377
S3150800C020C36343648364016401F1B80021461EF0CA
S3150800C0300BFF206C04F11001B8301EF005FF206CD0
S3150800C04004F12001B8301EF0FFFE206C04F1300127
S3150800C050B8301EF0F9FE204610BD00BF8B36030827
S3150800C060903603082D6F0208296F020895360308D3
S3150800C0701F6E02089A360308316F02082DE9F3414C
S3150800C0801E460B78044613F0300F0D46174638D176
S3150800C0904B78022B35D11AF0BFFE14F0EFFD0228BB
S3150800C0A00DD90320FAF7DCFB80460B20FAF7E4FBF0
S3150800C0B00B210090144A0320434622F086FB636C4A
S3150800C0C01BB138463146A26C9847206C2946B830D1
S3150800C0D032461EF012FFA0B920461AF09DFE14F053
S3150800C0E0CDFD02280DD90320FAF7BAFB04460B202A
S3150800C0F0FAF7C2FB0B210090044A0320234622F0DC
S3150800C10064FB02B0BDE8F081E63603080E37030883
S3150800C1102DE9F04705468846144699460E8CC4B064
S3150800C1200236B6B2002799F80130F1199F4289B252
S3150800C13080F0F880404601220DF10B03FAF738FC2F
S3150800C140012840F0F18028461AF066FE14F096FDA4
S3150800C150022810D90320FAF783FB82460B20FAF748
S3150800C1608BFB9DF80B300090019303200B21704A3E
S3150800C170534622F02AFB9DF80B30112B00F2D4808F
S3150800C180DFE803F009192A344959667A888DD2D22C
S3150800C190D2D2A5ADBABF00238DF80C3008238DF88E
S3150800C1A00D302B6CD3F8B828CDF80E20D3F8BC2860
S3150800C1B0CDF812205CE0286C01238DF80C3000F6CF
S3150800C1C0FC4002238DF80D3019F04EF8030A43EAB5
S3150800C1D00020ADF80E008BE002238DF80C30012309
S3150800C1E08DF80D302B6C93F8303D91E02B6C93F85D
S3150800C1F0302D120700F1948003228DF80C200422BA
S3150800C2008DF80D20D3F8003E20461BBACDF80E3027
S3150800C21003A9062281E0286C04238DF80C3000F669
S3150800C220FC400A2303A98DF80D3003F051F9204686
S3150800C23003A90C2271E0286C05238DF80C3000F652
S3150800C240FC40292303A98DF80D301CF0A6FC37E025
S3150800C250286C00F6FC4019F0A3F90A22014603A847
S3150800C26010F004FF06238DF80C3008238DF80D30E6
S3150800C270204603A90A2250E0286C07238DF80C30C3
S3150800C28000F6FC40FF2303A901228DF80D3019F0B2
S3150800C290B2FA15E0284621461AF0C3FD3FE0002110
S3150800C2A003A8262222F036F8286C09238DF80C30CC
S3150800C2B000F66C00242303A98DF80D3015F0C7FF8E
S3150800C2C09DF80D202046023203A9D2B225E00E239E
S3150800C2D08DF80C3001238DF80D30642318E00F23F8
S3150800C2E08DF80C3002238DF80D300023ADF80E3092
S3150800C2F0204603A9042210E0284621461AF0B8FD74
S3150800C3000DE011238DF80C3001238DF80D30002334
S3150800C31020468DF80E3003A90322FAF70DFC20B942
S3150800C320013700E7002000E0022044B0BDE8F087AE
S3150800C3303D3703082DE9F0410E46B2B004461746CC
S3150800C34003A800212C221D4621F0E4FF7378022B56
S3150800C35040F0B48020461AF05FFD14F08FFC0228E6
S3150800C3600DD90320FAF77CFA80460B20FAF784FAEF
S3150800C3700B210090534A0320434622F026FA3846FA
S3150800C380398C022202ABFAF713FB022840F096809A
S3150800C3909DF80830122B40F091809DF80930122B39
S3150800C3A000F28C80337813F0300F1BD1206C3146A5
S3150800C3B0B8302A461EF0A1FDA0B920461AF02CFD79
S3150800C3C014F05CFC02280DD90320FAF749FA064650
S3150800C3D00B20FAF751FA0B2100903B4A032033460B
S3150800C3E022F0F3F902220EA800211EF0F2FA0EA896
S3150800C3F0022105F01BFB0EA834491EF053FC9DF8DC
S3150800C400093013B10EA81EF0D7FC206C0EA900F552
S3150800C4108E701DF094FF064600284FD005F11003D4
S3150800C42003F1100E07AD2A4618685968083303C287
S3150800C43073451546F7D1206C03AD00F6FC4019F09C
S3150800C44004F8034600F1100E2A461868596808339E
S3150800C45003C273451546F7D14FF2BF03ADF82E3028
S3150800C460236C20461B7D39468DF83030324602ABA8
S3150800C470FFF74EFE0346F0B9206C3146009400F5EE
S3150800C4808E7003AA1EF018FAA8B920461AF0C4FC42
S3150800C49014F0F4FB022811D90320FAF7E1F904464F
S3150800C4A00B20FAF7E9F90B210090094A03202346E5
S3150800C4B022F08BF902E0304614F0F6FF32B0BDE800
S3150800C4C0F08100BF663703088D37030895360308E1
S3150800C4D0BF3703082DE9F0411D460F46B2B003AC3D
S3150800C4E0064690460FCD0FC40FCD0FC495E807003A
S3150800C4F03B7884E8070013F0300F6FD17B78022B66
S3150800C5006CD130461AF088FC14F0B8FB02280DD915
S3150800C5100320FAF7A5F904460B20FAF7ADF90B2123
S3150800C5200090304A0320234622F04FF94046B8F8D7
S3150800C5302010022202ABFAF73BFA02284ED19DF8E8
S3150800C5400830122B4AD19DF80930122B46D8306C88
S3150800C5500021B8301EF095FC044600283ED0394626
S3150800C5600EA81EF036FC0EA81EF026FC20460EA9C4
S3150800C5709DF8B820FAF7E0FA68BB304641462246ED
S3150800C58002ABFFF7C5FD30BBE38B9DF8B8109942A7
S3150800C59004D10139204689B214F08AFF306C21464D
S3150800C5A0B83003AA1EF09BFCA8B930461AF034FC32
S3150800C5B014F064FB022811D90320FAF751F904464E
S3150800C5C00B20FAF759F90B210090074A0320234656
S3150800C5D022F0FBF802E0204614F066FF32B0BDE810
S3150800C5E0F08100BFE33703080C3803082DE9FF473D
S3150800C5F00F461646984605461AF00EFC14F03EFB02
S3150800C60002280DD90320FAF72BF904460B20FAF76E
S3150800C61033F90B210090424A0320234622F0D5F82D
S3150800C6203C7814F0300478D17A78022A75D13046ED
S3150800C630318C03ABFAF7BCF902286ED19DF80C30A1
S3150800C640122B6AD19DF80D30122B66D8318C023127
S3150800C6501FFA81F99DF80D20E3B29A4241D9304676
S3150800C660494601220DF10B03FAF7A2F9012854D124
S3150800C6709DF80B30092B1AD1286C00F66C0015F0C2
S3150800C68038FE28461AF0C8FB14F0F8FA022826D90C
S3150800C6900320FAF7E5F882460B20FAF7EDF80B21A6
S3150800C6A00090204A0320534622F08FF817E02846C8
S3150800C6B01AF0B2FB14F0E2FA022810D90320FAF7AE
S3150800C6C0CFF882460B20FAF7D7F89DF80B30009082
S3150800C6D0019303200B21144A534622F076F80134BD
S3150800C6E0B8E7286C3946B83042461EF006FCA0B9B1
S3150800C6F028461AF091FB14F0C1FA02280DD9032036
S3150800C700FAF7AEF804460B20FAF7B6F80B210090B4
S3150800C710064A0320234622F058F804B0BDE8F087FD
S3150800C7205938030884380308BC380308FB3803085B
S3150800C73037B5B1F87E200C46C2F30C03B3B91AF02C
S3150800C740F9FB14F09BFA01281FD90220FAF788F89A
S3150800C75005460720FAF790F8A38A0090019302206D
S3150800C76007210B4A2B4622F030F80EE003F5FF535B
S3150800C7701F33C3F30C0363F30C02A1F87E2023B91D
S3150800C78003B0BDE830401AF07EBC03B030BD00BF30
S3150800C7902939030837B504460122FBF7A7FD2046C9
S3150800C7A03D4B214640F8B83B3C4B4FF2BF02009345
S3150800C7B03B4B05F069F93B4B3B4A214604F58E7025
S3150800C7C005F0AEF8214604F5BE7001F0E7F82146FB
S3150800C7D004F53D7000F096F8214604F5A96000F0CE
S3150800C7E0CFF904F5F86504F2BC7016F0FBFE214695
S3150800C7F02846FBF7D1FE214604F668001FF001FC27
S3150800C800214604F66C00FAF7B3FB214604F61440F9
S3150800C810FBF7A2FF214604F6FC4001F061FD04F592
S3150800C8202150214608301DF087FB04F52550214686
S3150800C830183004F01BFE04F52B5021463030FFF764
S3150800C840D5FB214604F52D5000F032F8214604F5B3
S3150800C8502E5000F0ABF904F52F502146383000F081
S3150800C860FDFD04F5315021463C3006F009F804F583
S3150800C87032502146303006F039FA04F53350214655
S3150800C880343006F09DF828460849102217F014FDA2
S3150800C890204603B030BD00BF28EA020849710208E5
S3150800C8A0457102083D710208417102087939030889
S3150800C8B0034601604A6800F1100102F5034204329A
S3150800C8C002610F4A30B542619861416290F83610AC
S3150800C8D0002241F03F0180F8361090F83710002406
S3150800C8E041F03F0162F386110025C26102620273BC
S3150800C8F080F8371042608260C0E90A4530BD00BF43
S3150800C900A775020810B5044605F04AFB064BC4F89D
S3150800C9104C42C4F84432054B2046C4F8483200233A
S3150800C920C4F8503210BD00BF893903080D760208D5
S3150800C93070B50446D0F81002A4B000F6FC4018F012
S3150800C94031FC002800F01681002168220AA821F08F
S3150800C950E1FC20460E211AF028FE0546E8B90E230A
S3150800C9608DF81430294608230DF1160006228DF895
S3150800C970153021F0CFFC204605A9ADF81C508DF8DE
S3150800C9801B508DF81A508DF819508DF818508DF8DF
S3150800C99017508DF816501EF0CFFE204600211AF0CB
S3150800C9A004FE88B903238DF81530D4F810328DF8B3
S3150800C9B014008DF8160093F8C43820461B0205A902
S3150800C9C0ADF817301EF0B8FE204635211AF0EDFDF9
S3150800C9D080B935238DF8143006238DF815300423D5
S3150800C9E08DF81730654B8DF8160005A92046069375
S3150800C9F01EF0A2FE204602211AF0D7FD88B9D4F807
S3150800CA0010120223082201F6D7010DF116008DF83F
S3150800CA1014308DF8152010F029FB204605A91EF0C4
S3150800CA208BFE204607211AF0C0FDA8B9D4F81002DB
S3150800CA300723082500F6FC408DF814308DF81550AC
S3150800CA4018F009FC2A4601460DF1160010F00EFBF7
S3150800CA50204605A91EF070FE052120461AF0A5FD00
S3150800CA600146A8B9D4F810020523102500F5F86088
S3150800CA708DF814308DF8155017F019FC2A46014622
S3150800CA800DF1160010F0F2FA204605A91EF054FE24
S3150800CA90204603211AF089FDC8B9D4F81052032399
S3150800CAA005F6C605102128468DF814308DF81510A0
S3150800CAB021F0C7FB064629460DF11600324610F04E
S3150800CAC0D5FA204605A98DF815601EF035FE2046D4
S3150800CAD001211AF06AFD98B901238DF81430022352
S3150800CAE08DF81530D4F810322046B3F8C22805A9B7
S3150800CAF0C2F3072343EA0223ADF816301EF01CFEE4
S3150800CB00042120461AF051FD0146A0B910252A46EF
S3150800CB1001A821F0FFFB04230DEB03010DF116001C
S3150800CB202A468DF814308DF8155010F09FFA2046D5
S3150800CB3005A91EF001FE20460C211AF036FDB8B9EB
S3150800CB400C238DF81430D4F8102203238DF81530F1
S3150800CB50D2F82C182046C1F3072343EA0123ADF87F
S3150800CB60163092F8643805A98DF818301EF0E4FDE1
S3150800CB70002000E00E2024B070BD00BF001FFFE0BB
S3150800CB8010B5044605F02EFA064BC4F86C42C4F8F4
S3150800CB906432054B2046C4F868320023C4F8703264
S3150800CBA010BD00BF8E3903087576020870B50446B5
S3150800CBB00E46002505604560856049680C301431CD
S3150800CBC017F019F9194BE4646364194B2565A364D6
S3150800CBD06665736804F1700003F503430433A365BF
S3150800CBE0144B2466E36504F15803E3666566A56697
S3150800CBF014F004FD94F87630606D03F0FE0365F3D7
S3150800CC00410384F876304FF47A73A38304F1440120
S3150800CC10A4F87450B8301EF017F9074B606D84E815
S3150800CC201800214616F09CFF204670BD933903086C
S3150800CC300B770208C3770208FD76020830B504466A
S3150800CC40406D89B090F8303D9A0747D5CB0545D554
S3150800CC50A18B00F2BC7016F02CFD606D04F10C057A
S3150800CC6000F5255018301AF069F8A0B300211022F3
S3150800CC7003A821F04FFB00232046ADF81C308DF8A1
S3150800CC801E301AF022FD2246ADF81C00144928462B
S3150800CC9017F0C5F803A9284617F007F9606DBDF81F
S3150800CCA01C1000F2BC7016F0F5FC20461AF0F7FCD2
S3150800CCB013F0E4FF022811D90320F9F7D1FD044641
S3150800CCC00A20F9F7D9FD0A210090064A03202346CF
S3150800CCD021F07BFD02E0284617F0C7F809B030BD01
S3150800CCE007770208983903082DE9F0410546BCB0D4
S3150800CCF00DA80F4690461AF0BFFC28461AF0CFFC3E
S3150800CD0013F0BCFF02280DD90320F9F7A9FD044644
S3150800CD100A20F9F7B1FD0A2100906A4A0320234642
S3150800CD2021F053FD28460DF10A011AF0BBFC002834
S3150800CD3040F0C480022218A810211DF04AFE18A847
S3150800CD40022104F073FE604918A81DF0ABFF18A86D
S3150800CD501EF032F8686D18A900F58E701DF006FBF6
S3150800CD600646002800F0AA80B8F8222012238DF87B
S3150800CD700C30C2F3072343EA0223022403A9042240
S3150800CD808DF80D40ADF80E30F9F7D6FE002840F0C4
S3150800CD9092800822132308F118010DF11A008DF864
S3150800CDA019208DF8183010F061F9304606A90A22C4
S3150800CDB0F9F7C2FE00287ED1686D142300F6FC4000
S3150800CDC08DF810308DF8114018F04EFA030A43EA30
S3150800CDD00020ADF8120004A930460422F9F7ACFE8B
S3150800CDE0002868D1304611233A8C8DF81430FB8B15
S3150800CDF005A99B1A9BB2FF228DF815201A0A42EA4A
S3150800CE000323ADF816300422F9F796FE002852D10E
S3150800CE10398CFC8BA14211D2641AA4B2102C28BFFB
S3150800CE201024224609AB3846F9F7C2FD2146384692
S3150800CE30F9F778FD304609A92246E5E7686D11AC91
S3150800CE4000F6FC4018F001FB034600F110072246E5
S3150800CE5018685968083303C2BB421446F7D1BDF8AF
S3150800CE600A20686DC2F3072343EA0223ADF852305D
S3150800CE704FF2BF03ADF856300023009300F58E70CD
S3150800CE8031460DAA1DF018FDA8B928461AF007FC68
S3150800CE9013F0F4FE022811D90320F9F7E1FC044641
S3150800CEA00A20F9F7E9FC0A210090084A03202346DC
S3150800CEB021F08BFC02E0304614F0F6FA3CB0BDE8EF
S3150800CEC0F08100BFB6390308DE390308E3390308E1
S3150800CED02DE9F04F8046E3B013A80E4691461AF0A6
S3150800CEE0CBFB1EA81AF0D0FB02223EA800211DF09B
S3150800CEF070FDB1493EA81DF0D5FE3EA81DF05CFFA9
S3150800CF00D8F854003EA900F58E701DF02FFA074692
S3150800CF10002800F0478190F83030042262F3840339
S3150800CF2080F83030D8F8540005234FF0100B002154
S3150800CF3000F5F8608DF824308DF825B017F0B7F9AC
S3150800CF405A4601460DF1260010F090F8384609A910
S3150800CF501222F9F7F1FD0446002840F02581D8F899
S3150800CF6054000723082500F6FC408DF80C308DF890
S3150800CF700D5018F070F92A4601460DF10E0010F012
S3150800CF8075F8384603A90A22F9F7D6FD044600289B
S3150800CF9040F00A81D8F85410022301F6D7012A4630
S3150800CFA00DF11A008DF818308DF8195010F05EF84A
S3150800CFB0384606A90A22F9F7BFFD0446002840F0BC
S3150800CFC0F38003238DF83830D8F85430594603F6E1
S3150800CFD0C60A50468DF839B021F033F90446514651
S3150800CFE022460DF13A0010F041F8E2B28DF83920E8
S3150800CFF038460EA90232F9F79FFD0446002840F08C
S3150800D000D380D8F854000E2100F57F701EF0E1F9A0
S3150800D010014618B14278384602320FE00E232146FF
S3150800D02006220DF1BA008DF8B8308DF8B95021F006
S3150800D03071F93846ADF8C0402EA90A22F9F77CFDE9
S3150800D0400446002840F0B080D8F85400352100F591
S3150800D0507F701EF0BEF9014618B142783846023292
S3150800D06007E08DF8B900384635238DF8B8302EA973
S3150800D0700222F9F761FD0446002840F09580D8F8A9
S3150800D0805400042100F57F701EF0A3F9014618B17B
S3150800D09042783846023208E0384604238DF8B8301C
S3150800D0A010238DF8B9302EA91222F9F745FD04464A
S3150800D0B0002879D1D8F854000C2100F57F701EF0AD
S3150800D0C088F9014618B142783846023208E03846EF
S3150800D0D00C238DF8B83003238DF8B9302EA9052214
S3150800D0E0F9F72AFD044600285ED104238DF8053099
S3150800D0F0D8F854300622D3F8D83738461BBA01A9CF
S3150800D1008DF80420CDF80630F9F716FD04460028F8
S3150800D1104AD10FCE13AD0FC50FCE0FC596E807003F
S3150800D1204FF2BF0385E80700ADF86E3021F041FBEA
S3150800D13006462EA832361AF09FFA39960DF1B80E21
S3150800D14013AE0FCEAEE80F000FCEAEE80F0095E88F
S3150800D15007001EAE8EE807002EAD09F10201102267
S3150800D1603AA80FF083FF0FCD0FC60FCD0FC60FCD10
S3150800D1700FC695E80F0086E80F0038461EA940221C
S3150800D180F9F7DAFC98B908F17000394614F0C9FACB
S3150800D190D8F86C0008F15808404508D1322114F037
S3150800D1A063FD04E0032402E0384614F07DF92046C6
S3150800D1B063B0BDE8F08F00BFFA3903082DE9F041E6
S3150800D1C00C4698B007460DA816461AF055FA237865
S3150800D1D003F03003102B40F0B7806378022B40F041
S3150800D1E0B38038461AF05BFA13F048FD02280DD9C9
S3150800D1F00320F9F735FB04460A20F9F73DFB0A2117
S3150800D2000090534A0320234621F0DFFA30461221C4
S3150800D210042204AB1EF019F8002840F095809DF80A
S3150800D2201130022B40F09080304613210A2205ABBC
S3150800D2301EF00BF8002840F087809DF81530082B63
S3150800D24040F082803046112103AA0DF10E031EF02C
S3150800D2501CF80446002877D107F10C0840462146F9
S3150800D26016F040FE054600286ED0214614F0FEFA58
S3150800D27095F8303064F3861385F83030BDF80E40E3
S3150800D280BDF80C10CCB1102C28BF1024224630460D
S3150800D29008ABF9F78DFB284608A92246F9F74CFC96
S3150800D2A000284ED1BDF80C302344ADF80C30BDF83B
S3150800D2B00E301C1BADF80E40E0E7224623460095CB
S3150800D2C0304614F068F948F2FE030DF116010822FB
S3150800D2D013A8ADF844300FF0C9FEBDF81220404639
S3150800D2E0C2F3072343EA0223ADF856307B6D29467D
S3150800D2F01B7D0DAA8DF8583016F0FAFD08BB30468E
S3150800D3001521122208AB1DF0A0FFE8B938461AF01D
S3150800D310C6F913F0B3FC02280DD90320F9F7A0FAD1
S3150800D32004460A20F9F7A8FA0A210090094A0320B8
S3150800D330234621F04AFA38460DA908AAFFF7C8FD80
S3150800D34002E0284614F0B0F818B0BDE8F08100BF36
S3150800D350FF390308203A0308F7B50446406D0E4620
S3150800D36015462349224600F58E701DF0DFF8204643
S3150800D3701AF095F913F082FC02280DD90320F9F763
S3150800D3806FFA07460A20F9F777FA0A210090194A30
S3150800D39003203B4621F019FA606D2A46009400F5F1
S3150800D3A08E703146124B1DF087FA0546E0B92046C5
S3150800D3B01AF075F913F062FC02280FD90320F9F761
S3150800D3C04FFA07460A20F9F757FAF38B00900193AC
S3150800D3D003200A21084A3B4621F0F7F994F87630EB
S3150800D3E043F0020384F87630284603B0F0BD00BF48
S3150800D3F0C7770208363A0308543A03082DE9F0417C
S3150800D40090F876309DF818706FF3410380F87630FF
S3150800D41004460D4616461AF07AF9DFB9D5B1CEB1EB
S3150800D4206B78442B16D120461AF039F913F026FCEE
S3150800D43002280FD90320F9F713FA04460A20F9F748
S3150800D4401BFA234606900A210320034ABDE8F04149
S3150800D45021F0BBB9BDE8F0817D3A030810B5044652
S3150800D460184B00220360184B4360184BA0600361F9
S3150800D470174BC2604361A061C2614B6803F5034361
S3150800D48004330362134B436200F12003A062436333
S3150800D49047F2305383634FF6FF73C2620263A0F804
S3150800D4A07E30C0F8801001F1B80021461DF0CCFC92
S3150800D4B0D4F8800004F11001B8301DF0C5FC2046F0
S3150800D4C010BD00BFA63A0308DF770208AB3A030887
S3150800D4D0E7770208FD7702082DE9F0410546D0F8FE
S3150800D4E08000A8B00C46B8300021174698461DF0B3
S3150800D4F0CAFC0646002867D0214604A81DF069FC28
S3150800D50004A81DF059FC304604A99DF89020F9F7A7
S3150800D51013FB0446002859D110238DF808303046ED
S3150800D520012302A903228DF809308DF80A80F9F73C
S3150800D53003FB0446002849D16A6B05F120039A4289
S3150800D54003D1B8F1010F20D10AE095F83D20304605
S3150800D55005F13C010232F9F7EFFA0446B0BBF0E7F1
S3150800D560B5F87E200B238DF80C3002238DF80D308C
S3150800D570C2F3072343EA0223304603A90422ADF87F
S3150800D5800E30F9F7D9FA044600BBD5F880003146C3
S3150800D590B8303A461DF0A3FC0446B8B928461AF036
S3150800D5A01AF913F06BFB022813D90320F9F758F977
S3150800D5B005460A20F9F760F90A210090074A032070
S3150800D5C02B4621F002F904E0032402E0304613F06A
S3150800D5D06BFF204628B0BDE8F08100BFB03A0308CB
S3150800D5E02DE9F0439BB00F4615461E4604461AF031
S3150800D5F0F2F813F043FB02280DD90320F9F730F9A6
S3150800D60080460A20F9F738F90A2100903B4A032098
S3150800D610434621F0DAF828460A21422209AB1DF0D2
S3150800D62014FE814608B1FF235EE09DF82530402BA5
S3150800D630F9D8D4F8348004F120039845F3D10923A6
S3150800D640F17F8DF80830B37F022243EA0123ADF853
S3150800D6500A300B238DF80C30B4F87E308DF809208B
S3150800D66001339BB28DF80D201A0AA4F87E3042EADF
S3150800D6700323ADF80E3010220823494601250DF183
S3150800D68012008DF810308DF8112020F043FE49461F
S3150800D6902A460DF112008DF8115020F03BFE9DF838
S3150800D6A009209DF80D30D4F8800013449DF8112008
S3150800D6B006331A4400F52550183002A9D2B219F0DB
S3150800D6C079FB0028AFD109A9422204F13C000FF0EA
S3150800D6D0CDFC21F06EF84CF25033E0622363206AE9
S3150800D6E041461DF054FD2B462046394632465BB26C
S3150800D6F0FFF7F2FE1BB0BDE8F08300BFD03A03087F
S3150800D7002DE9F0410646D0F88000A8B00C46B8309E
S3150800D7100021174698461DF0B6FB054600283CD062
S3150800D720214604A81DF055FB04A81DF045FB284614
S3150800D73004A99DF89020F9F7FFF9044678BB102351
S3150800D7408DF80C302846012303A903228DF80D30E5
S3150800D7508DF80E80F9F7F0F9044600BBD6F880007C
S3150800D7602946B8303A461DF0BAFB0446B8B93046E1
S3150800D7701AF031F813F082FA022813D90320F9F7C0
S3150800D7806FF805460A20F9F777F80A210090074A44
S3150800D79003202B4621F019F804E0032402E028466A
S3150800D7A013F082FE204628B0BDE8F081EB3A030864
S3150800D7B0F0B50646B3B02C220C4603A8002120F08B
S3150800D7C0A9FD02220EA800211DF003F90EA80221C8
S3150800D7D004F02CF923490EA81DF064FAD6F8800047
S3150800D7E00EA900F58E701CF0C1FD054688B32346C8
S3150800D7F007AC03F11007224618685968083303C2B4
S3150800D800BB421446F7D14FF2BF03D6F88000ADF8F5
S3150800D8102E300023009300F58E70294603AA1DF0CA
S3150800D8204BF80446B8B9304619F0D5FF13F026FA76
S3150800D830022813D90320F9F713F805460A20F9F741
S3150800D8401BF80A210090084A03202B4620F0BDFF4A
S3150800D85004E0032402E0284613F026FE204633B0EF
S3150800D860F0BD00BF0D3B0308123B03081FB5044675
S3150800D8700B238DF80C3002238DF80D30B0F87E306E
S3150800D88003A901339BB2A0F87E30D0F880001A0AAB
S3150800D89000F5255042EA032318300422ADF80E306D
S3150800D8A019F088FA204619F096FF13F0E7F90228CE
S3150800D8B00DD90320F8F7D4FF04460A20F8F7DCFF51
S3150800D8C00A210090034A0320234620F07EFF04B075
S3150800D8D010BD00BF303B03082DE9FF410F46154632
S3150800D8E01E46044619F077FF13F0C8F902280DD929
S3150800D8F00320F8F7B5FF80460A20F8F7BDFF0A218E
S3150800D9000090254A0320434620F05FFF2846102151
S3150800D910032202AB1DF099FC00283AD19DF8093084
S3150800D920012B36D128460B21042203AB1DF08DFCB2
S3150800D93078BB9DF80D30022B2BD1BDF80E20C2F313
S3150800D940072343EA0223B4F87E209BB29A4219D1F0
S3150800D9509DF90A5004F12008012D07D0206A414696
S3150800D9601DF0C3FB2046FFF781FF0BE020F021FFE7
S3150800D9704CF25033E0622363206A41461DF007FCEF
S3150800D9802B4600E0FF232046394632465BB2FFF7B6
S3150800D990B7FE04B0BDE8F0814F3B030810B5044656
S3150800D9A0274B284A0360284B4360A0600261274A38
S3150800D9B000234261264AC360A0610262254AC36108
S3150800D9C04262254AA062C362C0F85021C4F85401D5
S3150800D9D0C0F858314A6802F503420432C0F85C219F
S3150800D9E01E4AC0F86021C4F86401C0F86831C0F85E
S3150800D9F06C3100F5AE73C0F87031C0F8741119F0C7
S3150800DA0003FFD4F874012146B8301DF01DFAD4F886
S3150800DA10740104F11001B8301DF016FAD4F8740137
S3150800DA2004F12001B8301DF00FFAD4F8743104F56A
S3150800DA30A871586808301EF096F9204610BD00BF38
S3150800DA406C3B0308713B03087D790208817902085B
S3150800DA50763B030879790208677A0208157A02087C
S3150800DA60034637B500F5907493F8522091F8225082
S3150800DA70243395423CBF02F1FF3283F82E20A3429D
S3150800DA80F2D1072381F82230002381F8233019F0D8
S3150800DA90B7FE13F0F3F802280DD90320F8F7E0FED5
S3150800DAA004460320F8F7E8FE009003200146034ADF
S3150800DAB0234620F08AFE03B030BD00BF7B3B030837
S3150800DAC0F0B50446B7B02C220D4607A8002120F071
S3150800DAD021FC022212A810211CF07BFF444912A83F
S3150800DAE01DF0E0F812A81DF067F9D4F8740112A920
S3150800DAF000F58E701CF023FC064600285BD02946EC
S3150800DB0000238DF8083010238DF8093005F110022E
S3150800DB100DF10A0351F8040B914243F8040BF9D1AD
S3150800DB20304602A91222F9F707F80546002843D11C
S3150800DB3040F2FF33D4F87401ADF82C3000F6FC40FF
S3150800DB404FF40073ADF83A3017F07FFC034607AD83
S3150800DB5000F110072A4618685968083303C2BB4201
S3150800DB601546F7D14FF2BF03D4F87401ADF83E302D
S3150800DB70037D31468DF840300023009300F58E7002
S3150800DB8007AA1CF099FE0546B0B9204619F038FEDA
S3150800DB9013F074F802280FD90320F8F761FE074638
S3150800DBA00320F8F769FE009003200146114A3B4618
S3150800DBB020F00BFE00E00325D4F8707104F5AE736F
S3150800DBC09F420CD120F0F5FD4FF47A73C4F8680132
S3150800DBD0C4F86C31D4F85C0139461DF0D8FA1DB189
S3150800DBE016B1304613F060FC284637B0F0BD00BFCA
S3150800DBF0713B0308993B03082DE9F0411F4605468A
S3150800DC00B2B00C46904600212C2203A820F082FBD5
S3150800DC10002F0CBF1021002102220EA81CF0D9FEED
S3150800DC2039490EA81DF03EF80EA81DF0C5F8D5F81E
S3150800DC3074010EA900F58E701CF081FB06460028BB
S3150800DC4058D021461222F8F777FF0446002853D108
S3150800DC50304641460A22F8F76FFF044600284BD1A2
S3150800DC6047B940F2FF33ADF81C304FF40073ADF8F6
S3150800DC702A3004E007A8394610220FF0F7F9D5F83C
S3150800DC80740103AC00F6FC4017F0DFFB034600F115
S3150800DC901007224618685968083303C2BB4214465F
S3150800DCA0F7D14FF2BF03D5F87401ADF82E30037DD6
S3150800DCB031468DF830300023009300F58E7003AAA4
S3150800DCC01CF0FAFD0446B8B9284619F099FD12F079
S3150800DCD0D5FF022813D90320F8F7C2FD054603200D
S3150800DCE0F8F7CAFD009003200146084A2B4620F0A3
S3150800DCF06CFD04E0032402E0304613F0D5FB204611
S3150800DD0032B0BDE8F08100BF6C3B0308B53B0308A1
S3150800DD102DE9F04F98460B788FB013F0300F054673
S3150800DD200F46144640F0BD804B78022B40F0B98070
S3150800DD3019F066FD12F0A2FF022814D90320F8F79D
S3150800DD408FFD06460320F8F797FDB8F81E100090D9
S3150800DD500A0A42EA012292B2032001920146524A75
S3150800DD60334620F032FD20460021122209AB1DF071
S3150800DD706CFA002840F095809DF82530102B40F06D
S3150800DD809080204603210A2206AB1DF05EFA002881
S3150800DD9040F087809DF81930082B40F08280204695
S3150800DDA00221042203AB1DF050FA0646002878D15A
S3150800DDB09DF80D30022B74D1062120460A4604AB85
S3150800DDC01DF043FA40B99DF81130042B69D1DDF8EE
S3150800DDD0120013F047FF064605F1400405F5B07A30
S3150800DDE0A4F1100948460DF1260115F0F3FB834608
S3150800DDF0002853D1E37C012B12D0022B4ED12046AA
S3150800DE000DF11A01082220F043FA30B1284609A973
S3150800DE1006AA5B46FFF7F0FE43E0A3689E4240D29F
S3150800DE200DF11A01082220460FF020F9BDF80E2040
S3150800DE302846C2F3072343EA0223A3810023E3818A
S3150800DE402374637402234946A660E37419F0EEFC52
S3150800DE50D5F874013946B83042461DF04EF8A0B9D7
S3150800DE60284619F0CDFC12F009FF02280DD9032027
S3150800DE70F8F7F6FC81460320F8F7FEFC009003202D
S3150800DE8001460A4A4B4620F0A0FCD5F874010DF16C
S3150800DE90260100F61440002216F0DDFB2434544512
S3150800DEA09ED10FB0BDE8F08FD13B0308023C0308B2
S3150800DEB02DE9F0411F460B7892B013F0300F064655
S3150800DEC00C46154640F0C0804B78022B40F0BC80CB
S3150800DED019F096FC12F0D2FE02280DD90320F8F7A5
S3150800DEE0BFFC80460320F8F7C7FC009003200146D4
S3150800DEF0574A434620F069FC384615F084FAE0B9DB
S3150800DF00D6F874012146B8303A461CF0F6FFA0B997
S3150800DF10304619F075FC12F0B1FE02280DD903201F
S3150800DF20F8F79EFC04460320F8F7A6FC00900320A9
S3150800DF300146484A234620F048FC2846002112227A
S3150800DF400DAB1DF082F900287ED19DF83530102BD7
S3150800DF507AD1284603210A2206AB1DF076F9002855
S3150800DF6072D19DF81930082B6ED1D6F87431DC6859
S3150800DF70B4B120460DF13601102220F089F968B9AE
S3150800DF80D6F8740100F6FC4017F062FA15F0C2FAEA
S3150800DF900DF11A01082220F07BF9B8BB6469E7E79E
S3150800DFA0D6F874010DF10F0100F6FC401AF073F96A
S3150800DFB00DF11A010546082204A80FF057F89DF836
S3150800DFC0103083F002038DF810309DF80F309C4214
S3150800DFD03ADA2B7F03F00702062A14D1DB0612D49D
S3150800DFE005F1220705F1620838460DF1360115F0EC
S3150800DFF0E9FA28B1284604A9082220F049F958B9AF
S3150800E00010374745F0D101348035DEE7D6F874017C
S3150800E010214615F049FE17E000211022384620F067
S3150800E02079F91022002109A820F074F948F2FE03B4
S3150800E03009A82946ADF8243015F074FA30460DA91A
S3150800E04006AA09ABFFF7D8FD12B0BDE8F08100BFFC
S3150800E050343C0308613C03082DE9F0410546B2B09B
S3150800E0608846174600212C2203A81E4620F052F99E
S3150800E07002220EA800211CF0ACFC43490EA81CF095
S3150800E08011FE0EA81CF098FED5F874010EA900F52D
S3150800E0908E701CF054F90446002872D041461222AC
S3150800E0A0F8F74AFD002869D1204639460A22F8F7CA
S3150800E0B043FD002862D1D5F87401022300F6FC401E
S3150800E0C08DF808308DF8093017F0CEF8030A43EAC0
S3150800E0D00020ADF80A0002A920460422F8F72CFD14
S3150800E0E000284BD16EBB389B07AE03F110073246AA
S3150800E0F018685968083303C2BB421646F7D1D5F8E3
S3150800E100740103AE00F6FC4017F09FF9034600F1D0
S3150800E1101007324618685968083303C2BB421646C8
S3150800E120F7D14FF2BF03D5F87401ADF82E300023AE
S3150800E130009300F58E70214603AA1CF0BDFBE8B9D2
S3150800E14006E0204631460622F8F7F6FCB0B9CAE7DB
S3150800E150284619F055FB12F091FD022811D9032023
S3150800E160F8F77EFB04460320F8F786FB00900320A9
S3150800E1700146064A234620F028FB02E0204613F013
S3150800E18093F932B0BDE8F081763B0308993C030861
S3150800E1902DE9F0431D460B788FB003F03003102BA2
S3150800E1A00746144640F096804B78022B40F0928042
S3150800E1B019F026FB12F062FD022813D90320F8F79E
S3150800E1C04FFB06460320F8F757FB0090E98B032020
S3150800E1D00A0A42EA012292B2019201463F4A3346AE
S3150800E1E020F0F3FA20460021122209AB1DF02DF883
S3150800E1F0044600286ED19DF82530102B6AD10323DA
S3150800E2008DF8183006238DF810304FF008080423CF
S3150800E210D7F874010DF126018DF819808DF81130A3
S3150800E22015F018FD0646D7F8740100F6FC4086B1CD
S3150800E23017F00EF915F06EF91035014642460DF144
S3150800E2401A000EF013FF0095384609A906AA2346B8
S3150800E2503EE00DF10F011AF01EF8044605E008F13C
S3150800E2601008C84513D1013680349DF80F309E42F8
S3150800E27030DA237F03F00702062AF4D1DB06F2D44C
S3150800E280637F032BEFD804F1220804F162094046A4
S3150800E2900DF1260115F09EF90028E0D12146082245
S3150800E2A00DF11A000EF0E2FE9DF81A30103583F0D3
S3150800E2B002038DF81A3020F07CFAA368C01A13F00E
S3150800E2C0D1FCCDF812003846009509A906AA04AB78
S3150800E2D0FFF7C2FE0FB0BDE8F08300BFBC3C0308E1
S3150800E2E02DE9F3410D460446FBF7E4FC6968524AFA
S3150800E2F001F503410023009404F5DE70043103F0B0
S3150800E300ABFC6B6804F5FC7203F503430433C4F8ED
S3150800E310F8314A4BC4F80042C4F8FC31C4F80C2260
S3150800E3206A68002302F503420432C4F81022444AFC
S3150800E330C4F80432C4F8142204F50472C4F824227A
S3150800E340404AC4F80832C4F828223F4AC4F818429A
S3150800E350C4F82C223D4AC4F81C32C4F838223C4A78
S3150800E360C4F82032C4F83042C4F83432C4F83C2227
S3150800E370C4F84042C4F8443204F5147704F26E2512
S3150800E38004F64A362846243516F02EF8B542F9D151
S3150800E39004F5DA5604F5336804F64E350E36284683
S3150800E3A0803516F021F8B542F9D194F834300025B5
S3150800E3B043F0030384F8343041F6303340F2FF1259
S3150800E3C0E55441F63A332946E252404684F8485223
S3150800E3D04FF480521FF09EFF3846294640F6DC026D
S3150800E3E01FF098FF41F63C337822E25441F63D335C
S3150800E3F01022E25441F63E331722E25441F63F33E7
S3150800E4004022E25441F6453204F5DA531D602023D2
S3150800E41084F82C3B3F23A35441F64632A35441F6D5
S3150800E42048332046E55041F644330122C4F84C529D
S3150800E430E25402B0BDE8F0810B8D02080F8D020888
S3150800E44009820208ED3C0308958A0208F23C030893
S3150800E450998A02083E29F7B504460D4605D82423AD
S3150800E4604B4303F51476861904D11E48982120F0EB
S3150800E470AAF9FEE7034493F8732203F51C73C2F363
S3150800E480801757BB42F04002DA7020F092F93946FD
S3150800E4900822B06030461FF03DFF94F84832013339
S3150800E4A084F8483220F085F9C4F84C02204616F064
S3150800E4B0F9FD12F0E3FB022810D90320F8F7D0F98A
S3150800E4C004460220F8F7D8F902218DE82100064A09
S3150800E4D00320234620F079F900E03F25284603B0BB
S3150800E4E0F0BD00BFF73C03086B3D0308C37B73B55B
S3150800E4F0032B04460D4603D00068082115F0B8FB27
S3150800E5002946204616F0B4FE0025032304F14401EB
S3150800E510E373606C84F840501CF0E7FD204619F060
S3150800E5206FFB236801265E7541F64533E25C2423BA
S3150800E53003FB0243201D83F8722216F0ADFD41F657
S3150800E5404833E050206800F5255018301AF0CCFF03
S3150800E5504FF47A7104F5FC7013F086FB48F2083222
S3150800E56023685B689E54022283F854202B4694F84D
S3150800E5702C1B8B420FDA04EBC31292F84C2B02F0D9
S3150800E5800702012A05D104F50470642113F06CFB17
S3150800E59001E00133EDE7204616F084FD12F06EFB2C
S3150800E5A002280DD90320F8F75BF904460220F8F78C
S3150800E5B063F902210090044A0320234620F005F956
S3150800E5C0002002B070BD00BF853D0308C37B2DE95E
S3150800E5D0F743042B04460D4603D00068082115F0BE
S3150800E5E047FB41F645392946204616F041FE0025E7
S3150800E5F0042304F14401E373606C84F840501CF072
S3150800E60074FD204619F0FCFA204616F069FF2368C7
S3150800E6104FF0010883F8158014F80930242606FB04
S3150800E6200342271D82F87232384616F035FD41F648
S3150800E63048334FF47A71E05004F5FC7013F014FB7C
S3150800E64014F8093006FB034620F0B3F8C6F858025A
S3150800E650206800F5255018301AF02DFF206800F5BF
S3150800E6603D7018F0A9FF206800F5A96018F0D0FFE2
S3150800E670206804F50A71B8301CF0E6FB206804F53A
S3150800E6800E71B8301CF0E0FB48F2083223685B686C
S3150800E69003F80280022283F854202B4694F82C1B98
S3150800E6A08B420FDA04EBC31292F84C2B02F00702E6
S3150800E6B0012A05D104F50470642113F0D5FA01E0A6
S3150800E6C00133EDE7204616F0EDFC12F0D7FA0228E2
S3150800E6D012D90320F8F7C4F804460220F8F7CCF854
S3150800E6E00546384616F0D8FC00950190022103200D
S3150800E6F0034A234620F069F8002003B0BDE8F083FA
S3150800E7009D3D03083E29F7B504460D4663D82426E1
S3150800E71006FB010616F514765DD0C37B042B5CD187
S3150800E72016F0C0FC12F0AAFA02280ED90320F8F750
S3150800E73097F807460220F8F79FF802218DE821008E
S3150800E740274A03203B4620F040F82146242303FBB2
S3150800E750054393F8732202F0BF0242F0800283F861
S3150800E7607322337F00226FF3020333773F2386F841
S3150800E770223091F87232AB420BD13F2381F87232C4
S3150800E780242303FB024393F873026FF3850083F88F
S3150800E790730201323F2A01F12401EAD194F8483282
S3150800E7A0013384F8483220F004F8C4F84C02206893
S3150800E7B0294600F5BE7019F04CF82068A90200F544
S3150800E7C02550183001F47C411BF095FA204619F0C3
S3150800E7D017FA002002E0072000E00E2003B0F0BD83
S3150800E7E0B83D0308F0B5054687B010220F4602A8C3
S3150800E7F000211FF08FFD284616F0F5FE0646002874
S3150800E80000F0908028463146002216F001FF0446A3
S3150800E810002840F089802846314617F04AF8044611
S3150800E820002840F08180EB7B042B28D8DFE803F032
S3150800E8300309191010003F4840F231211FF0C3FFA9
S3150800E840FEE7284631463C4A022316F0FAFF13E053
S3150800E85028463146394A012316F0F3FF04460028B4
S3150800E86062D12846314616F0F9FE044600285BD1E7
S3150800E8702846314616F0ACFF0446002854D10FBB93
S3150800E88005F5D95405F5D957103418371FF0B3FFD5
S3150800E89004F8010FBC42F9D141F63033022705F5D9
S3150800E8A0D952EF54284631461132082316F023FF71
S3150800E8B00446C8BBFF238DF808308DF809708DF81B
S3150800E8C0177013E0384619F0E3F82846314607F181
S3150800E8D00C02082316F00FFF044628BB48F2FE0375
S3150800E8E002A83946ADF8083014F01CFE2846314611
S3150800E8F002AA17F019F90446B0B9284616F0D2FB51
S3150800E90012F0BCF902280DD90320F7F7A9FF04462F
S3150800E9100220F7F7B1FF02210090094A0320234697
S3150800E9201FF053FF002402E0304612F0BDFD2046DA
S3150800E93007B0F0BDF73C0308DF410308EA3C0308CB
S3150800E940D53D03080138C0B202289ABF014B185CAE
S3150800E95010207047E63C03082DE9F04F8FB00646B5
S3150800E9608946154616F03FFE0446002800F0D0807A
S3150800E97090F83030032262F38403C58580F830307E
S3150800E98021463046112216F043FE0546002840F07F
S3150800E990C1800EAF1A2307F82C3D204639460222BD
S3150800E9A0F8F7CAF80546002840F0B48081238DF8A8
S3150800E9B0103002238DF8113020238DF81230336879
S3150800E9C08DF8130093F8643820465B0648BF282361
S3150800E9D004A94FF00402B4F81E8048BF8DF812301F
S3150800E9E0F8F7AAF80546002840F0948031684FF0F9
S3150800E9F0080B022301F6D7015A460DF11A008DF8C5
S3150800EA0018308DF819B00EF031FB204606A90A22F7
S3150800EA10F8F792F8054600287CD103238DF82430B0
S3150800EA203368102103F6C60A50468DF825101FF0E4
S3150800EA3008FC054651462A460DF126000EF016FB3F
S3150800EA40EAB28DF82520204609A90232F8F774F8AB
S3150800EA50054600285ED13068594600F5255018301D
S3150800EA6018F07BF90146D8B9306812234FF0020A2C
S3150800EA7000F52E508DF814308DF815A018F025FEE7
S3150800EA809DF81520030A43EA0020ADF8160005A9EB
S3150800EA9020465244F8F750F8054600283AD106E0D1
S3150800EAA0427820460232F8F747F888BBDCE7A37FAE
S3150800EAB0A8F10201C8EB030389B252468DF80D305E
S3150800EAC020463B46F7F7D4FF1FF095FEFB23B0FB25
S3150800EAD0F3F202FB1303214630464A469BB217F06F
S3150800EAE02DF90546B0B9304616F0DCFA12F0C6F82C
S3150800EAF002280DD90320F7F7B3FE04465046F7F768
S3150800EB00BBFE51460090074A032023461FF05DFED0
S3150800EB10002502E0204612F0C7FC28460FB0BDE8E3
S3150800EB20F08F00BFF03D03082DE9F04389B00F468A
S3150800EB309146804616F0B6FA12F0A0F802280DD9CA
S3150800EB400320F7F78DFE04460220F7F795FE02210B
S3150800EB500090404A032023461FF037FE98F83430C9
S3150800EB609B0701D4002470E03D8CFC8BA5426AD239
S3150800EB7002AB384629460222F7F71AFF9DF80830F5
S3150800EB801A2B9DF8093003D002331D44ADB2EDE7C8
S3150800EB900433AE1C1D44B6B2ADB2AE422FD23846CF
S3150800EBA03146022203ABF7F703FF9DF80C40022C0F
S3150800EBB00CD0802C1DD104AB384631460422F7F719
S3150800EBC0F7FE9DF81130022B13D03CE00A22384696
S3150800EBD0314605ABF7F7ECFE9DF81520082A32D129
S3150800EBE0D8F800000DF1160100F6D7001FF050FB0B
S3150800EBF070B19DF80D3002331E44B6B2CDE74046DB
S3150800EC0009F11001FA8DFFF7A7FE04460028A9D0DE
S3150800EC10404616F047FA12F031F8012815D90220B5
S3150800EC20F7F71EFE05460720F7F726FE0646204696
S3150800EC30F7F730FE0096019007210220064A2B4678
S3150800EC401FF0C3FD01E00624E2E7204609B0BDE84F
S3150800EC50F08300BF113E0308353E0308F0B587B0C0
S3150800EC6006460F4616F0BFFC054600286DD030460E
S3150800EC7029460D2216F0CCFC0446002867D13046FA
S3150800EC80294616F0EBFC0446002860D13046294692
S3150800EC9016F09EFD0446002859D13A7F3046C2F345
S3150800ECA0C002294682F0010216F0B6FD0446002885
S3150800ECB04DD122463046294616F07DFE04460028E8
S3150800ECC045D13046294616F0A4FE044600283ED112
S3150800ECD030462946214A022316F0B3FD0446B0BB46
S3150800ECE0384618F0E1FE3046294607F1680208233F
S3150800ECF016F001FD044650BB2146102202A81FF05B
S3150800ED0009FB48F2FE0302A83946ADF8083014F0AC
S3150800ED1009FC3046294602AA16F006FF0446B0B991
S3150800ED20304616F0BFF911F0A9FF02280DD90320C5
S3150800ED30F7F796FD04460220F7F79EFD022100909C
S3150800ED40074A032023461FF040FD002402E0284618
S3150800ED5012F0AAFB204607B0F0BD00BFEB3C030843
S3150800ED606C3E030870B50E4611460546144619F062
S3150800ED70F6FB864216D1A4123F2C05D0242202FBAC
S3150800ED80045414F5147405D1074840F6E6511FF0EB
S3150800ED901AFDFEE73F2384F822302846BDE8704076
S3150800EDA018F02EBF70BD00BFF73C0308F0B5054646
S3150800EDB0B7B02C220F4607A800211FF0ABFA022293
S3150800EDC012A800211BF005FE12A8022102F02EFE51
S3150800EDD04D4912A81BF066FF12A81BF0EDFF286824
S3150800EDE012A900F58E701BF0AAFA0646002800F054
S3150800EDF0828001238DF8103008238DF811302B6896
S3150800EE0004A9D3F8B828CDF81220D3F8BC28CDF831
S3150800EE1016200A22F7F790FE044600286DD141F61F
S3150800EE204633EB5C3E2B10D904238DF80830304668
S3150800EE30012302A903228DF809308DF80A70F7F725
S3150800EE407BFE0446002858D112E0022293408DF832
S3150800EE500C208DF80D2003F0FC03304603A904228C
S3150800EE60ADF80E30F7F768FE0446002845D1DBE713
S3150800EE7028460BA916F0EFFA044600283DD1284685
S3150800EE8016F0E3FA034607AC00F1100722461868A5
S3150800EE905968083303C2BB421446F7D14FF2BF0381
S3150800EEA02868ADF83E30009500F58E70314607AA01
S3150800EEB0164B1BF001FD0446F8B9284616F0F2F881
S3150800EEC011F0DCFE02281BD90320F7F7C9FC05461A
S3150800EED00220F7F7D1FCBDF83A100090C1F30722DB
S3150800EEE042EA012292B2019203200221084A2B46E5
S3150800EEF01FF06BFC04E0032402E0304612F0D4FA5B
S3150800EF00204637B0F0BD00BFED3C0308778F0208F6
S3150800EF10983E030838B5C37B04460D46002B4BD0F4
S3150800EF20032B4BD018F0CCFD002849D0002224230F
S3150800EF3003FB024393F8731293F86C0201F0BF01C6
S3150800EF406FF3C71183F8731201323F216FF3020082
S3150800EF508A4283F86C0283F87212E8D104F5DE70EF
S3150800EF601CF0D4F9206800F5BE7018F04DFC206836
S3150800EF70012100F6144015F03BFDE37B0021012B2F
S3150800EF8084F8751007D0022B11D120462946BDE812
S3150800EF903840FFF70BBF2046FFF724FC054680B92B
S3150800EFA004F5FC704FF47A7112F05EFE09E006482B
S3150800EFB0F3211FF008FCFEE70E2502E0002500E01D
S3150800EFC01D25284638BD00BFF73C0308F0B50546A1
S3150800EFD0B7B000212C2207A81FF09CF9022212A81C
S3150800EFE000211BF0F6FC12A8022102F01FFD36498B
S3150800EFF012A81BF057FE12A81BF0DEFE286812A9FD
S3150800F00000F58E701BF09BF90746002854D041F690
S3150800F0104533EB5C0226B34003F0FC0303A9042244
S3150800F0208DF80C608DF80D60ADF80E30F7F784FD9D
S3150800F0300446002842D101238DF8103008238DF8A4
S3150800F04011302B683846D3F8B82804A9CDF8122011
S3150800F050D3F8BC28CDF816200A22F7F76DFD04462A
S3150800F06060BB28460BA916F0F6F9044630BB4FF2EA
S3150800F070BF032868ADF83E300094234600F58E702D
S3150800F080394607AA1BF018FC0446B8B9284616F0F4
S3150800F09009F811F0F3FDB04213D90320F7F7E0FBA6
S3150800F0A005463046F7F7E8FB31460090074A032045
S3150800F0B02B461FF08AFB04E0032402E0384612F0D0
S3150800F0C0F3F9204637B0F0BDF23C0308BE3E03080C
S3150800F0D02DE9F04106460068ACB08846B8300021F4
S3150800F0E014461F461BF0CDFE0546002800F0898011
S3150800F0F0414608A81BF06DFE08A81BF05DFE2846D1
S3150800F10008A99DF8A020F7F717FD002876D1012356
S3150800F1103E2C8DF80D304FF0040894BF00230123D0
S3150800F120284603A903228DF80C808DF80E30F7F7D0
S3150800F13003FD002862D13E2C08D930682946B8302C
S3150800F1403A461BF0CCFE002858D141E002239C40E9
S3150800F15004F0FC04284604A94246ADF812408DF88E
S3150800F16010308DF81130F7F7E7FC0446002845D132
S3150800F17007238DF8143009238DF8153096F8483290
S3150800F1800DF11700214608228DF816301FF0C2F837
S3150800F1902046242202FB006292F87322C3B252066A
S3150800F1A00CD52CAA02EBD301802203F0070342FAFE
S3150800F1B003F311F8992C134301F8993C01303F28C1
S3150800F1C0E7D1284605A90B22F7F7B6FCB0B9B4E78C
S3150800F1D0304615F067FF11F051FD022811D90320BA
S3150800F1E0F7F73EFB04460220F7F746FB022100909C
S3150800F1F0054A032023461FF0E8FA02E0284612F0E3
S3150800F20053F92CB0BDE8F081DC3E03082DE9F04740
S3150800F2101F460B7888B013F0300F04460E46914609
S3150800F22040F0D8804D78022D40F0D48015F03AFF92
S3150800F23011F024FD02280DD90320F7F711FB8046AB
S3150800F2402846F7F719FB29460090644A03204346E7
S3150800F2501FF0BBFA484601210A2205AB1BF0F5FF51
S3150800F260002840F0B7809DF81530082B40F0B28092
S3150800F27048460421032203AB1BF0E7FF002840F0B1
S3150800F280A9809DF80D30012B40F0A480054604F5B1
S3150800F290147A242303FB054393F873325FFA85F83F
S3150800F2A0580608D550460DF1160108221EF0F0FF43
S3150800F2B0002800F0898001353F2D0AF1240AE8D19B
S3150800F2C09DF80E30022B04D0C0F08480042B08D998
S3150800F2D080E0204618F040FE41F63D33E35C834269
S3150800F2E071D948460221042204AB1BF0AEFF30BB9D
S3150800F2F09DF81130022B6DD1BDF81230C3F3850885
S3150800F300B8F13F0F5FFA88F519D0242202FB08F2FC
S3150800F31002F51470224492F873322044590605D532
S3150800F3200DF1160108221EF0B3FF40B9242303FB92
S3150800F330084393F873325A0608D4DB0906D02046E8
S3150800F34018F0D3FB3E28804627D81BE020462946DE
S3150800F350FFF780F83E288046F1D8204615F0A2FE31
S3150800F36011F08CFC02280DD90320F7F779FA054627
S3150800F3700220F7F781FA02210090194A03202B464A
S3150800F3801FF023FA242308AA03FB084352F80A0DA0
S3150800F39003F51473516803C316E0204615F082FE80
S3150800F3A011F06CFC02280FD90320F7F759FA054625
S3150800F3B00220F7F761FA022100900A4A03202B4639
S3150800F3C01FF003FA00E0A8462046314642463B466F
S3150800F3D0FFF77EFE08B0BDE8F08700BFF83E0308D9
S3150800F3E01A3F0308453F03082DE9F0431F460B78EB
S3150800F3F087B013F0300F04460D46904660D14E781C
S3150800F400022E5DD115F04EFE11F038FC02280DD9FA
S3150800F4100320F7F725FA81463046F7F72DFA3146E5
S3150800F4200090294A03204B461FF0CFF94046022197
S3150800F430042202AB1BF009FF002841D19DF80960A0
S3150800F440022E3DD1404601210A2203AB1BF0FDFEE8
S3150800F450B0BB9DF80D20082A32D1BDF80A30C3F397
S3150800F46085033F2B5FFA83F82AD0242000FB034349
S3150800F47013F5147024D00DF10E011EF009FFF8B92A
S3150800F48041462046FFF73EF920682946B8303A46F5
S3150800F4901BF033FDA0B9204615F004FE11F0EEFB73
S3150800F4A002280DD90320F7F7DBF904463046F7F7AB
S3150800F4B0E3F931460090054A032023461FF085F9F3
S3150800F4C007B0BDE8F08300BF6A3F03088C3F030816
S3150800F4D02DE9F8430C46002105460B4690F82C2BDF
S3150800F4E091420BDA05EBC11090F84C0B013100F094
S3150800F4F00700062804BF0133DBB2F1E70321D31A5C
S3150800F500B2FBF1F29342B8BFC0224FF00003A8BF86
S3150800F510A37063712371E370B8BFA270284615F013
S3150800F5207CFF242707FB0050EB7B90F87362C6F339
S3150800F5308306042B4FD8DFE803F00303092D4D009B
S3150800F540524840F6EB711FF03EF9FEE7296805F1CF
S3150800F5502E07384601F5126114F0DDFF022807D0A0
S3150800F560032809D001280AD163790133637106E0BB
S3150800F57023790133237102E0E3780133E3702968C4
S3150800F580384601F5126114F0C6FFFFF7DBF930447F
S3150800F590C6B220E0284615F040FF07FB0053284670
S3150800F5A093F8721218F007FC8046284615F035FFC6
S3150800F5B007FB005090F872323E2B43D8284615F0C8
S3150800F5C02CFF0146284618F0F6FB4644F6B2B04230
S3150800F5D038D300E000260027277205F26E294FF07F
S3150800F5E0240808FB075393F8733208FB07585B0691
S3150800F5F042BF237A0133237298F86C3203F007036B
S3150800F600062B0BD105F5DA5305331B789F4222D119
S3150800F61004E0012802D163790133637101373F2F72
S3150800F62009F12409DBD1102E28BF1026A67195F8FA
S3150800F6304832E371052363720023A3720123E37240
S3150800F640BDE8F883284615F0E8FE0146284618F076
S3150800F650B2FB0646BFE72968484601F5126114F071
S3150800F6605AFF98F8733203F00303984228BF1846E6
S3150800F670C0B2022803D1237901332371CEE70328C8
S3150800F680C7D1E3780133E370C8E700BFF73C030846
S3150800F6902DE9F04186B004460E461746984615F001
S3150800F6A0A2FF0546002800F09D80204629460A222A
S3150800F6B015F0AEFF002840F092802046294615F046
S3150800F6C0CDFF002840F08B802046294616F080F8AA
S3150800F6D0002840F084802046294616F039F800288C
S3150800F6E07DD12046294616F049F8002877D12046CC
S3150800F6F02946BA1C7B7816F014F800286FD13046D4
S3150800F70018F0D2F92046294606F16802082315F0B2
S3150800F710F2FF002863D194F835305BB104F1380064
S3150800F720314608221EF0B4FD20B92046294694F831
S3150800F730372009E0216806F11E0001F5126114F070
S3150800F7409CFE29460246204616F0A2F8002846D115
S3150800F7502046294619F0A2F9002840D12946204614
S3150800F76016F0A7F80146002839D102A810221EF083
S3150800F770D1FD48F2FE0302A83146ADF8083013F071
S3150800F780D1FEB8F1000F04D01FF035F84FF4FA7324
S3150800F79003E01FF030F84FF47A73B0FBF3F202FB84
S3150800F7A01300431C9BB22046294602AA16F0C6FA45
S3150800F7B0A8B9204615F076FC11F060FA022811D98E
S3150800F7C00320F7F74DF804460220F7F755F802210B
S3150800F7D00090064A032023461EF0F7FF02E028465B
S3150800F7E011F062FE002006B0BDE8F081B33F0308C1
S3150800F7F02DE9F0438BB00D469146D2F82880044691
S3150800F80015F050FC11F03AFA02280DD90320F7F743
S3150800F81027F806460220F7F72FF802210090684AD3
S3150800F820032033461EF0D1FF204618F099F941F619
S3150800F8303C33E35C984201D30226BCE0E37B042B0D
S3150800F8402FD0204615F0E9FD0146204618F0B3FAF8
S3150800F8500F2826D9E37B022B17D0204615F0DDFDAD
S3150800F860242707FB004090F87362204615F0D5FD63
S3150800F87007FB0047204697F8721218F09CFAC6F361
S3150800F880830630440F28D7DC0BE0204615F0C5FD6B
S3150800F890242303FB004090F87332C3F383030F2B32
S3150800F8A0DBD005AF384609F1100112F028FD2846CD
S3150800F8B01221042204AB1BF0C8FC064600287AD1A4
S3150800F8C09DF81130022B01D0062674E0BDF81220EF
S3150800F8D0C2F3072343EA02239BB2022BF4D128463C
S3150800F8E00E21032203AB1BF0B0FC0646002862D1AA
S3150800F8F09DF80D30012BE7D1E37B042B0DD8DFE80B
S3150800F90003F05A5A030808009DF80E305A0604D424
S3150800F91051E09DF90E30002B4DDA284603210A22C4
S3150800F92007AB1BF092FC002844D107A818F09DF8F5
S3150800F9300028C9D02046394618F01EFA054630B1C7
S3150800F940037FDB062BD42046294618F095FE204671
S3150800F95018F0E4F9054670B38022002105F11E0669
S3150800F9601EF0D8FC97E8030085E80300304614F03B
S3150800F97048FD2168304601F5126198F9032014F014
S3150800F98099FD2B7F0221002261F3020362F3C7135C
S3150800F9902B776A771EF00DFF0523A8606B669DF826
S3150800F9A00E30204683F04003294607AAC3F3801386
S3150800F9B0FFF76EFE064630460BB0BDE8F08300BF83
S3150800F9C0D43F03082DE9F74FDDF8349005460E4677
S3150800F9D0924698469DF830B015F005FE0446002874
S3150800F9E000F0AD80284621460E2215F011FE0028AB
S3150800F9F040F0A2804746C8EB07035B457FDA17F855
S3150800FA00013B132BF7D801A252F823F0CFFA0008CE
S3150800FA107FFA0008D9FA0008F7F90008BDFA0008C5
S3150800FA20EFFA0008F7F90008F7F90008E5FA000800
S3150800FA30F7F90008F7F9000875FA00088FFA0008C0
S3150800FA40F7F90008F7F90008F7F90008F7F90008C8
S3150800FA505DFA0008F7F9000869FA00082846214601
S3150800FA60012215F013FE46E028462146324619F0D3
S3150800FA7027F840E02846214615F0AAFE3BE0327FEB
S3150800FA8028462146C2F3C30215F011FE33E0327F41
S3150800FA902846C2F3C00282F00102214615F0BCFED8
S3150800FAA00246002848D12846214615F084FF00283A
S3150800FAB042D12846214615F0ACFF1CE028462146CF
S3150800FAC009F1020299F8013015F02BFE13E02846D9
S3150800FAD0214615F0C3FD0EE028462146726E15F044
S3150800FAE0F6FD08E02846214615F048FE03E02846BC
S3150800FAF0214615F02DFE00283FF47DAF1CE0284670
S3150800FB0021460AF1100216F00FF8A8B9284615F092
S3150800FB10C9FA11F0B3F8022811D90320F6F7A0FEA6
S3150800FB2004460220F6F7A8FE02210090064A0320A2
S3150800FB3023461EF04AFE02E0204611F0B5FC0020DE
S3150800FB4003B0BDE8F08F00BFF53F03082DE9F04785
S3150800FB50A2B00F469146064615F0A4FA11F08EF8A3
S3150800FB6002280DD90320F6F77BFE04460220F6F795
S3150800FB7083FE02210090614A032023461EF025FEDB
S3150800FB8038460121032202AB1BF05FFB80460028A2
S3150800FB9040F0B0809DF80940012C02D04FF00608CD
S3150800FBA0A8E005A809F1100112F0A9FB304605A93D
S3150800FBB018F0E2F88DF8348005469DF80A2010B151
S3150800FBC0037F59070BD1130740F1948011238DF851
S3150800FBD035300021022300930191304657E062F345
S3150800FBE0C60303770DF11C0A0B238DF83630384609
S3150800FBF003210A2253468DF835401BF026FB0028C0
S3150800FC0076D1504617F031FF0028C7D004238DF867
S3150800FC10373008238DF8383005238DF83930062417
S3150800FC2038461321462210AB1BF00FFB002833D0B1
S3150800FC3038460B210A220AAB1BF007FB00283DD1E8
S3150800FC409DF82930082BA9D12B7F1A074BBF42F6FE
S3150800FC50652242F664229DF82F309DF830304BBF5E
S3150800FC6085F87D3085F87D30316831688A5C9A423E
S3150800FC7024D138460221062203AB1BF0E6FA28B344
S3150800FC801EF097FD2946A86030468DE810044A46BE
S3150800FC900DABFFF797FE2DE09DF84130442B3FF65C
S3150800FCA07DAF2A46304610A918F034FA22AA631CFA
S3150800FCB01444132204F8542CDCB2B9E722AA631CB4
S3150800FCC014440C2204F8542CDCB2D2E79DF80D300B
S3150800FCD0042B7FF463AFDDF80E0011F0C3FF22AAF0
S3150800FCE0631C1444022204F8542C6866DCB2C7E785
S3150800FCF0032495E7404622B0BDE8F0872240030872
S3150800FD0070B586B0064615F06EFC0546002852D03A
S3150800FD1030462946042215F07BFC044600284CD1BF
S3150800FD203046294615F09AFC0446002845D1304647
S3150800FD30294615F04DFD044600283ED1F37B042BD9
S3150800FD4010D8DFE803F003030F0909001E4840F244
S3150800FD5003211EF038FDFEE73046294618F0B2FFAB
S3150800FD60044650BB0021102202A81EF0D3FA40F226
S3150800FD70FF233046ADF8083029464FF4807302AAAF
S3150800FD80ADF8163015F0D0FE0446B0B9304615F079
S3150800FD9089F910F073FF02280DD90320F6F760FDE4
S3150800FDA004460220F6F768FD02210090074A032060
S3150800FDB023461EF00AFD002402E0284611F074FBD3
S3150800FDC0204606B070BD00BFF73C03085440030840
S3150800FDD041F630322DE9F047835C04460BB1013B0E
S3150800FDE0835494F8755035B1013DEDB284F87550D9
S3150800FDF0B5FA85F56D09E37B042B56D8DFE803F0E1
S3150800FE0003090E304700724840F2AE611EF0DBFC73
S3150800FE10FEE72046BDE8F04716F073B805B320465E
S3150800FE2018F09AF841F63D33E35C834205D920463B
S3150800FE30BDE8F0470221FFF76DB804F5DE752846E0
S3150800FE401BF05DFA002840F0C1802046FFF758FFF6
S3150800FE502846BDE8F0475F495F4A012301F016BF0F
S3150800FE60204617F07DFE41F63C33E35C984203D307
S3150800FE702046012115F0E9FFBDB1204618F06CF8BF
S3150800FE8041F63E33E35C8342C0F096800DE020469F
S3150800FE9017F066FE092808D994F84832013384F821
S3150800FEA048321EF086FCC4F84C0204F53366002777
S3150800FEB094F82C3B9F422CDA04EBC71393F84C2B8F
S3150800FEC002F00702072A16D00123934013F0090F00
S3150800FED01CD113F0660F08D113F010050CD03C485E
S3150800FEE040F2FC611EF06FFC04E0756E4FF47A7305
S3150800FEF05D4301E0FEE700251EF05BFCB368C01A0F
S3150800FF00A84203D32046314618F0B6FB013780369F
S3150800FF10CEE704F514750027242303FB074393F85B
S3150800FF206C325FFA87F803F00703062B0AD11EF036
S3150800FF3040FCAB68C01A294B984203D9204629468B
S3150800FF4018F09AFBE37B042B29D1242606FB0746E7
S3150800FF5006F51C76F378C3F38019B9F1000F11D0B2
S3150800FF6095F822303E2B1AD92046414617F023FF32
S3150800FF700F2814D91EF01DFCAB68C01A184B9842FE
S3150800FF801FD80CE0DB090AD01EF013FCAB68C01AB8
S3150800FF90144B984282BFF37869F3C713F37001379D
S3150800FFA03F2F05F12405B7D104F5FC704FF47A719B
S3150800FFB011F05AFEBDE8F0872046012115F045FFED
S3150800FFC073E720464146FEF79DFBE8E7BDE8F08764
S3150800FFD0F73C030890B20800F09C09009F860100D0
S3150800FFE08F5F01002FE602002DE9F74FDDF830A0FC
S3150800FFF0054688469946D1F828B017463AB1137F80
S3150801000003F00703062B0CBF0124022400E0012498
S31508010010284615F0E8FA0646002800F0F780224639
S315080100202846314615F0F4FA0446002840F0DF80E8
S315080100302846314615F03DFC0446002840F0D78095
S315080100402846314615F00AFB0446002840F0CF80C1
S31508010050284631460AF102029AF8013015F061FB89
S315080100600446002840F0C3802846314615F070FB47
S315080100700446002840F0BB802846314615F07EFB31
S315080100800446002840F0B38028689BF9031000F560
S31508010090126014F0E4F995F8353004464BB147B1CE
S315080100A0384605F1380108221EF0F2F8002800F05A
S315080100B0A28022462846314615F0EAFB0446002866
S315080100C040F0958017B94FF0000A0EE0BB8AC3F3DA
S315080100D00803002B00F09280F5E74B449B780A2B26
S315080100E011D0102B08D10AF1010A99F801205FFAFB
S315080100F08AF39A42F1D811E0092B77D1284631467D
S3150801010018F0E0FD06E0002F70D028463146BA8A7D
S3150801011015F04AFB04460028E5D068E0FFB13B7FAD
S3150801012003F00703062B1AD0384617F0B1FC284608
S31508010130314607F10C02082315F0DDFA04460028BA
S3150801014055D128463146344A012315F07AFB04462F
S3150801015000284CD13B7F042262F302033B774046D9
S3150801016013F051F908F1100818B31EF044FB4FF4C7
S315080101707A73B0FBF3F202FB1300431C314628469F
S3150801018042469BB215F0DAFD044680BB284614F0B8
S3150801019089FF10F073FD022838D90320F6F760FBB2
S315080101A004460220F6F768FB022100901B4A032049
S315080101B018E028463146424615F0B6FC0446B0B961
S315080101C0284614F06FFF10F059FD02281ED90320A6
S315080101D0F6F746FB04460220F6F74EFB104A009056
S315080101E00221032023461EF0F0FA0FE002243046CE
S315080101F011F05AF90BE095F837405AE72846314687
S3150801020015F0E6FA04460028F1D15CE700242046F9
S3150801021003B0BDE8F08F00BFE93C0308704003084E
S315080102208D4003082DE9F04F91B00F4690460546DB
S3150801023014F038FF10F022FD02280DD90320F6F735
S315080102400FFB04460220F6F717FB02210090694AC4
S31508010250032023461EF0B9FAEB7B033B012B01D998
S315080102600020C4E095F84030002BF9D105AE3046A0
S3150801027008F110010DF11C0912F041F83846032165
S315080102800A224B461AF0E1FF002840F0B0804846A2
S3150801029017F0EBFB08B90620A9E03846122104221B
S315080102A003AB1AF0D2FF002840F0A1809DF80D306B
S315080102B0022BF0D1BDF80E20C2F3072343EA02232D
S315080102C09BB2022BE7D138460B210A220AAB1AF058
S315080102D0BCFF60B99DF82930082BDCD10AA814F0B7
S315080102E0DBFE0446281D14F0D7FE8442B8D13846F1
S315080102F00021042204AB1AF0A8FF002847D19DF873
S315080103001130022BC7D1BDF812403146C4F3072379
S31508010310284643EA042418F015F8A4B2014610B198
S31508010320838AA3425FD1C4F3080ABAF1000F3ED10A
S31508010330A4123F2CAFD0242303FB045404F51474F0
S31508010340237F03F00703062B1AD096E8030004F16E
S315080103501E06D8F828B084E80300304614F051F890
S3150801036029689BF90320304601F5126114F0A2F8B9
S31508010370237F042262F3020384F81DA0237717E082
S315080103802046314608221DF083FF88B168E72846D2
S31508010390314617F0D7FF044618B3037F03F0070366
S315080103A0062B1ED1838AC3F30803D3B900E00024C0
S315080103B038460D210A220DAB1AF047FF28B99DF8D8
S315080103C03530082B3FF667AF02E000238DF835304C
S315080103D0CDF800902846414622460DABFFF704FEAC
S315080103E005E0022003E0284618F046F99BE711B01C
S315080103F0BDE8F08FA74003082DE9F04F8846A9B05C
S3150801040002F1100B05930DF13C09936A594605460D
S3150801041048469246039311F072FF40461221042280
S3150801042008AB1AF012FF0446002840F0CB819DF86C
S315080104302130022B01D00624C4E1404604210A22B8
S3150801044011AB1AF002FF0446002840F0BB819DF863
S315080104504530082BEFD121464046042209AB1AF054
S31508010460F4FE0446002840F0AD819DF82530022BA4
S31508010470E1D14946284617F065FF014650B1BDF856
S315080104802620C2F3072343EA0223828A9BB29A42B1
S3150801049040F05D814046052106220BAB1AF0D5FED8
S315080104A00446002840F08E819DF82D30042BC2D1D8
S315080104B04046082106220DAB1AF0C7FE20B99DF861
S315080104C03530042BB7D107E0DDF82E0011F0CAFB51
S315080104D011F0C8FBCDF83600BDF82670C7F307231F
S315080104E043EA0727BFB2C7F30803002BA3D1BF12FC
S315080104F0FBB23F2F04939ED0242606FB075616F51A
S31508010500147698D0337F03F00703042B05D0062B06
S3150801051016D0002B40F0088112E006F10C000DF10F
S31508010520460108221DF0B4FE002840F01481EB7B39
S31508010530042B00F29A80DFE803F00D133E5A5A00A5
S3150801054041F63033EB5C002B00F0058105F5D950F7
S315080105501130E4E79D4840F291311EF034F9FEE787
S3150801056040460A2104220AAB1AF06FFE002840F021
S31508010570EC809DF82970022F7FF45DAF284614F0B0
S3150801058073FEBDF82A20C2F3072343EA02239BB26E
S31508010590984240F0D880404609212B221DAB1AF01B
S315080105A054FE002840F0D1809DF87530093B202B78
S315080105B040F2BC803FE740461021032207AB1AF000
S315080105C044FE002840F0C1809DF81D30012B7FF4C0
S315080105D032AF9DF81E0013F037FF242303FB07579C
S315080105E097F8733260F3010387F873323DE04046AA
S315080105F00B210A2214AB1AF028FE002840F0A58028
S315080106009DF85130082B7FF416AF14A814F044FD59
S315080106108346281D14F040FD834540F0D3804046AB
S315080106201021032207AB1AF010FE002840F08D8036
S315080106309DF81D30012B7FF4FEAE9DF81E0013F0C8
S3150801064003FF242303FB075797F87332049A60F3D1
S31508010650010387F8733241F64533EB5C934204D0C4
S3150801066096F822303E2B00F2A98099E8030086E825
S315080106700300BDF82620DDF82E00C2F3072343EA5E
S315080106800223B38211F0EEFAF060DDF8360011F0BC
S31508010690E9FA30611EF08DF8337F0B2262F3C60347
S315080106A006F11E07B0603377384613F0AAFE039B9E
S315080106B0296893F90320384601F5126113F0FAFE09
S315080106C000237377337F062262F302033377059B90
S315080106D0B3619DF8C830002B74D017AF404603218B
S315080106E00A223B461AF0B1FD044600286AD138466B
S315080106F017F0BBF900283FF49EAE40460D210A22A9
S315080107001AAB1AF0A2FD28B99DF86930082B3FF6F5
S3150801071092AE01E08DF86940009728465146324667
S315080107201AABFFF761FC10E00E244BE028461DA921
S3150801073017F07AFB48B940460B210A2214AB1AF086
S3150801074084FD074648B13C463CE004463AE0284663
S3150801075017F092FF9EE6FF2434E09DF85130082BEE
S315080107607FF469AE14A814F097FC9DF8562001464B
S315080107709DF85930284614F052FE6B7B284604939F
S3150801078014F072FD049BC0F387208342284606D1E4
S3150801079014F06AFD01462846FDF718FF65E714F0CF
S315080107A063FD01462846FDF7A1FE0123AB730097B9
S315080107B028465946064AF9F7FBFE56E7284617F032
S315080107C01FFA52E7204629B0BDE8F08FF73C030827
S315080107D0E24103082DE9F3410E4615461C46074634
S315080107E014F060FC10F04AFA02280DD90320F6F736
S315080107F037F880460220F6F73FF802210090084AAA
S31508010800032043461DF0E1FF002300933846314695
S315080108102A462346FFF7F0FD02B0BDE8F08100BF86
S31508010820C64003082DE9F3410E4615461C46074600
S3150801083014F038FC10F022FA02280DD90320F6F735
S315080108400FF880460220F6F717F802210090084AA9
S31508010850032043461DF0B9FF01230093384631466C
S315080108602A462346FFF7C8FD02B0BDE8F08100BF5E
S31508010870E44003082DE9F74F06460F4692469B4684
S31508010880BDF8309014F0AFFE0546002873D0304607
S315080108902946082214F0BCFE044600286DD13046CC
S315080108A0294614F0DBFE0446002866D1304629465F
S315080108B014F08EFF044600285FD1224630462946A9
S315080108C015F079F80446002857D13046294615F01F
S315080108D0A0F80446002850D1D046CAEB08035B4568
S315080108E025DA18F8013B182B14D0192B17D00C2B25
S315080108F0F3D13046394617F07AFD28B1007F80F0EA
S315080109000800C0F3C00200E002463046294614F04A
S3150801091083FF08E03046294618F0FBF903E0304624
S31508010920294618F0FFF904460028D6D025E03046B6
S3150801093029463A46B9F1000F1AD04B4615F0FEF989
S315080109400446D0B9304614F0ADFB10F097F90228E9
S3150801095011D90320F5F784FF04460220F5F78CFF29
S3150801096002210090084A032023461DF02EFF02E0CB
S3150801097015F0DAF8E4E7002402E0284610F094FDC1
S31508010980204603B0BDE8F08F0E410308F0B58DB0DF
S315080109900C461746054614F085FB10F06FF9022838
S315080109A00DD90320F5F75CFF06460220F5F764FF2B
S315080109B0022100903F4A032033461DF006FF2046D8
S315080109C00D210A2203AB1AF040FC064600286ED117
S315080109D09DF80D30042B01D9062668E08DF819001B
S315080109E0162120460A2206AB1AF02FFC18B99DF8E3
S315080109F01930082BF0D100238DF825302046172110
S31508010A000A2209AB1AF021FC18B99DF82530082BE2
S31508010A10E2D1FF21042202A81DF07CFC02A80DF1F7
S31508010A200E019DF80D200CF021FB9DF819309DF85B
S31508010A300D4063B3286800F57F701AF0DFFD30B307
S31508010A40286800F57F701AF0D9FD0DF11A011BF01F
S31508010A5036F9E0B99DF825300BB3286800F5CA6068
S31508010A601AF0CCFDD8B1286800F5CA601AF0C6FD9F
S31508010A700DF126011BF023F988B9002300932846B6
S31508010A8007F1100102AA2346FFF7F4FE0FE00CABAB
S31508010A90621C1C44182304F8283CD4B2DAE70CABD0
S31508010AA0621C1C44192304F8283CD4B2E5E73046F5
S31508010AB00DB0F0BD2A410308F0B5C37B87B0033BEF
S31508010AC0012B054661D802A8002110221DF022FC3F
S31508010AD040F2FF23ADF808304FF48073ADF81630B5
S31508010AE0EB7B042B09D01DF086FE4FF4FA73B0FB9D
S31508010AF0F3F202FB130080B200E00020009002A985
S31508010B002846234A0123FFF7B5FE002695F82C3B14
S31508010B10F4B2A34239D9E4012F1907F648373B79CC
S31508010B2003F00702062A2AD1C3F3C30303F0080315
S31508010B3003F0FF011BBB102202A81DF0EBFB48F2D4
S31508010B40FE0304F533642C4402A82146ADF80830A7
S31508010B5012F0E8FC3B7994F87D2013F0080F2B6816
S31508010B600FD003F5295325331B789A4207D0002362
S31508010B700093284602A9064A0123FFF77BFE0136A0
S31508010B80C4E703F529532433EEE7002007B0F0BD87
S31508010B90E14103082DE9F043A5B00D4614469846F0
S31508010BA0976A064614F07EFA10F068F802280DD9FD
S31508010BB00320F5F755FE81460220F5F75DFE022171
S31508010BC00090554A03204B461DF0FFFD04F1100124
S31508010BD00AA811F094FB30460AA917F0CDF8044685
S31508010BE0002800F0938028460021042203AB1AF05E
S31508010BF02CFB78B99DF80D30022B01D0062088E030
S31508010C00BDF80E20C2F3072343EA0223A28A9BB248
S31508010C109A42F3D1284604210A220CAB1AF015FB95
S31508010C2038B128460521062206AB1AF00EFB68B133
S31508010C3015E09DF83120082A6AD10DF1320004F138
S31508010C4068011DF025FB002862D1EAE79DF81930F5
S31508010C50042BD3D1DDF81A0011F004F8E060284618
S31508010C600821062208AB1AF0F0FA40B99DF821309E
S31508010C70042BC3D1DDF8220010F0F4FF20612846C9
S31508010C800221062204AB1AF0E0FA40B99DF81130A8
S31508010C90042BB3D1DDF8120010F0E4FF6066284694
S31508010CA01321462212AB1AF0D0FA40B99DF8493001
S31508010CB0442BA3D8304612A9224617F02BFA284608
S31508010CC00B210A220FAB1AF0C0FA60B99DF83D3024
S31508010CD0082B93D1237F1B074CBF9DF843309DF802
S31508010CE0443084F87D302146304618F078F81DF0F6
S31508010CF060FD3168A060C4F8188004F11E0001F592
S31508010D00126197F9032013F0D5FB01E0192000E0E1
S31508010D10002025B0BDE8F083494103082DE9F041DB
S31508010D2086B004460E4614F05EFC0546002800F01F
S31508010D30BC80204629460C2214F06AFC002840F0A3
S31508010D40B1802046294614F089FC002840F0AA8083
S31508010D502046294614F03CFD0246002840F0A280B0
S31508010D602046294614F027FE002840F09B8020469D
S31508010D70294614F04EFE002840F09480337F03F094
S31508010D800703062B16D004F5D9531A331A882046B9
S31508010D90013292B2B2F5007F28BF01221A801F885C
S31508010DA0394616F0CFFF0028EDD12368B3F8C018ED
S31508010DB03943B18220462946B28A14F0F5FC002847
S31508010DC070D106F1670706F16C0817F8013F0C2B7D
S31508010DD010D006D8092B1DD12046294617F072FFD7
S31508010DE016E0182B10D0192B14D12046294617F0D6
S31508010DF099FF0DE0327F2046C2F3C002294682F0F0
S31508010E00010214F009FD03E02046294617F081FF87
S31508010E10002847D14745D8D1337FDB0612D520466E
S31508010E20314617F0DCFF337FC3F3C30303F008032E
S31508010E3003F0FF026BB92068314600F6F44016F05C
S31508010E405BF906E020462946324617F039FE48BBCB
S31508010E50E5E71022002102A81DF05CFA48F2FE031C
S31508010E6002A83146ADF8083012F05CFB2046294647
S31508010E7002AA14F059FEA8B9204614F013F90FF086
S31508010E80FDFE022811D90320F5F7EAFC04460220E3
S31508010E90F5F7F2FC02210090064A032023461DF0CD
S31508010EA094FC02E0284610F0FFFA002006B0BDE8DF
S31508010EB0F08100BF7C4103082DE9F04FABB00F4626
S31508010EC014469A46D2F82890054614F0EBF80FF026
S31508010ED0D5FE02280DD90320F5F7C2FC06460220E5
S31508010EE0F5F7CAFC02210090BF4A032033461DF0DC
S31508010EF06CFCEB7B012B26D904F110010AA811F031
S31508010F00FEF928460AA916F037FF0446E8B138461D
S31508010F1004210A220CAB1AF098F90646002840F07B
S31508010F205F819DF831B0BBF1080F40F0598104F19A
S31508010F3068080DF1320041465A461DF0A9F9002804
S31508010F4040F04E8103E00E264AE1064648E138465E
S31508010F500521062204AB1AF078F90646002840F066
S31508010F603F819DF81130042B01D0062638E1384619
S31508010F705946062206AB1AF068F920B99DF81930C8
S31508010F80042BF2D107E0DDF8120010F06BFE10F029
S31508010F9069FECDF81A0038460121032203AB1AF07F
S31508010FA054F90646002840F01B819DF80D30012BA7
S31508010FB0DBD138460221062208AB1AF046F9064665
S31508010FC0002840F00D819DF82130042BCDD19DF8E4
S31508010FD00E308DF86100980708D538460D210A228A
S31508010FE00FAB1AF032F9064678B1F9E03846132103
S31508010FF0462218AB1AF029F90646002840F0F08077
S315080110009DF86130442BB0D8E7E79DF83D30052BB4
S31508011010ABD88DF84900162138460A2212AB1AF0C8
S3150801102014F918B99DF84930082B9ED100238DF87B
S315080110305530384617210A2215AB1AF006F918B9A0
S315080110409DF85530082B90D105F5147B00272423EC
S3150801105003FB075393F86C32590700F0AE805846E4
S315080110600AA908221DF014F9002840F0A68028468E
S31508011070594617F001FB237F03F00702062A04D01D
S31508011080032262F3020323770CE02846A18A17F0AC
S31508011090C9FA237F5A0605D42868214600F6144062
S315080110A013F015FB1DF085FBA060DDF8120010F0AA
S315080110B0D9FDE060DDF81A0010F0D4FD237F9DF814
S315080110C00E20206162F3C60323772968C4F818A0A5
S315080110D001F5126199F9032004F11E0013F0EAF9EA
S315080110E0DDF8220010F0BEFD9DF80E306066DB07C4
S315080110F04CBFEB7A2B7B18A984F87D30224628460B
S3150801110017F008F805224046FF211DF003F99DF85E
S315080111103D7004F167020023D9B2B94206D20FA97C
S3150801112019448978013302F8011FF5E79DF849301A
S31508011130002B49D0286800F57F701AF05FFA00285D
S3150801114042D0286800F57F701AF058FA0DF14A0165
S315080111501AF0B5FD002837D19DF85530002B3AD045
S31508011160286800F5CA601AF049FAA0B3286800F59C
S31508011170CA601AF043FA0DF156011AF0A0FD50BBE8
S31508011180EB7B042B2CD8DFE803F0030309121200CA
S31508011190164840F643011DF016FBFEE7237F03219F
S315080111A061F3020323772846FDF7B4FE18E02846C3
S315080111B02146FFF7B3FD064612E001373F2F0BF133
S315080111C0240B7FF444AF56E77B1C1822274487F883
S315080111D06820DFB2C0E72744192387F86830CFE7CC
S315080111E030462BB0BDE8F08F9C410308F73C030855
S315080111F0F0B589B09DF8383004461546002B40F005
S315080112001B81002900F01881002A00F015814B780E
S31508011210442B40F0118113F045FF0FF02FFD0228F2
S315080112200DD90320F5F71CFB06460220F5F724FB2A
S3150801123002210090814A032033461DF0C6FA28464A
S315080112400421032203AB1AF000F8002840F0F480C9
S315080112509DF80D30012B40F0EF809DF80E30A3B1BB
S3150801126041F64633E35C3E2B00F2E680204617F052
S31508011270CDFD10B1204617F0E0FD41F645323F237A
S31508011280A35441F64632A354D6E028460221042245
S3150801129004AB19F0DAFF002840F0CE809DF8113032
S315080112A0022B40F0C980BDF81230C3F385073F2FE2
S315080112B0FEB200F0C180242303FB074313F5147F14
S315080112C000F0BA80284607210B2205AB19F0BDFFAD
S315080112D0002840F0B1809DF81530092B40F0AC800C
S315080112E041F64633E35C3E2B08D89E4206D020469B
S315080112F017F08CFD10B1204617F09FFD41F64533D6
S31508011300E65441F646332046E654B902FDF7EEF8AF
S315080113100546002840F09080242303FB074393F8F1
S31508011320732260F3850283F873229DF8163084F8D8
S3150801133048321DF03EFAC4F84C02242303FB054348
S31508011340E9B208AA02EBD10293F8730212F8096C02
S3150801135001F0070780223A411642064614BF0122C8
S31508011360002262F3861683F87362430601D5002AC2
S315080113705CD001353F2DE0D1204614F04EF82425E6
S3150801138005FB004090F8733213F03C0F0CD1204650
S3150801139014F043F805FB004094F87C2090F873326A
S315080113A062F3850380F87332204614F036F8242751
S315080113B007FB0040A38C04F110069B1280F87232D9
S315080113C0A38C9B1207FB03470FCE07F514750FC5B0
S315080113D00FCE0FC5336820462B6097F8733200216C
S315080113E043F0400387F87332FDF7FCF904F53366D9
S315080113F0002594F82C3B9D421EDA04EBC51393F89D
S315080114004C3B03F00703032B07D0042B0BD10C48E5
S3150801141040F6E9611DF0D7F904E020463146FFF7A9
S315080114207DFC00E0FEE701358036E2E7206800F53D
S31508011430BE7016F00EFA9CE709B0F0BDBF4103086D
S31508011440F73C030810B5044615F062FA04F58870EE
S3150801145000213C221CF05EFF0023A4F80E31024B4A
S31508011460C4F84C3110BD00BF00A3020038B50446CC
S315080114700D4615F062FA04F5A8726B68C4F8642182
S31508011480184A03F50343C4F86821174A0433C4F814
S315080114906C21164AC4F85031C4F87821144A154B00
S315080114A0C4F87C21144AC4F85431C4F88821134A73
S315080114B000232046C4F85841C4F85C31C4F86031A9
S315080114C0C4F87041C4F87431C4F88041C4F8843151
S315080114D0C4F88C21C4F89041C4F89431FFF7B2FFDF
S315080114E0204638BD863603082B9E0208E3410308C9
S315080114F0C1950208359F0208E8410308C796020804
S315080115002DE9F04F0646D0F80001A7B00C46B830D1
S315080115100021174699469DF8C08019F0B4FC054686
S31508011520002877D0214602A819F053FC02A819F021
S3150801153043FC284602A99DF88820F5F7FDFA0028FC
S3150801154065D1314696F8FF30334499425FD20A781D
S315080115505210042A04D18C1C91F801B004D156E02A
S315080115604A7802321144F0E7BBF1000F4FD0B8F1C7
S31508011570000F02D04FF0000A27E0284621465A46B6
S31508011580F5F7DAFA002842D1EB8B9DF888109942D3
S315080115901FD10139284689B20FF08AFF19E04B7825
S315080115A00233194404EB0B0399420CD25FFA8AF30E
S315080115B00A7819F803309A42F1D14A782846023254
S315080115C0F5F7BAFA18BB0AF1010AC245DCD0214679
S315080115D0E8E7D6F800012946B8303A4619F07FFC03
S315080115E0A8B9304614F0D8FE0FF048FB022811D9E5
S315080115F00320F5F735F904460A20F5F73DF90A21DE
S315080116000090064A032023461DF0DFF802E028462B
S315080116100FF04AFF27B0BDE8F08F00BFED41030880
S315080116202DE9F0410546D0F80001A8B08846B83042
S31508011630002116461F4619F026FC044600283CD010
S31508011640414604A819F0C5FB04A819F0B5FB2046C4
S3150801165004A99DF89020F5F76FFA58BB10238DF869
S315080116600C302046012303A903228DF80D308DF88D
S315080116700E70F5F761FAE8B9D5F800012146B830D8
S31508011680324619F02CFCA8B9284614F085FE0FF04D
S31508011690F5FA022811D90320F5F7E2F804460A20DB
S315080116A0F5F7EAF80A210090054A032023461DF0BA
S315080116B08CF802E020460FF0F7FE28B0BDE8F0816D
S315080116C01E42030837B5B0F80E21012342FA03F189
S315080116D0C9071BD41C460123A3401A43A0F80E21AF
S315080116E014F05AFE0FF0CAFA022814D90320F5F7A6
S315080116F0B7F805460420F5F7BFF804218DE811006F
S31508011700064A03202B461DF060F804E00133102B2E
S31508011710DCD14FF0FF34204603B030BD4F420308F9
S315080117202DE9F041C4B00E4617461D46044614F08D
S3150801173033FE0FF0A3FA02280DD90320F5F790F826
S3150801174080460420F5F798F804210090274A0320DB
S3150801175043461DF03AF838460221042202AB19F035
S3150801176074FD68B99DF80930022B3BD1BDF80A1002
S315080117702046C1F3072343EA012189B218F0BBFACF
S3150801178038460A2140F2011203AB19F05EFD60B931
S31508011790E98B2046C1F3072343EA012189B20DF1FA
S315080117A00E029DF80D3018F0D5FAD4F8000131462D
S315080117B0B8302A4619F0A1FBA0B9204614F0ECFD71
S315080117C00FF05CFA02280DD90320F5F749F804460B
S315080117D00420F5F751F804210090054A0320234611
S315080117E01CF0F3FF44B0BDE8F08100BF7242030864
S315080117F09E42030873B50D46044614F0CDFD0FF05D
S315080118003DFA02280ED90320F5F72AF806460420E0
S31508011810F5F732F804218DE82100124A03203346F0
S315080118201CF0D3FF2946204618F030FBB4F80E21E8
S315080118300123AB4022EA0303A4F80E3194F80D31D3
S31508011840D4F80001013384F80D3194F80C314FF4C2
S315080118508071013384F80C3112F00AFA002002B0C3
S3150801186070BD00BFD542030870B505460E46CC7853
S31508011870073401EBE40404347378023333449C429D
S3150801188017D223785B0806D0022B09D128462146B0
S3150801189018F022FC09E02846214618F00FFC04E05E
S315080118A00548B6211CF08FFFFEE7637802331C4416
S315080118B0E2E7002070BD00BFF342030838B50546CC
S315080118C0044695F8FF302B449C4210D223785B08D6
S315080118D0012B07D121462846FFF7C6FF6378023355
S315080118E01C44EEE704489D211CF06DFFFEE72846DF
S315080118F015F00AF8002038BDF342030838B5024648
S315080119000D460649044612F08AFA28B920462946A0
S31508011910BDE8384012F0C9BA38BD00BF3BA302087A
S31508011920F8B5044617461E460D464968143112F0A5
S3150801193062FAA763E66304F140000FF05FFE6B6885
S31508011940246503F503430433A364074BE3640023C7
S315080119506365A36504F14803E3651CF04CFFA4F82D
S3150801196044002046F8BD00BF1FA702082DE9F84329
S3150801197040300E4690461D46089F0FF042FE04462B
S3150801198000284DD02146384607F1100918F063FDA5
S31508011990484608F1100111F015FE28B13A8CB8F83D
S315080119A022309A4212D115E0484611F02CFD002842
S315080119B0F4D1484611F09CFD0028EFD106E03378B2
S315080119C003F03003102B25D011D81BB320460FF096
S315080119D060FED4E728462146342219F008F8002883
S315080119E0EDD0114840F239111CF0EDFEFEE7202B2F
S315080119F001D0302BEAD172886988C2F3072343EAFA
S31508011A000222C1F3072343EA012392B29BB29A4207
S31508011A10DCD105E03046294618F0DAFC0028D5D095
S31508011A202046BDE8F88300BF6F4303080829F7B5C8
S31508011A3005460C4605D913484FF4DA711CF0C3FE66
S31508011A40FEE700234E1E009301930DF1FF376E4406
S31508011A50B74204D01CF0CFFE07F8010FF8E7284675
S31508011A602B78224623F00F03234300F8043B6946EB
S31508011A700BF0FCFA95F880301C4485F8804003B0D9
S31508011A80F0BD00BFE2430308F8B504461D460E46FD
S31508011A9017464968143112F0AEF9069BA56304F19D
S31508011AA04805E36328460FF0A9FD736804F14C0263
S31508011AB003F503430433E364054B65652365002396
S31508011AC0A365E3652266A4F8407063642046F8BD01
S31508011AD0A1B002082DE9F0430546BDB000248846A9
S31508011AE0174621462C220DA899460C941CF012FC87
S31508011AF001A821462C221CF00DFC28460FF081FD79
S31508011B000646002844D031460CA801AC0DAD19F0A3
S31508011B107EF90FCD0FC40FCD0FC495E8070084E8F1
S31508011B2007007B8CBDF826209A422DD105A807F11E
S31508011B30100111F04FFD38BB18A83146302218F0B4
S31508011B4056FF08BBBDF86220B8F80210C2F3072396
S31508011B5043EA0222C1F3072343EA012392B29BB265
S31508011B609A4211D13046F18B0FF0E5FEC9F8000013
S31508011B7080B1C18B303989B20FF09AFC58B1074848
S31508011B8097211CF020FEFEE730460FF082FDB7E7ED
S31508011B90192000E003203DB0BDE8F0835544030851
S31508011BA02DE9F0419046B2B00F4606461CF001FEFB
S31508011BB0454600F57130D83003AC02900FCD0FC4FD
S31508011BC00FCD0FC495E8070084E807000EA839462B
S31508011BD0002218F00CFF002838D19DF838309B06F2
S31508011BE034D530463946424601AB19F056F918B98B
S31508011BF001980FF059FC29E0192827D13046694682
S31508011C000DF102020FF058FDBDF80030092B02D97B
S31508011C10304619F054F93846F98B0FF08CFE0190CD
S31508011C20A0B102A93022F4F787FF304601990FF0D7
S31508011C3078FDB469331D9C4208D11CF0BAFD054BE9
S31508011C40306173617068214619F0A1FA32B0BDE8B6
S31508011C50F08100BFD8C4030010B5044601600A49E3
S31508011C6041600021A060C160016160614363029B1C
S31508011C708161C16180F8201041628162012180F889
S31508011C802C100263836310BDA1B3020810B5044684
S31508011C9090F82C00012804D00E4849211CF093FD28
S31508011CA0FEE79142A161E26184F8203001D16162C7
S31508011CB00AE01CF0A0FDA269E3699B1AB0FBF3F1E7
S31508011CC001FB1300104460622046BDE8104019F07C
S31508011CD024BB00BFC844030890F82C2038B5022A53
S31508011CE04FF00103044680F82C3002D0032A25D090
S31508011CF037E0036B806B9847002837D094F820307B
S31508011D00012B0BD11CF077FDA269E3699B1AB0FB85
S31508011D10F3F101FB13001044606219E0032384F810
S31508011D202C30A56A636A5D1B1CF043FD2561E060E2
S31508011D3021462068BDE8384019F029BA426A02B13D
S31508011D405300E269934294BF63626262636B23B98B
S31508011D502046BDE8384019F0E0BAA06B984728B18B
S31508011D60F6E70348EB211CF02EFDFEE738BD00BF60
S31508011D70C8440308F8B5044608461F460D461646E4
S31508011D8015F04BFA32460146204619F00BFB284658
S31508011D9015F043FA3246014604F5847019F002FB40
S31508011DA0C4F810526A680D4B02F50342C4F818329A
S31508011DB004F505730432C4F82832069BC4F81422C4
S31508011DC00022C4F81C42C4F82022C4F82422C4F80C
S31508011DD02C72C4F830322046F8BD00BF97BB020802
S31508011DE02DE9F0410546D0F81002A8B08846B8306A
S31508011DF0002116461F4619F046F8044600283CD02D
S31508011E00414604A818F0E5FF04A818F0D5FF2046B6
S31508011E1004A99DF89020F4F78FFE58BB10238DF87E
S31508011E200C302046012303A903228DF80D308DF8C5
S31508011E300E70F4F781FEE8B9D5F810022146B830DC
S31508011E40324619F04CF8A8B9284619F0EBFC0EF001
S31508011E5015FF022811D90320F4F702FD04460A20CA
S31508011E60F4F70AFD0A210090054A032023461CF0CF
S31508011E70ACFC02E020460FF017FB28B0BDE8F08164
S31508011E808D4503082DE9F0430546D0F81002A7B0A1
S31508011E908846B8300021174699469DF8B86018F06B
S31508011EA0F2FF0446002876D0414602A818F091FFB1
S31508011EB002A818F081FF204602A99DF88820F4F7A8
S31508011EC03BFE002864D126B1013E09F1FF384E4494
S31508011ED01DE0B5F80A8205F20916B044464518D23E
S31508011EE03378052B3DD1D5F8103293F96438002B98
S31508011EF037DB737802331E44F0E718F8011F05290A
S31508011F0038D1D5F8103293F96438002B32DBB04555
S31508011F10F3D1E38B9DF88810994204D10139204603
S31508011F2089B20FF0C5FAD5F810022146B8303A46FB
S31508011F3018F0D5FF60BB284619F074FC0EF09EFE1A
S31508011F40022828D90320F4F78BFC04460A20F4F763
S31508011F5093FC0A210090114A032023461CF035FC04
S31508011F6019E07278204631460232F4F7E5FD002879
S31508011F70BFD00DE005F5847019F02BFA014600284B
S31508011F80C5D04A7820460232F4F7D6FD0028BED0DD
S31508011F9020460FF089FA27B0BDE8F083B04503085B
S31508011FA037B504460C4D0E2200950C4BFFF7E2FEA1
S31508011FB00B4BD4F81002C4F838320023C4F8345253
S31508011FC0C4F83C42C4F8403204F50D71B83018F033
S31508011FD03BFF204603B030BDD345030889390308C2
S31508011FE049BA020873B50E460446184D33220095C0
S31508011FF0174BFFF7BFFE736804F50D7203F503432C
S315080120000433C4F83432134BC4F84822D4F8100206
S31508012010114AC4F838320023C4F83C42C4F84032A5
S31508012020C4F84432C4F84C32C4F85032C4F8545295
S31508012030C4F85822C4F85C42C4F8603204F5157134
S31508012040B83018F001FF204602B070BDD845030824
S315080120508E39030817BC02084DBA02082DE9F0416A
S315080120600446B6B000212C2207A81CF053F9022217
S3150801207012A8002118F0ADFC12A80221FFF7D6FC20
S31508012080D4F82C1212A818F00DFE12A818F094FE16
S31508012090D4F82C0229491CF009F910B9204619F07F
S315080120A037FDD4F8100212A900F58E7018F05EF902
S315080120B08046C8B3611CB4F80221F4F73DFD054614
S315080120C0A0BBD4F8100203AE314600F6FC400BAFB4
S315080120D013F0E4F996E80F0087E80F004FF2BF0303
S315080120E0D4F81002ADF83E3000952B4600F58E70F7
S315080120F0414607AA18F0E0FB0546B8B9204619F08B
S3150801210091FB0EF0BBFD022813D90320F4F7A8FBB7
S3150801211004460A20F4F7B0FB0A210090084A032076
S3150801212023461CF052FB04E0032502E040460FF06B
S31508012130BBF9284636B0BDE8F08100BF8E390308E1
S31508012140DD45030873B5044619F06CFB0EF096FDE0
S3150801215002280DD90320F4F783FB05460A20F4F774
S315080121608BFB0A210090144A03202B461CF02DFBF9
S31508012170204604F5847619F0CBFC3046342119F053
S3150801218028F928B1D0F802000FF06CFD054628B1F0
S315080121900A484FF48B611CF016FBFEE7D4F81002CF
S315080121A0314600F53D7019F067FC2046294602B014
S315080121B0BDE8704019F0FDBCFD4503082246030839
S315080121C037B5CA0704460D4603D51CF0F2FAC4F81A
S315080121D04C02AB0734D51CF0ECFA04F50D75C4F8BE
S315080121E050022946D4F8340218F07FFF04F58470AA
S315080121F0342119F0EEF818B3D0F802000FF032FDC9
S31508012200014628B9204603B0BDE83040FFF79ABF1A
S3150801221028460FF029FD204619F004FB0EF02EFD85
S3150801222002280DD90320F4F71BFB04460A20F4F70C
S3150801223023FB0A210090034A032023461CF0C5FA12
S3150801224003B030BD9C4603082DE9F04F984699B076
S3150801225000238DF815308DF821308DF80D308DF865
S3150801226039308DF82D308DF809308DF80530D0F8D4
S315080122701032044693F80B3D0F46042B1646158C6F
S315080122800ED0FF23E6E06B46304629460222F4F7D4
S315080122908FFB9DF80130102BF3D802331D44ADB2E4
S315080122A0F38BAB42EFD8338CED1AB5F5807FE8DCBA
S315080122B0D949D4F82C021BF0F9FF0E2100284FF05A
S315080122C00A02304605AB0CBF4FF00E094FF0330931
S315080122D018F0BBFF0028D4D19DF81530082BD0D1B2
S315080122E0304633210A2208AB18F0AFFF18B99DF81A
S315080122F02130082BC5D1B9F10E0F204614BF0DF1B7
S3150801230022050DF1160519F079F938B1204619F0AB
S3150801231075F9294619F0D3FC0028B2DD30460021AB
S31508012320052203AB18F091FF002800F0A2800025D2
S3150801233030460121042202AB18F087FF002800F07D
S31508012340B080304607210A220BAB18F07EFF78B918
S31508012350D4F8100200F6FC4012F07DFF9DF82D20FE
S3150801236001460DF12E001BF093FF002818BF012529
S315080123700521304612220EAB18F067FF01460028E8
S3150801238040F0B980D4F8100200F5F86011F08FFF1B
S315080123909DF8392001460DF13A001BF079FF002816
S315080123A000F0A9800125AA46B9F1330F00F08D8006
S315080123B0042230460B210DEB020318F046FF0028D4
S315080123C040F0D080D4F810020B2100F525501830C2
S315080123D014F0C3FC9DF80530022B7FF452AF002898
S315080123E03FF44FAF4288BDF80610130A43EA0222AA
S315080123F0C1F3072343EA012392B29BB29A427FF4BF
S3150801240040AFB9F1330F00F02681002D7FF439AFC3
S315080124100125B6F82090F38B4B456FD8204619F065
S3150801242028F921464FF4847204F584700AF01EFED9
S31508012430D4F8100200F52550183017F06EF8D4F8C4
S31508012440100200F52550183017F078F8002D00F025
S3150801245098800123D4F810225DB292F80B2D042A34
S3150801246040F005812046394642462B46FFF7B8FC1F
S31508012470FDE09DF80D30032B7FF403AFBDF80F5037
S315080124802B0A43EA0525ABB2A3F10B020F2A3FF645
S31508012490F8AED4F8102292F8C458ED1A18BF0125DF
S315080124A046E79DF80930022B7FF44BAFBDF80A20A9
S315080124B0C2F3072343EA0223D4F810229BB2B2F8E7
S315080124C0C2289A4218BF01253BE79DF83930002BEF
S315080124D000F09080D4F81002002100F5F86011F0A0
S315080124E0E6FE9DF8392001460DF13A001BF0D0FEB3
S315080124F000287FD05CE74FF0000A55E749460222DB
S3150801250013AB3046F4F754FA09F102010DF14E0303
S31508012510304689B29DF84D20F4F74AFA9DF84C30B9
S315080125200B2B18D0342B12D1DDF84EB0BAF1000FAF
S3150801253076D058460FF096FB384B984270D84FF430
S315080125408063ADF84E304EF29303ADF85030204615
S3150801255013A919F0F1F89DF84D30023399441FFA81
S3150801256089F958E7B9F1330F73D0002D3FF451AF0C
S31508012570D4F810020DF1160100F5A960324619F0DA
S315080125804CFBD4F81002092100F52550183014F037
S31508012590E4FB064600283FF45CAF0021102213A88D
S315080125A01BF0B8FED4F8100213AD00F6FC4012F089
S315080125B04CFF034600F1100E2A461868596808337D
S315080125C003C273451546F7D10023ADF854304FF4CD
S315080125D07F43ADF85630D4F81002FE23ADF85830D3
S315080125E0738800F52F5013A93830ADF85A30FBF728
S315080125F0DFF82EE7D4F8100200F57F7018F0FEFF19
S3150801260000283FF4D5AE0DF1160119F058FB002844
S315080126103FF7CEAE35E600BF89390308DF930400DC
S3150801262058460FF01FFB8346D4F8100200F52F50C9
S31508012630383015F0D6F8834589D2D4F8100200F55A
S315080126402F50383015F0CDF80FF00CFBCDF84E00B1
S315080126507DE70025DDE62046012118F0AAFED4F81B
S315080126601012204601F57F7119F0C2F8D0E6012D46
S315080126700CBF0020022019B0BDE8F08F2DE9F0410A
S315080126801C46064690B08846174600212C2205A806
S3150801269005AD1BF03FFE0FCC0FC50FCC0FC594E857
S315080126A0070085E80700B068002110F0ADF8054677
S315080126B0A8B330210EF0FCFE044690BB082128225F
S315080126C0169B2846F4F7D4F92146082203AB284677
S315080126D0ADF80E4004948DF80C808DF80D70F4F762
S315080126E0C7F9B068294605AA3A2310F035FC04460D
S315080126F0B8B9304619F034FB0EF0C0FA022813D9DE
S315080127000320F4F7ADF805460520F4F7B5F80521D9
S315080127100090074A03202B461CF057F804E00324CF
S3150801272002E028460EF0C0FE204610B0BDE8F08152
S31508012730E04603082DE9F043064691B08846174658
S3150801274000212C2205A81BF0E5FD304619F008FBEF
S315080127500EF094FA02280DD90320F4F781F80446FD
S315080127600520F4F789F805210090434A03202346FA
S315080127701CF02BF800218123B0688DF80D10ADF8F7
S315080127800E1004918DF80C3010F03EF8054600281D
S3150801279067D0B8F81E30B8F820401C1BA4B22146F1
S315080127A00EF086FE814600285ED14946042203AB17
S315080127B02846F4F75DF9B8F82010231F043140467E
S315080127C09BB2009589B204220EF0E5FE07F11003CB
S315080127D0984609AC07F1200E22461868596808334D
S315080127E003C273451446F7D1384610F00CFE48B9B2
S315080127F03B4605AC224618685968083303C2434567
S315080128001446F7D197F82430B0688DF83830294640
S3150801281005AA3A2310F0A0FB814628BB298C082279
S3150801282003AB2846F4F7C4F8304619F099FA0EF0C6
S3150801283025FA022815D90320F4F712F804460520CB
S31508012840F4F71AF8BDF812100090C1F3072242EA0C
S31508012850012292B2019203200521084A23461BF060
S31508012860B4FF4FF0000902E028460EF01DFE484667
S3150801287011B0BDE8F08300BFFB4603081A470308F9
S3150801288010B5044600238371C3714A68036002F5D3
S315080128900342043282600C4A8380C26000F1080256
S315080128A02061C261094A43610262094A836142623F
S315080128B0A062C362016301F1B80004F1200118F0B6
S315080128C0C3FA204610BD00BF2FBF02083E470308C2
S315080128D0D7BE02082DE9F0411D46884692B007ACDD
S315080128E0074616460FCD0FC40FCD0FC495E807004E
S315080128F098F8013084E80700022B5CD1304635216F
S31508012900082205AB18F0A1FC002854D19DF8153012
S31508012910062B50D19DF81630002B4CD19DF8174047
S31508012920042C48D130463621032203AB18F08DFC1E
S31508012930002840D19DF80D30012B3CD12246304666
S31508012940372104AB18F081FC0446A0BB9DF8113071
S31508012950022B30D105A819F077FABDF812200146E5
S31508012960C2F3072343EA02239BB29DF80E20384699
S3150801297019F08EFA2146102207A81BF0CBFC386BFA
S315080129804146B83007AA18F0B8FAA0B9384619F07E
S315080129907CFA0EF073F902280DD90320F3F760FFCC
S315080129A004460A20F3F768FF0A210090034A032028
S315080129B023461BF00AFF12B0BDE8F081434703081E
S315080129C010B504460023037780F85E304A68036130
S315080129D002F5034204320266154A4361426600F172
S315080129E06002038343834377A0664267114AC3663D
S315080129F0C0F88420104A0367C0F88820C0F88030E0
S31508012A00C4F88C00C0F890300C4BC0F8941083675A
S31508012A10E067084604F1780111F0A2F8D4F89400A9
S31508012A2004F18401B83018F00FFA204610BD00BF32
S31508012A30C7BF02086947030879BF0208F9BF020838
S31508012A402DE9F0431D46894693B007AC06469046E4
S31508012A501F460FCD0FC40FCD0FC495E8070099F88F
S31508012A60013084E80700022B40F08B80404636216E
S31508012A70032202AB18F0E9FB002840F082809DF89A
S31508012A800930012B7DD140463721042203AB18F0CA
S31508012A90DCFB002875D19DF80D30022B71D140461B
S31508012AA03821042204AB18F0D0FB002869D19DF81F
S31508012AB01130022B65D140463521082205AB18F0A5
S31508012AC0C4FB00285DD19DF81530062B59D19DF818
S31508012AD01630002B55D19DF81730042B51D1069885
S31508012AE00FF0C0F819F025FA3446BDF80E209DF806
S31508012AF00A3030613377C2F3072343EA0223BDF86C
S31508012B0012203383C2F3072343EA02237383002384
S31508012B1086F85E3001237061737706F160004FF421
S31508012B207A710FF0A1F807F1200507F11003224683
S31508012B3018685968083303C2AB421446F7D1002115
S31508012B40102207A81BF0E6FBD6F894004946B830D0
S31508012B5007AA18F0D2F9A0B9304619F009FA0EF009
S31508012B608DF802280DD90320F3F77AFE04460A20C8
S31508012B70F3F782FE0A210090034A032023461BF03D
S31508012B8024FE13B0BDE8F0836E470308F0B504468A
S31508012B90B5B000212C2205A81BF0BCFB022210A807
S31508012BA0002117F016FF10A80221FEF73FFF3F4943
S31508012BB010A818F077F810A818F0FEF8D4F89400C1
S31508012BC010A900F58E7017F0D1FB0646002863D0D0
S31508012BD035238DF80C3006238DF80D3000238DF83A
S31508012BE00E30206904238DF80F3019F0A2F90FF081
S31508012BF039F803A9049008223046F3F79DFF0546E4
S31508012C0000284BD139238DF8083094F85E303046C8
S31508012C1002A902228DF80930F3F78EFF054600282E
S31508012C203CD1304604F11E0194F85E20F3F784FF87
S31508012C30054698BB234609AD04F110072A461868CC
S31508012C405968083303C2BB421546F7D14FF2BF0391
S31508012C50D4F89400ADF836300023009300F58E7051
S31508012C60314605AA17F028FE0546B8B9204619F0D7
S31508012C707FF90EF003F8022813D90320F3F7F0FDC4
S31508012C8006460A20F3F7F8FD0A210090084A0320B0
S31508012C9033461BF09AFD04E0032502E030460EF0A8
S31508012CA003FC28460023637735B0F0BD9747030830
S31508012CB09C470308427F13B503469AB1027F62B166
S31508012CC04169D0F894004C425A8B2140009300F692
S31508012CD06C00054B0FF06BFA04E002B0BDE810403A
S31508012CE0FFF754BF02B010BDC3BF02084FF6FF730A
S31508012CF010B5044683824B68002203F50343043367
S31508012D0083610C4B0261C36100F118032062C3623F
S31508012D10094B42620363094B82624363A063C26340
S31508012D20016401F1B80004F1300118F08DF820466C
S31508012D3010BD00BF79CF0208B74703083BCF020889
S31508012D402DE9F0431D46884691B005AC06469146E5
S31508012D501F460FCD0FC40FCD0FC495E8070098F88D
S31508012D60013084E80700022B64D148463521082240
S31508012D7003AB18F06AFA00285CD19DF80D30062BD2
S31508012D8058D19DF80E30002B54D19DF80F20042AF6
S31508012D9050D14846012102AB18F057FA002849D10B
S31508012DA09DF80930022B45D104980EF05BFF19F006
S31508012DB0C0F83446306107F1100307F120052246B1
S31508012DC018685968083303C2AB421446F7D1BDF8EF
S31508012DD00A20C2F3072343EA0223B3821BF0E9FC64
S31508012DE04FF47A737062B362B06906F1180118F08C
S31508012DF0CEF90021102205A81BF08CFA306C414649
S31508012E00B83005AA18F079F8A0B930461AF092F840
S31508012E100DF034FF02280DD90320F3F721FD0446EE
S31508012E200A20F3F729FD0A210090044A03202346C4
S31508012E301BF0CBFC11B0BDE8F08300BFBC4703080B
S31508012E40F0B50546B5B000212C2205A81BF062FA9B
S31508012E50022210A8002117F0BCFD10A80221FEF7D6
S31508012E60E5FD3B4910A817F01DFF10A817F0A4FFB0
S31508012E70286C10A900F58E7017F078FA0646002816
S31508012E805ED035238DF80C3006238DF80D30286970
S31508012E90002304278DF80E308DF80F7019F049F8C4
S31508012EA00EF0E0FE03A9049008223046F3F744FE2B
S31508012EB00446002846D1AA8A01238DF80830022340
S31508012EC08DF80930C2F3072343EA0223304602A9E3
S31508012ED03A46ADF80A30F3F72FFE044690BB2B4667
S31508012EE009AC05F11007224618685968083303C268
S31508012EF0BB421446F7D14FF2BF03286CADF8363002
S31508012F000023009300F58E70314605AA17F0D4FC0C
S31508012F100446B8B928461AF00DF80DF0AFFE022896
S31508012F2013D90320F3F79CFC05460A20F3F7A4FC02
S31508012F300A210090074A03202B461BF046FC04E0B1
S31508012F40032402E030460EF0AFFA204635B0F0BD54
S31508012F50DF470308E447030813B50446006C2169F3
S31508012F6000940022044B00F66C000FF00FF90023C1
S31508012F70236102B010BD00BF75CF020808B503482A
S31508012F8040F65A411BF01FFCFEE700BF0148030843
S31508012F90F8B504460F4640F8041B40F6C41204F17E
S31508012FA08B011AF09CF9354B00256366A36604F17B
S31508012FB07006C82307F50441A4F86C302566234634
S31508012FC03046AC312E4A0EF011FD20684FF0004311
S31508012FD0C4F8803084F8845084F8855084F8865083
S31508012FE0A4F8885084F88A5084F84F5A84F8505ABD
S31508012FF084F8515A84F8525AC4F8545AC4F8585A9B
S31508013000C4F85C5AC4F8605AC4F8645AC4F8685AD1
S31508013010C4F86C5AC4F8705AC4F8745AC4F8785A81
S3150801302028B9184840F227211BF0CDFBFEE7164BBD
S31508013030224616491C600DF0F9FD224620681449FE
S315080130400DF03FFE206801210DF043FE224620685F
S3150801305010490DF054FF294620681BF059FC3046EB
S315080130600EF0E7FC84F8885AC4F87C5A04F52860FF
S31508013070294608221BF04EF92046F8BD00F8FF073D
S31508013080ADD002080148030870F000201DD00208DF
S31508013090DBD102088FD00208014B1868704700BFC0
S315080130A070F0002090F8513AF7B504460D4643B33F
S315080130B0071D38461AF0BAF918BB712300932B7904
S315080130C06E7A01932046104980220623C6F34006EC
S315080130D019F0D0FFA8B9384629682A791AF0ABF948
S315080130E078B995F906200096204608496FF07F03BE
S315080130F019F0C0FF28B9204603B0BDE8F04019F021
S3150801310096BF03B0F0BD00BF6B48030870480308BB
S315080131102DE9FF4116460AAA52F8045B0446043013
S315080131200F46984603921AF081F988B9CDF80080BE
S31508013130204609493A46334619F09CFF40B92046CC
S315080131402946039A19F07FFF10B9204619F06FFF37
S3150801315004B0BDE8F08100BF7A48030810B50446FB
S315080131608CB071B391F83920130103F0F00390067E
S3150801317048BF43F00103D206194A48BF43F0080382
S31508013180009291F836202046019291F93720039151
S3150801319002924FF6FF7204924A8E059291F83820F0
S315080131A0089301F1080306920993032219310823AA
S315080131B007920A910B93802107223323FFF7A8FF71
S315080131C00BE0084B01910093802106223023FFF77B
S315080131D09FFF10B1012384F884300CB010BD00BFE5
S315080131E07E480308A54803081FB5044661B10D4B7F
S315080131F0072200930B78019391F9013080210293FC
S315080132003923FFF785FF0BE0074B019100938021D6
S3150801321006223023FFF77CFF10B1012384F884309E
S3150801322004B010BD8F480308A548030807B5074B26
S3150801323011F0300F08BF026600930192002306229F
S31508013240FFF766FF03B05DF804FB00BF7C4803087F
S31508013250F0B59E460B0606460D46BDF8147028D5F0
S31508013260C1F301146CB920460C214143124C0B5988
S31508013270934208D001300928F6D13046294605225D
S3150801328013E0062211E0214488684C6810F0010F0A
S315080132904FEA600001D031580C5905973044294648
S315080132A07346A446BDE8F0406047BDE8F040FFF725
S315080132B0BDBF0720F0BD00BFA4F2020870B5002308
S315080132C088B08DF8133005930693079305AB0093E1
S315080132D006AB019307AB1646029304460DF1130399
S315080132E0084611461D4A1AF08CFA9DF81310B04289
S315080132F001F00F0518D1BDF81C3020460093059A38
S31508013300069BFFF7A5FF94F88A3033B19D421EBF8D
S31508013310D4F85C3A0133C4F85C3A0F2D14BF6B1C20
S31508013320012384F88A3003E020460922FFF77EFF4D
S3150801333003280CD15DB194F886300BB984F8865010
S31508013340B4F888200123AB401343A4F88830D4F895
S31508013350583A0133C4F8583A08B070BD9248030880
S3150801336070B500240C2363430C4D5E59964207D071
S3150801337001347B2CF6D10D22BDE87040FFF756BF0C
S315080133802B449C685B6814F0010F4FEA640401D072
S315080133900559EB582044BDE87040184758F3020810
S315080133A038B50446D4F88030002B00F0D58013DAFE
S315080133B020680CF071FF082896BF684B77221A5CC3
S315080133C080212046FFF732FF002840F0C680D4F856
S315080133D0803023F00043BCE098050CD520468021B7
S315080133E06022FFF7BDFF002840F0B780D4F880308F
S315080133F023F40073ADE013F480650CD020468021D8
S315080134006122FFF7ADFF002840F0A780D4F880308D
S3150801341023F480639DE0190741D594F8503A33B9EE
S31508013420204680214322FFF79BFF98B338BD2068C9
S31508013430F3F704FA0138012888BF84F8505A20683E
S31508013440F3F7FCF905281DD120680DF0D0FFC8B1A6
S3150801345094F8881AB1B9D4F88030206823F010039B
S31508013460C4F880300DF092FF204680216822FFF7CC
S31508013470DDFE002871D1204680214222FFF770FF28
S3150801348000286AD1204680214922FFF769FF0028D2
S31508013490C6D038BDD4F8803023F0080359E0DA06DF
S315080134A00BD5204680214822FFF75AFF002854D120
S315080134B0D4F8803023F010034BE09D060BD5204647
S315080134C080214722FFF74CFF002846D1D4F88030E7
S315080134D023F020033DE098070AD020468021632285
S315080134E0FFF73EFFC8BBD4F8803023F0030330E072
S315080134F013F0C00F0AD0204680215222FFF730FF71
S3150801350058BBD4F8803023F0C00322E0D9050DD585
S315080135102046802141F20D52FFF722FFE8B9D4F87F
S31508013520803023F4807343F0804312E05A000AD5B1
S31508013530204680215A22FFF713FF70B9D4F880304C
S3150801354023F0804305E013F4C05F3FF42BAF23F467
S31508013550C053C4F8803025E738BD38BDFF48030895
S31508013560F0B59E46BDF8146000250C246C430E4F39
S31508013570E359934207D001352E2DF6D10D22BDE828
S31508013580F040FFF753BE3C44A568646815F0010F87
S315080135904FEA650501D047593C59059628447346B3
S315080135A0A446BDE8F04060477CF00208F0B59E46A7
S315080135B0BDF8146000250C246C430E4FE359934261
S315080135C007D00135062DF6D1BDE8F0400D22FFF7EB
S315080135D02DBE3C44A568646815F0010F4FEA6505E0
S315080135E001D047593C59059628447346A446BDE877
S315080135F0F040604734F00208F0B59E46BDF8146005
S3150801360000250C246C430E4FE359934207D001352C
S31508013610062DF6D1BDE8F0400D22FFF707BE3C4462
S31508013620A568646815F0010F4FEA650501D0475989
S315080136303C59059628447346A446BDE8F0406047C0
S3150801364010F3020873B5002202AC44F8042D0646AD
S315080136500D461846BDF81810084A23461AF0D1F83F
S3150801366000282946304603DD019AFFF779FE02E074
S315080136700922FFF7DBFD02B070BD00BF7C480308D5
S31508013680F0B587B006AC002244F80C2DBDF83070B1
S3150801369004AA009205AA019206460D46184639461D
S315080136A00B4A23461AF0ADF8B84209D1BDF81430D1
S315080136B0304600932946039A049BFFF751FF04E01D
S315080136C0304629460922FFF7B1FD07B0F0BD00BF14
S315080136D093480308F0B587B006AC002244F80C2DD0
S315080136E0BDF8307004AA009205AA019206460D4655
S315080136F0184639460B4A23461AF083F8B84209D1C7
S31508013700BDF81430304600932946039A049BFFF707
S315080137104DFF04E0304629460922FFF787FD07B029
S31508013720F0BD00BF93480308F0B587B006AC002288
S3150801373044F80C2DBDF8307004AA009205AA01922E
S3150801374006460D46184639460B4A23461AF059F8D5
S31508013750B84209D1BDF81430304600932946039A78
S31508013760049BFFF749FF04E0304629460922FFF783
S315080137705DFD07B0F0BD00BF93480308F7B51746CE
S3150801378002AD002205F8012D04460E461846BDF87D
S3150801379020100C4A2B461AF034F800280ADD206856
S315080137A09DF907100DF058FB204631463A46FFF7BA
S315080137B0D7FD04E0204631460922FFF737FD03B05D
S315080137C0F0BD00BF97280308F7B5174602AE0022D9
S315080137D046F8042D04460D461846BDF820100F4A32
S315080137E033461AF00EF8002811DD20689DF80410FA
S315080137F00DF012FB28B9204629463A46FFF7B0FDD7
S315080138000AE019F0BBFB29460246204602E020469B
S3150801381029460922FFF70AFD03B0F0BD7C480308D3
S31508013820F7B5174602AE002206F8012D04460D46E5
S315080138301846BDF82010124A334619F0E2FF00284F
S3150801384010DD9DF8071021B102290FD82068012142
S3150801385000E020680DF096F9204629463A46FFF71A
S315080138607FFD0BE020462946092205E0072019F0CD
S3150801387085FB294602462046FFF7D8FC03B0F0BD72
S31508013880A5480308F7B51746B0F86C2002AD25F828
S31508013890022D04460E461846BDF820100B4A2B4643
S315080138A019F0AFFF002809DDBDF806302046A4F857
S315080138B06C3031463A46FFF753FD04E0204631465F
S315080138C00922FFF7B3FC03B0F0BD00BF435003085C
S315080138D0F7B5174690F8502A02AD05F8012D0446AA
S315080138E00E461846BDF820100B4A2B4619F089FFDB
S315080138F0002809DD9DF80730204684F8503A3146FC
S315080139003A46FFF72DFD04E0204631460922FFF726
S315080139108DFC03B0F0BD00BF41470308F0B585B083
S3150801392004AE1746002206F8012D04460D46184630
S31508013930BDF828101B4A334619F063FF00281CDD21
S315080139409DF80F30012B0BD01BD3022B1FD1B4F8D6
S315080139506C2000942068A16E134BF2F763FF07E011
S31508013960B4F86C2000942068A16E104BF2F74EFF54
S3150801397070B9002384F8843003E0204629460922D9
S315080139800BE0204629463A46FFF7EAFC07E00720FE
S3150801399019F0F4FA294602462046FFF747FC05B016
S315080139A0F0BD00BFA5480308A3D0020899D00208B4
S315080139B073B504460D4618461646BDF81810104A42
S315080139C00DF1060319F01DFF002811DD2068BDF869
S315080139D006100DF04AFA28B9204629463246FFF75D
S315080139E0BFFC0AE019F0CAFA29460246204602E057
S315080139F0204629460922FFF719FC02B070BD00BF0F
S31508013A004350030873B504460D4618461646BDF8D5
S31508013A1018100F4A01AB19F0F4FE002810DD2068D2
S31508013A2001990DF002FA28B9204629463246FFF7D0
S31508013A3097FC0AE019F0A2FA29460246204602E056
S31508013A40204629460922FFF7F1FB02B070BD00BFE7
S31508013A506C520308F7B5174602AD002205F8012D89
S31508013A6004460E461846BDF820100D4A2B4619F095
S31508013A70C8FE002809DD9DF80730204684F8513A2A
S31508013A8031463A46FFF76CFC07E0062019F076FA4C
S31508013A90314602462046FFF7C9FB03B0F0BD00BF19
S31508013AA041470308F7B5174602AD002205F8012D6F
S31508013AB004460E461846BDF820100E4A2B4619F044
S31508013AC0A0FE00280BDD20689DF807100DF0DFF831
S31508013AD030B9204631463A46FFF742FC07E0062050
S31508013AE019F04CFA314602462046FFF79FFB03B010
S31508013AF0F0BD00BF414703082DE9F7434FF0000920
S31508013B0002AD05F8019D04460F4618469046BDF8D4
S31508013B102810204A2B4619F074FE48452EDD2068E8
S31508013B209DF80750F2F78AFE10F1FF3018BF012001
S31508013B30A84205D1204639464246FFF711FC26E040
S31508013B409DF80760206856B101210DF01FFCD4F8D5
S31508013B507C3A054684F8889A6BB11B6809E03146B8
S31508013B600DF014FCD4F87C3A054684F8886A13B13A
S31508013B705B6803B19847002DDCD000E0062528468E
S31508013B8019F0FCF9394602462046FFF74FFB03B008
S31508013B90BDE8F08341470308F7B5174602AE002290
S31508013BA046F8042D04460D461846BDF82010184A55
S31508013BB0334619F026FE002823DD019B032B14D872
S31508013BC0DFE803F0020E060A20680DF02FFB0BE072
S31508013BD020680DF035FB07E020680DF043FB03E094
S31508013BE0206800210DF027FB28B9204629463A46C8
S31508013BF0FFF7B6FB0AE019F0C1F929460246204645
S31508013C0002E0204629460922FFF710FB03B0F0BD62
S31508013C107C480308F7B5174602AE002246F8042D7C
S31508013C2004460D461846BDF820100F4A334619F0CA
S31508013C30E8FD002811DD019979B120680DF0AFFA88
S31508013C4028B9204629463A46FFF78AFB0AE019F0C1
S31508013C5095F929460246204602E0204629460922C8
S31508013C60FFF7E4FA03B0F0BD144F0308F0B585B0C9
S31508013C7004AD1746002245F8082D03AA009204460A
S31508013C800E461846BDF828100C4A2B4619F0B9FD00
S31508013C9000280CDD039B082B09D1206802990DF039
S31508013CA0F5F9204631463A46FFF75AFB04E0204625
S31508013CB031460922FFF7BAFA05B0F0BDBF4D030830
S31508013CC0F0B585B004AE1746002246F8082D03AABA
S31508013CD0009204460D461846BDF82810104A334688
S31508013CE019F08FFD002814DD039A632A11D820687C
S31508013CF00299D2B20DF03BFA28B9204629463A462E
S31508013D00FFF72EFB0AE019F039F929460246204643
S31508013D1002E0204629460922FFF788FA05B0F0BDD8
S31508013D20BF4D0308F7B5174602AD002245F8042D25
S31508013D3004460E461846BDF820100B4A2B4619F0C4
S31508013D4060FD002809DD206801990DF04DFA20462D
S31508013D5031463A46FFF704FB04E02046314609227C
S31508013D60FFF764FA03B0F0BD05540308F7B5174623
S31508013D7002AD002245F8042D04460E461846BDF844
S31508013D8020100B4A2B4619F03CFD002809DD206856
S31508013D9001990DF032FA204631463A46FFF7E0FA24
S31508013DA004E0204631460922FFF740FA03B0F0BD88
S31508013DB005540308F7B5174602AD002205F8012D8B
S31508013DC004460E461846BDF820100D4A2B4619F032
S31508013DD018FD00280ADD20689DF807100DF0F2F994
S31508013DE0204631463A46FFF7BBFA07E0062019F0A6
S31508013DF0C5F8314602462046FFF718FA03B0F0BD6A
S31508013E00A5480308F0B5054689B00F4600680021A4
S31508013E101C4604910591069107910CF06CFF064624
S31508013E2048B305AB009306AB019307AB0293204653
S31508013E30BDF838101B4A04AB19F0E3FC3046049967
S31508013E40BDF814200DF084F8044630461CBB012148
S31508013E500DF073F8286831460CF03FFF044658B94F
S31508013E60D5F8683A0133C5F8683A3B0716D02846AB
S31508013E70394622460BE00324D5F8783A2046013321
S31508013E80C5F8783A19F07AF8394602462846FFF70E
S31508013E90CDF9044602E00DF045F8EDE7204609B0F4
S31508013EA0F0BD00BF96480308F0B5002289B0054663
S31508013EB00F46006801211C46049205920692079254
S31508013EC00CF019FF064628B305AB009306AB019320
S31508013ED007AB02932046BDF838101A4A04AB19F00D
S31508013EE090FC30460499BDF814200DF031F80446CB
S31508013EF000BB286831460CF0F0FE044658B9D5F8DF
S31508013F00643A0133C5F8643A3B0717D0284639465F
S31508013F1022460BE00324D5F8783A20460133C5F842
S31508013F20783A19F02BF8394602462846FFF77EF902
S31508013F30044603E030460CF0F5FFECE7204609B0ED
S31508013F40F0BD00BF96480308F7B5174602AD002233
S31508013F5005F8012D04460E461846BDF820100C4AF0
S31508013F602B4619F04EFC00280ADD20689DF807103B
S31508013F701AF0CEFC204631463A46FFF7F1F904E03D
S31508013F80204631460922FFF751F903B0F0BD00BFBB
S31508013F9041470308F7B5174602AD002205F8012D7A
S31508013FA004460E461846BDF820100D4A2B4619F050
S31508013FB028FC00280CDD9DF80710206881F0010116
S31508013FC00CF087FE204631463A46FFF7C9F904E068
S31508013FD0204631460922FFF729F903B0F0BD00BF93
S31508013FE0414703082DE9F3478946002402A90546F6
S31508013FF001F8034D006892469846BDF828600CF012
S3150801400094FE07469DF80530FBB1286837F8141069
S315080140100CF086FE28BB9DF805300134013B8DF86E
S315080140200530EFE740463146174A0DF1060319F008
S31508014030E8FB071E0CDD2868BDF806100CF06BFEC0
S3150801404078B9F61BB844B6B20134012EEAD801E0B4
S31508014050062006E0284649465246FFF781F90646F4
S315080140600DE018F08BFF494602462846FFF7DEF8B1
S31508014070064624B1284680215246FFF771F9304693
S3150801408002B0BDE8F08700BF43500308F7B51746ED
S3150801409002AD002205F8012D04460E461846BDF864
S315080140A02010134A2B4619F0ACFB002813DD94F8AF
S315080140B04F5A9DF807300DB183F00105314684F852
S315080140C04F3A20463A46FFF74BF9064665B120684E
S315080140D016F01EF908E0062018F050FF3146024690
S315080140E02046FFF7A3F80646304603B0F0BD00BFE9
S315080140F04147030873B504460D4618461646BDF8EA
S3150801410018100C4A0DF1070319F07BFB00280ADD8C
S3150801411020689DF807100DF04CF8204629463246CE
S31508014120FFF71EF904E0204629460922FFF77EF823
S3150801413002B070BD4147030873B5002202AC04F80A
S31508014140012D06460D461846BDF818100B4A23469A
S3150801415019F057FB002806DD9DF80730012B0CBF27
S315080141600D20072000E0062018F008FF2946024620
S315080141703046FFF75BF802B070BD00BFA5480308DB
S315080141802DE9FF4704460068894690461F46BDF853
S3150801419030500CF09FFE6DB3002303930DF10B0312
S315080141A000934FF07F0A384629461E4A03AB8DF81D
S315080141B00BA019F026FB061E0BDC384629461A4ABF
S315080141C003AB8DF80BA019F01CFB061E01DC0620BB
S315080141D017E09DF90B2020687F2A039902D10CF07C
S315080141E057FE01E00CF05FFEAD1B3744ADB2002867
S315080141F0D1D006E0204649464246FFF7B1F80546C2
S315080142000CE018F0BBFE494602462046FFF70EF8B9
S315080142108021054642462046FFF7A2F8284604B003
S31508014220BDE8F087994803089F48030873B5044613
S315080142300D4618461646BDF818100C4A0DF1070327
S3150801424019F0DFFA00280ADD20689DF807100CF03E
S315080142504EFE204629463246FFF782F804E02046FC
S3150801426029460922FEF7E2FF02B070BD414703085D
S31508014270F7B5174602AE002206F8012D04460D468B
S315080142801846BDF82010174A334619F0BAFA00281D
S3150801429021DD4FF000019DF807302068C3F3C00205
S315080142A062F30001C3F3800262F34101C3F34002E2
S315080142B062F3820163F3C3010CF03CFF28B920467F
S315080142C029463A46FFF74CF80AE018F057FE294600
S315080142D00246204602E0204629460922FEF7A6FFA5
S315080142E003B0F0BDA5480308F7B5174602AD00228D
S315080142F005F8012D04460E461846BDF820100C4A4D
S315080143002B4619F07EFA00280ADD9DF80710206869
S315080143100CF0AAFE204631463A46FFF721F804E09A
S31508014320204631460922FEF781FF03B0F0BD00BFE2
S31508014330A5480308F7B5174602AD002245F8042D2E
S3150801434004460E461846BDF820100B4A2B4619F0AE
S3150801435058FA002809DD206801990CF08EFE2046DE
S3150801436031463A46FEF7FCFF04E02046314609226B
S31508014370FEF75CFF03B0F0BD05540308F7B5174611
S3150801438002AD002205F8012D04460E461846BDF871
S3150801439020100C4A2B4619F034FA00280ADD206849
S315080143A09DF807100CF039FF204631463A46FEF7CC
S315080143B0D7FF04E0204631460922FEF737FF03B04E
S315080143C0F0BD00BFA5480308F7B5174602AD0022A0
S315080143D005F8012D04460E461846BDF820100C4A6C
S315080143E02B4619F00EFA00280ADD20689DF80710F9
S315080143F00CF041FF204631463A46FEF7B1FF04E08C
S31508014400204631460922FEF711FF03B0F0BD00BF71
S31508014410A5480308F7B5174602AD002205F8012D90
S3150801442004460E461846BDF820100C4A2B4619F0CC
S31508014430E8F900280ADD20689DF807100CF023FF2B
S31508014440204631463A46FEF78BFF04E020463146C0
S315080144500922FEF7EBFE03B0F0BD00BFA54803082D
S31508014460F7B5174602AE002206F8012D04460D4699
S315080144701846BDF820101C4A334619F0C2F900281F
S3150801448016DD9DF80730072B0BD8DFE803F0171761
S31508014490041919060608012113E0032111E0042174
S315080144A00FE0072018F06AFD29460246204602E079
S315080144B0204629460922FEF7B9FE13E0002100E04D
S315080144C0022120680CF0DEFB03462BB9204629465B
S315080144D03A46FEF745FF05E01D2BE3D1204629465E
S315080144E01522E8E703B0F0BDA5480308F7B5174656
S315080144F002AD002245F8042D04460E461846BDF8BD
S3150801450020100B4A2B4619F07CF9002809DD206892
S3150801451001990CF060FE204631463A46FEF720FF27
S3150801452004E0204631460922FEF780FE03B0F0BDBD
S3150801453005540308F7B5174602AD002205F8012D03
S3150801454004460E461846BDF820100C4A2B4619F0AB
S3150801455058F900280ADD20689DF807100CF055FE69
S31508014560204631463A46FEF7FBFE04E02046314630
S315080145700922FEF75BFE03B0F0BD00BFA54803089C
S3150801458073B504460D4618461646BDF818100F4A67
S315080145900DF1070319F035F9002810DD9DF80730EC
S315080145A0206823B10A4922461AF0D8F901E01AF01F
S315080145B0DAF9204629463246FEF7D2FE04E02046BD
S315080145C029460922FEF732FE02B070BD41470308AB
S315080145D0F1D10208F7B5174602AE002206F8012DF9
S315080145E004460D461846BDF820100F4A334619F001
S315080145F008F9002811DD20689DF907101AF08BF9D2
S3150801460028B9204629463A46FEF7AAFE0AE018F0D6
S31508014610B5FC29460246204602E0204629460922DB
S31508014620FEF704FE03B0F0BD97280308F7B5174651
S3150801463002AE002206F8012D04460D461846BDF8BD
S3150801464020100F4A334619F0DCF8002811DD2068DE
S315080146509DF807101AF068F928B9204629463A46FE
S31508014660FEF77EFE0AE018F089FC29460246204636
S3150801467002E0204629460922FEF7D8FD03B0F0BD1F
S31508014680A5480308F7B5174602AE002206F8012D1C
S3150801469004460D461846BDF820100F4A334619F050
S315080146A0B0F8002811DD20689DF807101AF049F9BD
S315080146B028B9204629463A46FEF752FE0AE018F07E
S315080146C05DFC29460246204602E020462946092283
S315080146D0FEF7ACFD03B0F0BDA54803082DE9FF417F
S315080146E0002704AD45F8087D904603AA00920446C2
S315080146F00E461846BDF82810144A2B4619F081F8BB
S31508014700B8421BDD039B082B18D804F528653946E2
S315080147100822284619F0FEFD28460299039A08F050
S31508014720A5FCD4F87C3A1BB1DB680BB1284698473F
S31508014730204631464246FEF713FE04E0204631463E
S315080147400922FEF773FD04B0BDE8F081BF4D0308E9
S3150801475013B5044694F8861009B3204641F0800142
S315080147600B22FEF763FD002842D194F88630B4F88F
S31508014770881001229A4021EA0202A4F8882012B977
S3150801478084F886200BE00E2B9ABF0133DBB2012396
S3150801479042FA03F1C907F6D584F88630DAE794F8C0
S315080147A0843063B1134B2046009300230193802183
S315080147B006223023FEF7ACFCD0B984F8840094F8BD
S315080147C085307BB120681AF0DBF80B4B019000931A
S315080147D020468021062241F20123FEF799FC38B9C9
S315080147E084F88500204602B0BDE81040FEF7D8BD22
S315080147F002B010BDA54803084147030807B513468B
S31508014800044A0092026E01920622FEF781FC03B069
S315080148105DF804FB7C4803081FB51346054A009258
S3150801482004220192032202920622FEF771FC05B0C8
S315080148305DF804FB7B48030807B51346044A009252
S31508014840032201920622FEF763FC03B05DF804FB1E
S315080148507C48030807B51346044A009200220192D0
S315080148600622FEF755FC03B05DF804FB7C480308F5
S3150801487073B5144606460D46F1F7EEFF054B019052
S3150801488000933046294606222346FEF741FC02B02C
S3150801489070BD00BF144F030807B51346044A0092BA
S315080148A0012201920622FEF733FC03B05DF804FBF0
S315080148B0A548030807B51346044A00920422019243
S315080148C00622FEF725FC03B05DF804FBA54803089C
S315080148D0F0B5164604460F4685B002AD294600686E
S315080148E00CF0B4FA054B20468DE828003946062215
S315080148F03346FEF70DFC05B0F0BD00BF6C52030848
S3150801490007B51346044A0092002201920622FEF7D1
S31508014910FFFB03B05DF804FB41470308F7B50546FD
S3150801492000680F4616460CF073FAA8B10A2808D88B
S315080149304FF4FA6404FB00F202F55C2202F53462D4
S315080149400DE019280AD841F28832504302F50F12B0
S3150801495002F62802024402E0064A00E00022064B5B
S31508014960019200932846394606223346FEF7D0FBC4
S3150801497003B0F0BDCC3F0D000554030873B50446DA
S31508014980006815460E460CF043FA054B0190009354
S315080149902046314606222B46FEF7BAFB02B070BD09
S315080149A0A548030873B50446006815460E460CF07B
S315080149B0DBF8054B019000932046314606222B462B
S315080149C0FEF7A6FB02B070BD9728030873B5044627
S315080149D0006815460E460CF03BFA054B019000930C
S315080149E02046314606222B46FEF792FB02B070BDE1
S315080149F097280308F7B5044600680E4615460CF0D5
S31508014A0087FA0B4F10B10097012305E020680CF0D7
S31508014A1084FA009710B10223019300E00190204621
